:100000000C945E0F0C94860F0C94860F0C94860F44
:100010000C94860F0C94860F0C94860F0C94860F0C
:100020000C94860F0C94860F0C9490140C944C66D0
:100030000C94CA680C947B660C94860F0C94EF1495
:100040000C947E140C94860F0C94D66C0C94860F32
:100050000C94860F0C94860F0C94860F0C94860FCC
:100060000C943C690C9437150C94E5660C947C69EF
:100070000C94860F0C94860F0C94860F0C94860FAC
:100080000C94860F0C94860F0C94860FD016D41601
:1000900097169D16A316A316A316C816CC16D0162F
:1000A000D416D816DC16E0167F3D3F3D4A3D593D3B
:1000B0005F3D633D683D55426B4279428E429C42B2
:1000C000AB42BD42E3420C431A4340435E436C43A0
:1000D0007A438843396123611D6127612C61326154
:1000E000206136613B61DE6AE46AF16AFA6A106B8C
:1000F000296B3C6B4B6B5F6B746B7D6B9A6BA06B6E
:10010000A86BAD6BB26B1A6C246CBA6BC16BCB6B0A
:10011000D56BDB6BDF6BE66B016C066C0B6C136CE9
:10012000EA6AEA6BF16BF96B204F6C6420566572DA
:1001300073696F6E20454550524F4D202020434833
:1001400045434B2053455454494E47532F43414C4C
:10015000494200416C61726D732044697361626C45
:10016000656400506C656173652052657365742029
:100170005377697463686573005468726F74746C44
:1001800065206E6F742069646C65005265736574D8
:10019000207468726F74746C6500454550524F4D01
:1001A000206C6F77206D656D004C4F4144494E4780
:1001B000006D537461636B206F666C6F77006D53D5
:1001C0007461636B2075666C6F77004D45535341C6
:1001D000474500414C45525400707265737320616D
:1001E0006E79204B657900507265737320616E796A
:1001F000206B657920746F20736B697000414C45EA
:10020000525400034F4646414253525573525525AE
:10021000454C73454C25544873544825414C734113
:100220004C2550312050312550322050322550334A
:100230002050332500544852525544454C454944BA
:100240003049443149443241494C47454154524E6A
:1002500053573153573253573353573453573553FA
:1002600057365357375357385357395357415357C6
:1002700042535743002D2D2D004348002D2D2D2096
:10028000000450312020503220205033202048419B
:100290004C4646554C4C43594331435943324359DC
:1002A000433350504D3150504D3250504D335050DB
:1002B0004D3450504D3550504D3650504D375050B4
:1002C0004D38434831204348322043483320434887
:1002D000342043483520434836204348372043489C
:1002E000382043483920434831304348313143486E
:1002F0003132434831334348313443483135434840
:10030000313633504F5347563120475632204756E7
:100310003320475634204756352047563620475617
:100320003720002D2D2D2D0000006428100703011B
:1003300052554420454C45205448522041494C20B8
:100340000001020304010302040402030104030286
:10035000014F4E20004F4646001B1E272D36394BBD
:100360004E636C7278878D939CB1B4C6C9D2D8E1C4
:10037000E453706C6173680080400000000000006E
:10038000000000000000000000000000000000006D
:10039000000000000000000000000000000000005D
:1003A000000000000000000000000000000000004D
:1003B000000000000000000000000000000000003D
:1003C000000000000080C0E0E0F0F8F8FCFCFCF861
:1003D000F8F8F0400000000000808080000000007D
:1003E000000000000000000000000000000000808D
:1003F000C0C0E0E0E0F0F0F0E0C00000000000C0AD
:10040000F8FFFF9F8783838383838383838383832F
:10041000838383838383838383838303838083832F
:10042000838383838383838383838383838383839C
:100430008383838383C3E3733F1F0000000080E056
:10044000F0F8FCFEFFFFFFFF7F3F1F1F0F0783C376
:10045000E1E1E0E0C0000E1F3F7F7FFFF3E0E080BE
:100460000000000000000000000080F0FCFEFFFF24
:10047000FFFF7F3F0F0301010100000080F0FEFF3E
:10048000FFC7C1C1C1C1C1C1C1C1C1C1C1C1C1C118
:10049000C1C1C1C1C1C1C1C101C1F0FEFF3F0F0750
:1004A0000F0D0D0D1D19191919313131317161619E
:1004B00061E1C1C1C18100000080E0F8FCFFFFFFE5
:1004C000FF2F170F038180C0E0F0F8FCFEFFFFFF55
:1004D000FFFFFF7F01000000000000000101030793
:1004E000070E1E1C3870E0F0F8FEFFFF7F1F0F03A1
:1004F00000010000000000000000000000000000FB
:1005000000000000000000000000000000000000EB
:1005100000000000000000000000000000000000DB
:1005200000000000000000000000000000000000CB
:1005300000000000000000007EFFFFFFFFFFFFFB48
:10054000F8FCFCFEFF7F3F1F0F07C3FFFFFFFFFF0D
:10055000FF7F070000000000000000000000000016
:1005600000C0E0F8FEFFFF7F1F0F1F3D7CF8F8F092
:10057000E08000000000000000000000000000001B
:10058000000000000000000000000000000000006B
:10059000000000000000000000000000000000005B
:1005A000000000000000000000000000000000004B
:1005B0000000000000000000000001010101010333
:1005C0000707070301000000E0FCFFFFFFFFFF1F1C
:1005D000030000000000000000000000C0F078DE12
:1005E0002713090E070300000000000000000103AC
:1005F0000F7FFFFC7878F80000000000000000008A
:1006000000008080808080808080800080800080EA
:10061000800000000000000080808080808080805A
:1006200080808080808080808080000000000000CA
:1006300000000000000000000000000000000000BA
:10064000000000000080F0FEFFFFFFFF3F0F0100F1
:1006500000000000000000C0E0381E0F0300010091
:10066000000000000000000000000000000000008A
:100670000000000000030301000000000000000073
:1006800000000E0E02020202020303000F0F000F11
:100690000F080808080808080F0F08080808080FBE
:1006A0000F000000000F0F0000000000000000001D
:1006B000000000000000000000000000000000003A
:1006C000000000C0F8BFFFFFFF1F7F010000000017
:1006D00000000000F0FCFF7F783000000000000008
:1006E000000000000000000000000000000000000A
:1006F00000000000000000000000000000000000FA
:1007000000000000000000000000000000000000E9
:1007100000000000000000000000000000000000D9
:1007200000000000000000000000000000000000C9
:1007300000000000000000000000000000000000B9
:1007400000301C070E0F0701000000000000000031
:100750000000000000000000000000000000000099
:100760000000000000000000000000000000000089
:100770000000000000000000000000204D4F443A3F
:10078000204A4554492020202020002053564E3A2C
:1007900020657239782D723739310054494D453A08
:1007A0002032313A31323A333900444154453A200B
:1007B00031312E30352E3230313300564552533AD6
:1007C0002056312E3635352D4D696B650022047C5F
:1007D0005E54546D0003457870457846466E654D0D
:1007E00065644372730011544F54000153544B110C
:1007F0005354250001544D4511545357005354414F
:1008000054004A45544900035B4D454E555D2074E4
:100810006F207265667265736800746D61696E0F32
:100820006D7300746D7231204A69747465720F754E
:100830007300746D72314C6174206D696E0F757345
:1008400000746D72314C6174206D61780F757300A6
:100850005354415432004D6F64650043726F73739B
:100860005472696D00456E61626C652050504D5345
:10087000494D0042616E6447617000537469636B57
:100880005363726F6C6C00506F745363726F6C6C57
:1008900000416C61726D205761726E696E67004D28
:1008A000656D6F7279205761726E696E670044657D
:1008B0006661756C74205377005468726F74746C41
:1008C00065205761726E696E670053706C61736862
:1008D000204E616D650053706C61736820736372A4
:1008E00065656E004C69676874206F6E2053746B89
:1008F000204D76004C69676874206F6666206166DB
:10090000746572004261636B6C6967687420696E1C
:1009100076657274004C69676874207377697463D4
:100920006800466C617368206F6E206265657000B8
:100930004265657020636F756E74646F776E004DED
:10094000696E7574652062656570005468726F74B5
:10095000746C65207265766572736500496E6163BB
:1009600074697669747920616C61726D136D0042EF
:10097000617474657279207761726E696E67004385
:100980006F6E7472617374002048617074696320C3
:10099000537472656E6774680020537065616B658F
:1009A0007220506974636800566F6C756D65000A3B
:1009B00042656570657220202020506953706B720B
:1009C000202020204265657072566F69636550690A
:1009D00053706B566F69636500536F756E64204D7D
:1009E0006F646500065175696574204E6F4B6579BB
:1009F000207853686F727453686F7274204E6F72F0
:100A00006D20204C6F6E672020784C6F6E67200041
:100A1000426565706572004F776E6572204E616D3C
:100A20006500524144494F20534554555000036DD1
:100A30006F64650A25207372632020737700436119
:100A40006C004D756C7469706C6965720003636845
:100A50003163683263683363683400036F6666200D
:100A60002B3D203A3D0007536C617665000003037F
:100A7000030300545241494E4552005645525349D2
:100A80004F4E005472696D2D202B0005204D656E70
:100A900075204578697420446F776E20202055704A
:100AA0005269676874204C65667400444941470088
:100AB000424700414E4100034D4F56452053544993
:100AC000434B532F504F54530005534554204D4929
:100AD00044504F494E5400035B4D454E555D2054E4
:100AE0004F2053544152540043414C4942524154C7
:100AF000494F4E000966726565004D4F44454C53A1
:100B0000454C00434F4C20446972656374696F6EB5
:100B10000041494C20446972656374696F6E0045F9
:100B20004C4520446972656374696F6E0053776148
:100B300073682052696E6700436F6C6C65637469FB
:100B4000766500062D2D2D202020313230202020EA
:100B500031323058202031343020202039302020CC
:100B60002020005377617368205479706500004835
:100B7000454C4920534554555000464D00464D3094
:100B80000F52455441004D4F444553005472696D16
:100B90007300537769746368000003464C204D4F1F
:100BA00044450001524554410044454C45544520BC
:100BB0004D4F44454C0F5B4D454E555D00543254EE
:100BC000685472696700547261696E657200452EDF
:100BD000204C696D6974730003504F534E454700B4
:100BE00053686966742053656C0050504D20317312
:100BF00074204368616E004C50342F4C50352020D7
:100C000044534D326F6E6C792044534D322F445310
:100C10004D580044534D20547970650053656E64FF
:100C2000205278204E756D626572205B4D454E55A1
:100C30005D0050504D2046724C656E0D6D536563DE
:100C4000000B52784E756D000434434820364348FB
:100C5000203843482031304348313243483134430F
:100C600048313643480013755300117553656300CE
:100C700050504D20202050585820202044534D32B1
:100C8000202050504D31362050504D53494D00508A
:100C9000726F746F005245544131323300426565C2
:100CA0007020436E74005472696D205377000645BE
:100CB0007870202020457846696E6546696E65200B
:100CC000204D656469756D436F6172736500547280
:100CD000696D20496E6300542D4578706F00542D66
:100CE0005472696D000A436F756E7420446F776E9D
:100CF000436F756E742055702020005472696767C9
:100D0000657242005472696767657200566F696365
:100D10006520496E646578114D454E55004E616DF4
:100D2000650000090001000000000000000602004C
:100D30005345545550004475706C69636174696E15
:100D400067206D6F64656C0044454C455445204DEB
:100D50004F44454C004455504C4943415445204D67
:100D60004F44454C00657870202025202073773152
:100D7000207377320000034558504F2F44520044EF
:100D8000522048696768004452204C6F77004452F3
:100D9000204D6964004472537732004472537731B6
:100DA00000576569676874004578706F00004558A2
:100DB000504F2F445200012B2A52004D49584552A2
:100DC00000032044454C455445200003204D4F5618
:100DD00045202020000320434F50592020200003AD
:100DE00020494E5345525420000320454449542085
:100DF00020200044454C455445204D49583F0003B0
:100E00005B4D454E555D0B5B455849545D0003599C
:100E100045530B4E4F005072657373205B45584924
:100E2000545D20746F2061626F7274004D61782090
:100E30006D69786572732072656163683A20333238
:100E40000002536C6F77202055700002536C6F774F
:100E50002020446F776E000244656C6179205570E4
:100E6000000244656C617920446F776E000841642C
:100E70006420202020204D756C7469706C79526557
:100E8000706C6163652000024D756C7470780002AF
:100E90005761726E696E6700025377697463680008
:100EA0004375727665000D44696666000254726986
:100EB0006D0002466C4D6F64657472696D00024688
:100EC0006978204F6666736574004F666673657453
:100ED00000466D5472696D56616C00025765696712
:100EE00068740002536F757263650045444954206D
:100EF0004D49582000494E53455254204D495820E1
:100F000000032D2D2D783E30783C307C787C663E79
:100F100030663C307C667C63312063322063332052
:100F200063342063352063362063372063382063C1
:100F300039206331306331316331326331336331AE
:100F400034633135633136000E4F6E00072D2D2D81
:100F50002D202020763E6F66732020763C6F6673CE
:100F600020207C767C3E6F66737C767C3C6F66735B
:100F7000414E44202020204F522020202020584F36
:100F8000522020202076313D3D7632207631213DA1
:100F900076322076313E7632202076313C76322011
:100FA0002076313E3D76322076313C3D76322054FB
:100FB000696D654F666600535700000343555354EF
:100FC0004F4D20535749544348455300064F4E2038
:100FD0002020204F4646202020424F5448202031D8
:100FE00035536563733330536563733630536563CC
:100FF0007356617269626C005653000720382053A3
:1010000065637331322053656373313620536563F2
:1010100073004E756D62657220566F69636520536B
:101020007700000002534146455459205357495414
:101030004348455300434C454152204D4958455380
:10104000205B4D454E555D00205245544100014303
:1010500068616E6E656C204F726465720054454D18
:10106000504C4154455300032D2D2D52746D457441
:101070006D54746D41746D52454E525544454C4506
:1010800054485241494C5031205032205033206353
:10109000312063322063332063342063352063368C
:1010A0002063372063382063392063313063313166
:1010B0006331326331336331346331356331360048
:1010C0004756000001474C4F42414C205641525375
:1010D00000434F5059205452494D205B4D454E55C9
:1010E0005D0000034C494D4954530043560043559D
:1010F00052564553005052455345540045444954B7
:101100002D3E000900435552564500032D2D2D4913
:101110004E56004756005B4D454E555D205748459D
:101120004E20444F4E4500FC46BD24EC237123F174
:10113000226E266E30BC4D2452212F252D3645DDE2
:1011400052A443384C3B546A441A24120812000833
:101150001C0808081C08000008220049002208009A
:1011600000000000227F2200000008220049002227
:1011700008000008220049002208000000227F2207
:101180000000000000082200490022080000081C9E
:101190000808081C0800065761726E3120576172FA
:1011A0006E322043686561702052696E672020535B
:1011B0006369466920526F626F7420436869727078
:1011C00020546164612020437269636B74536972B7
:1011D000656E20416C6D436C6B5261746174615437
:1011E00069636B2020486170746331486170746377
:1011F000324861707463330054696D6572005452F3
:10120000453031324147002041424344454647483A
:10121000494A4B4C4D4E4F505152535455565758C6
:10122000595A6162636465666768696A6B6C6D6E62
:101230006F707172737475767778797A3031323372
:101240003435363738395F2D2E00FEFFFDF6F7F8BE
:10125000F9FAFBFC042D2D2D2D54494D3154494DE7
:101260003242415454477672314776723247767231
:1012700033477672344776723547767236477672E0
:101280003700537769746368205761726E696E67BF
:101290000067656E7772697465206572726F72009F
:1012A000454550524F4D20466F726D617474696EA2
:1012B000670042616420454570726F6D204461741F
:1012C00061004D4F44454C2020202020004D4520FA
:1012D0002020202020202000454550524F4D206FD7
:1012E000766572666C6F7700A06080000000000079
:1012F000000000000000000000FFFF0000000000F0
:10130000001F3F00003F1F00003030FFFF3030FF64
:10131000FF30303078CCCCFFFFCCCC8C0C060F0FDC
:1013200086C0E070381C0C3CFEC7E3F33B1E0C008B
:10133000000000333B1F0F000000000000F0F81C0D
:101340000E07030000000003070E1CF8F000003039
:1013500030E0C0FCFCC0E03030C0C0C0C0FCFCC00D
:10136000C0C0C000000000000000000000C0C0C0FD
:10137000C0C0C0C0C0C0C00000000000000000002D
:101380000000000080C0E070381C0C00000000006D
:1013900000000000000000000038380000000000DD
:1013A00000000000000000000003033F3F03033F74
:1013B0003F03030C0C0C0C3F3F0C0C07030C0E07F7
:1013C000030100183C3C180F1F383133331E1E3305
:1013D0003300000000000000000000000003070EC2
:1013E0001C38300000000030381C0E0703000003DA
:1013F0000301000F0F00010303000000000F0F00A6
:101400000000000000333B1F0F0000000000000040
:10141000000000000000000000183C3C1800000024
:10142000000C0E07030100000000000000FCFE8716
:10143000C3E377FEFC00000C0EFFFF00000000007D
:10144000000C0E0783C3E77E3C00000303C3C3C345
:10145000E7FE3C0000C0E070381C0EFFFF00003FBC
:101460003F33333373E3C30000FCFEC7C3C3C78EEF
:101470000C00000303C3E3733B1F0F00003CFEE7B7
:10148000C3C3E7FE3C00003C7EE7C3C3E7FEFC00AD
:1014900000183C3C18000000000000183C3C1800FC
:1014A0000000000000C0E0F0381C0E0703303030B0
:1014B0003030303030303003070E1C38F0E0C000E0
:1014C000000C0E07030383C3E77E3C00000F1F3BA5
:1014D0003130381F0F000030303F3F303000000007
:1014E000003C3E3733313030300000303030303067
:1014F000391F0F00000303030303033F3F00000CE9
:101500001C383030381F0F00000F1F383030391FA3
:101510000F000000003F3F0000000000000F1F39D7
:101520003030391F0F0000000030381C0E07030058
:1015300000060F0F06000000000000333B1F0F00E5
:101540000000000000000103070E1C3830030303F5
:101550000303030303030330381C0E0703010000D9
:10156000000000000033330100000000003C7EE773
:10157000C3C3E77E3CF0F8DCCEC7C7CEDCF8F0FF93
:10158000FFC3C3C3C3C3E7FE3CFCFE07030303035F
:10159000070E0CFFFF030303070E1CF8F0FFFFC349
:1015A000C3C3C3C3C30303FFFFC3C3C3C3C3C303D3
:1015B00003FCFE0703C3C3C3C7CECCFFFFC0C0C03C
:1015C000C0C0C0FFFF00000303FFFF0303000000D3
:1015D0000000000303FFFF0303FFFFC0E0F0381C1F
:1015E0000E0703FFFF0000000000000000FFFF0ED9
:1015F0001CF8F81C0EFFFFFFFF3870E0C08000FFF2
:10160000FFFCFE070303030307FEFC0000000000CD
:1016100000000000003F3F0000000000003F3F3F8F
:101620003F3030303030391F0F0F1F3830303030FE
:10163000381C0C3F3F303030381C0E07033F3F3022
:10164000303030303030303F3F00000000000000CC
:10165000000F1F3830303030303F3F3F3F00000038
:101660000000003F3F000030303F3F303000000CB2
:101670001C383030381F0F00003F3F000103070EB9
:101680001C38303F3F30303030303030303F3F005A
:1016900000000000003F3F3F3F0000000103033F08
:1016A0003F0F1F3830303030381F0FFFFFC3C3C328
:1016B000C3C3E77E3CFCFE070303030307FEFCFFF6
:1016C000FFC3C3C3C3C3E77E3C3C7EE7C3C3C3C3FE
:1016D000C78E0C03030303FFFF03030303FFFF0095
:1016E0000000000000FFFFFFFF000000000000FFFF
:1016F000FFFFFF000000000000FFFF0F1F38F0E0B9
:10170000E0F0381F0F3F7FE0C08080C0E07F3F03E4
:10171000030383C3E3733B1F0F0000FFFF030303B7
:101720000300000C1C3870E0C080000000000003C3
:10173000030303FFFF000030381C0E07070E1C38A0
:1017400030000000000000000000003F3F000000EB
:1017500000000000000F1F383033371E1C3F333F9E
:101760003F000003070E1C38300C1C38303030307E
:10177000391F0F000000003F3F000000000F1F381E
:1017800030303030381F0F03070E1C38381C0E075E
:10179000030F1F38381F1F38381F0F3C3E07030147
:1017A0000103073E3C000000013F3F010000003CF8
:1017B0003E373331303030303000003F3F30303052
:1017C00030000000000000000103070E0C00003094
:1017D0003030303F3F0000000000000000000000FB
:1017E0000030303030303030303030000003070E01
:1017F0001C383000000000303030303070E0C0FF66
:10180000FFC0E070303070E0C0C0E0703030303089
:10181000300000C0E070303070E0C0FFFFC0E0700A
:101820003030303070E0C0C0C0FCFEC7C303070ECC
:101830000CF0F89C0C0C0C0C0CFCFCFFFFC0E070D6
:10184000303070E0C000003030F3F30000000000E2
:101850000000003030F3F30000FFFF0080C0E070B4
:1018600030000000000303FFFF00000000F0F03034
:1018700070E0E07070E0C0F0F0C0E070303070E018
:10188000C0C0E0703030303070E0C00000000000B8
:1018900000000000000C1E3F33333333333F3F3F23
:1018A0003F3030303030381F0F0F1F38303030307D
:1018B000381C0C0F1F3830303030303F3F0F1F3B8B
:1018C0003333333333030300003F3F000000000095
:1018D00000000133333333333B1F0F3F3F00000021
:1018E0000000003F3F000030303F3F303000000C30
:1018F0001C383030381F0F00003F3F03070F1C38E3
:10190000300000000030303F3F303000003F3F00EB
:1019100000030300003F3F3F3F0000000000003F86
:101920003F0F1F3830303030381F0FF0F03030307C
:101930003030F0E0C0C0E0F0303030E0C0F0F0F027
:10194000F0C0E070303070E0C0C0E0F030303030D7
:101950003000003030FFFF303000000000F0F000B9
:101960000000000000F0F0F0F0000000000000F0C7
:10197000F0F0F0000000000000F0F03070E0C080F7
:1019800080C0E07030F0F0800000000000F0F03027
:1019900030303030B0F0F070300000C0E03C3E0736
:1019A00003000000000000FFFF0000000000000333
:1019B000073E3CE0C00000C0C0C0C00C1CF8F0E016
:1019C000C0C0E0F0F81C0CC0C0C0C03F3F03030320
:1019D000030303010000010303030303033F3F3F2D
:1019E0003F00000000000000003031333333333358
:1019F0003F1E0C00000F1F383030381C0C0F1F38F2
:101A00003030381C0C3F3F03070E1C38381C0E07C3
:101A1000030F1F38381C1C38381F0F30381C0F07B5
:101A2000070F1C3830000133333333333B1F0F3083
:101A3000383C3E373331303030000000010F1F3862
:101A4000300000000000003F3F00000000000030B8
:101A5000381F0F01000000000000000C0E070301FA
:101A600000000103070E0C000000005008500000A9
:101A70000000000000006F000007000700147F1442
:101A80007F14242A7F2A12231308646236495522C0
:101A9000500005030000001C2241000041221C00F0
:101AA00014083E081408083E0808005030000008DA
:101AB0000808080800606000002010080402003ECA
:101AC00049453E0000427F4000625149460041497D
:101AD0004936001814127F0027454539003E494910
:101AE0003200017905030036494936000649291EAE
:101AF000000036360000005636000008142241145B
:101B0000141414144122140800020151090600069D
:101B10000909067E0909097E7F494949363E414146
:101B200041227F4141221C7F494949417F090909DE
:101B3000013E4149497A7F0808087F00417F410002
:101B40002040413F017F081422417F404040407FB8
:101B5000020C027F7F0408107F3E4141413E7F0915
:101B60000909063E4151215E7F0919294626494946
:101B7000493201017F01013F4040403F1F2040208A
:101B80001F3F4030403F6314081463070870080784
:101B90006151494543007F41410002040810200083
:101BA00041417F00040201020440404040400001E6
:101BB00002040020545454787F4844443838444444
:101BC0004420384444487F3854545418087E09014E
:101BD000020C5252523E7F0804047800447D4000BB
:101BE0002040443D007F1028440000417F40007C9D
:101BF000041804787C0804047838444444387C147D
:101C0000141408081414187C7C080404084854545C
:101C10005420043F4440203C4040207C1C20402075
:101C20001C3C4020403C44281028440C5050503C60
:101C30004464544C44000836410000007F0000001A
:101C4000413608000808221C08081C2208084080A9
:101C5000080420100201536572766F205465737476
:101C6000004779726F2053657475700048656C6920
:101C700020536574757000456C65766F6E5C4465C5
:101C80006C746100562D5461696C00537469636B08
:101C90007920542D43757400542D43757400536995
:101CA0006D706C6520342D4348009E1C981C8B1C65
:101CB000841C771C6C1C611C561C000089111223AB
:101CC0009B322446AD573665BF74488CC19D5AAFD0
:101CD000D3BE6CCAE5DB7EE9F7F8811008019333C7
:101CE0001A22A5562C47B7753E64C99C408DDBBFB0
:101CF00052AEEDDA64CBFFF976E802218B301002A8
:101D000099132667AF763444BD554AADC3BC588E8F
:101D1000D19F6EEBE7FA7CC8F5D983310A20911286
:101D20001803A7772E66B5543C45CBBD42ACD99E6F
:101D3000508FEFFB66EAFDD874C904428D531661DB
:101D40009F702004A9153227BB364CCEC5DF5EED4F
:101D5000D7FC6888E1997AABF3BA85520C43977146
:101D60001E60A1142805B3373A26CDDE44CFDFFD2F
:101D700056ECE9986089FBBB72AA06638F72144027
:101D80009D512225AB343006B9174EEFC7FE5CCC0F
:101D9000D5DD6AA9E3B8788AF19B87730E62955006
:101DA0001C41A3352A24B1163807CFFF46EEDDDCEF
:101DB00054CDEBB962A8F99A708B088481951AA763
:101DC00093B62CC2A5D33EE1B7F04008C919522BF7
:101DD000DB3A644EED5F766DFF7C899400859BB79E
:101DE00012A6ADD224C3BFF136E0C1184809D33BD7
:101DF0005A2AE55E6C4FF77D7E6C0AA583B418867F
:101E000091972EE3A7F23CC0B5D14229CB38500AB6
:101E1000D91B666FEF7E744CFD5D8BB502A499965D
:101E20001087AFF326E2BDD034C1C3394A28D11A96
:101E3000580BE77F6E6EF55C7C4D0CC685D71EE5B2
:101E400097F42880A1913AA3B3B2444ACD5B566976
:101E5000DF78600CE91D722FFB3E8DD604C79FF51D
:101E600016E4A9902081BBB332A2C55A4C4BD77956
:101E70005E68E11C680DF33F7A2E0EE787F61CC4FE
:101E800095D52AA1A3B03882B193466BCF7A544836
:101E9000DD59622DEB3C700EF91F8FF706E69DD4DD
:101EA00014C5ABB122A0B9923083C77B4E6AD55816
:101EB0005C49E33D6A2CF11E780F276F11241FBE89
:101EC000CFEFD0E1DEBFCDBF11E0A0E0B1E0ECE3A9
:101ED000F0EE02C005900D92A434B107D9F71DE0D1
:101EE000A4E4B1E001C01D92A737B107E1F71EE1FC
:101EF000CCEBDEE104C02297FE010E94D76FCA3B03
:101F0000D107C9F70E94596D0C941C700C94000005
:101F1000EDE3F5E040E0842F806487B9369A369986
:101F2000FECF24B135B1369A3699FECF84B195B142
:101F3000820F931F819391934F5F483061F708950B
:101F4000853050F0883020F08E3020F482E0089503
:101F500081E0089583E0089580E008952AE0829F5B
:101F6000C001112481509E4F089525E0829FC00139
:101F70001124815C9C4F08958F929F92AF92BF92E3
:101F8000DF92EF92FF920F931F93CF93DF93C82FAF
:101F9000D62F5A01122FF02E822F8470D82E57FF81
:101FA00010C0882311F08CE101C08FE0212F4DE299
:101FB0006D2F9C2F981B892F0E945D5CB194A1947A
:101FC000B108212F2F214AE36D2F8C2F0E945D5CD9
:101FD0006CE370E0C5010E94806F4B015C01012F32
:101FE00000619B0140E050E062E0E62E6D2F8C2FF7
:101FF0000E944F5EDD2011F08AE101C08FE00F2DBD
:102000000061950140E050E092E0E92E6D2F8C0FC9
:102010000E944F5EDF91CF911F910F91FF90EF9043
:10202000DF90BF90AF909F908F900895CF93DF93F4
:10203000D62FC22F206250E00E945F5FC7FD09C00B
:102040002C2F46E76D2F8091580CDF91CF910C9487
:102050005D5CDF91CF910895242F409102010C9493
:1020600016100F93022F24FF03C00F7E9CE201C0C5
:1020700094E2411104C024E043E253E015C045302E
:10208000B0F4E091160594E0E99FF0011124319736
:10209000E40FF11DEF5BFC4FE49194E0E99FA00198
:1020A0001124445D5C4F24E00E94125D08C0941727
:1020B00030F02BEF240F41E852E00E94345D0F9185
:1020C00008950F93CF93DF93C82FD62F022F41117E
:1020D00004C024E04CE752E00EC04A3010F086E124
:1020E00001C081E18C0F50E0202F6D2F0E945F5FB7
:1020F00022E049E752E06D2F8C2F0E94125DDF91A4
:10210000CF910F9108950F931F93CF93DF93D62F05
:10211000C42F022F16E0180F442341F0463151F02E
:102120004A3E61F423E045E553E016C023E045E76D
:1021300052E012C023E041E553E00EC047FF04C067
:1021400041E20E945D5CC195C1504C2F440F4C0F81
:1021500050E04B5C5D4F23E06D2F812F0E94125D9C
:10216000DF91CF911F910F91089585E392E008953B
:10217000DF92EF92FF920F931F93CF93DF93F82E8E
:10218000D62F142FE22EC091F00181E08217E0F1EA
:102190004FE04C0F4F31D0F42C2F332727FD3095D3
:1021A00037FF03C0319521953109012F43E052E0FB
:1021B0006D2F8F2D0E94345DCF3FC4F5212F41E25A
:1021C0006D2F8AEF8F0D0E945D5C30C074E2D72EB8
:1021D000DC0E0AEF0F0D88E48D1520F01C1674F448
:1021E00041EF09C0212F4DE682E18F0D0E945D5C19
:1021F0001C161CF44CED4C0F01C04D2D212F6D2FE2
:10220000802F0E94831012C082E0281313C0212F58
:10221000409160046D2F8AEF8F0DDF91CF911F9158
:102220000F91FF90EF90DF900C948310E11002C0AB
:10223000C13069F3DF91CF911F910F91FF90EF9023
:10224000DF9008958C3038F4E82FF0E0EE0FFF1F98
:10225000EE55F84F22C08431C0F4482F50E0DA0127
:10226000AA0FBB1FA25DBE4F2D913C91803148F457
:10227000FA01EE0FFF1FE451FB4F80819181281B73
:10228000390BC901880F991F0895843248F4E82F4B
:10229000F0E0EE0FFF1FE65AF84F8081918108951C
:1022A0008E3218F484520C94531D80E090E008950F
:1022B0000E94556D8111FCCF1092890C08950F93E7
:1022C0001F93CF93DF938C01EB010E940D5C24E000
:1022D0004DEF51E060E082E20E94485DB80180E28B
:1022E0000E94685DBE0188E20E94685D67EE71E051
:1022F00080E30E94685D0E9423600E941F60DF915E
:10230000CF911F910F910C9458110F93462F50E0CD
:102310004B5C5D4F00E023E060E10E94125D0F9195
:1023200008950F931F93CF93DF93082FC5EED1E04D
:102330001AE0499124E0602F812F0E945D5C155FB7
:102340001837B9F7DF91CF911F910F9108951F931F
:10235000CF93DF93EC01162F0E940D5CBE0188E144
:102360000E94685D111109C049ED51E068E38CE1FC
:102370000E946E5D43ED51E002C04BEC51E024E061
:1023800060E082E20E94485DDF91CF911F910C9442
:10239000236061E00E94A7110C941F6070E0882305
:1023A00099F090E0019725E0289FF001299FF00D1A
:1023B0001124E60FF71FEE0FFF1FE655FB4F80813C
:1023C00091818B509E4F0895FB01EE0FFF1FED5F33
:1023D000FE4F0190F081E02D8081992787FD909537
:1023E00008951F93CF93DF93D82F162FC4E0DD23DA
:1023F00099F0612F8D2F0E94CE119C01253F81E025
:10240000380764F08BE0820F8D1710F08CE0820F9C
:10241000C15029F0D82FEBCFC0E001C0CD2F8C2FB9
:10242000DF91CF911F910895CF93C62F0E94F11194
:102430006C2FCF910C94CE110F931F93CF93DF93FA
:10244000EA01062F10E08823B9F00E94F1118823D9
:1024500099F090E0019725E0289FF001299FF00D69
:102460001124E00FF11FEE0FFF1FE655FB4FC55F74
:10247000D140D183C08317C0CE0183589F4F8B3F7B
:10248000910540F01C161D061CF4CDE7D0E002C0FB
:10249000C3E8DFEFF801EE0FFF1FED5FFE4F019085
:1024A000F081E02DC08386E0DF91CF911F910F91E5
:1024B0000C94A5579F92AF92BF92CF92DF92EF926A
:1024C000FF920F931F93CF93DF938C017B016A01DF
:1024D000922EB090C7019B2D9F7D943439F080914E
:1024E0008007882309F487C0933439F4E8012196E2
:1024F00083E10E943F6C85E00BC0953419F0923463
:1025000009F07CC0E801219784E10E943F6C84E0DF
:102510000E940161811164C0E114F104E1F481E0E1
:10252000C816D104C1F480E6B81619F08EE2B812CC
:1025300012C010928007C1E00115110509F0C0E03A
:10254000D0E08B2D0E9452618EE2B81206C081E06D
:102550008093B00702C0A12C02C0AA24A39440918A
:102560005C0150915D01C41BD50B8091B007833095
:1025700031F48091D001C80FD11D87FDDA95CC16BA
:10258000DD0644F48B2D0E94526183E10E943F6C72
:10259000E6010AC0CE15DF053CF48B2D0E94526186
:1025A00084E10E943F6CE701C017D107B1F020978A
:1025B00061F4A11003C08B2D0E94426117FF02C07D
:1025C00083E101C084E10E943F6C892D83700E94E9
:1025D000A55781E08093640113C01092640110C07C
:1025E000CC27DD27C01BD10B85E00E94526184E01F
:1025F0000E94526191CF953409F484CFE8018CCFC9
:10260000CE01DF91CF911F910F91FF90EF90DF905E
:10261000CF90BF90AF909F900895552747FD50955C
:10262000772767FD7095992787FD90950E945A122C
:10263000089522E00C940D13462F22E060E00C94E4
:102640000D1321E00C940D13462F21E060E00C9453
:102650000D13E0916501F0E0EE0FFF1FE859FE4F0A
:10266000808191810895FC01A0916501B0E0AA0FDD
:10267000BB1FAA59BE4FED93FC938FEB099587E1E1
:102680000C943F6CE1EBF7E0108E168A158A178ADE
:102690000895E8E2FDE037A1303180F420A541E063
:1026A000420F40A7DF01A20FB11DA20FB11D8D93F4
:1026B0009C93403108F010A63F5F37A3089590E047
:1026C0008C5F9E4F0C94491390E00C9449138091B9
:1026D0002E05992787FD909509970C944913FC01C5
:1026E0009091210580A191FF74C091A1882311F0E0
:1026F000946001C09B7F91A386A1813059F5C79A50
:1027000037A121A1332321F181A541E0480F41A741
:10271000DF01A80FB11DA80FB11D8D919C9195A34C
:1027200084A3403108F011A6315037A397FD02C0B1
:1027300031E101C038E233A32C7F97FD226021A351
:1027400081A18BBBC7988FE182A382E086A3089505
:102750002BBB48C081110CC0C79A81A1836081A3A3
:102760008BBB8091590C8D3308F43CC086E02FC0A0
:10277000823009F438C081A18BBBC79ABF9800C0D2
:10278000000000C086B38078BF9A96A1933049F4C8
:10279000882329F083A1815083A3811123C084E081
:1027A00016C0943021F48823E9F083E00EC0953000
:1027B00039F483A1815083A3811114C081E007C043
:1027C000963081F4882371F084E183A385E086A3A9
:1027D00009C090911E0596FB992790F9891711F071
:1027E000C79A0895C79808951BBA8FE18ABB00C0A5
:1027F00099B38FEF8ABBE8ECF1E08781882311F071
:1028000080E202C0892F807E8483292F207C8081F2
:10281000281759F08074880F90783181891711F04A
:10282000315001C03F5F31832083828193818917BA
:1028300011F08383818308959091160590FD02C065
:1028400093E08927E82FF0E0EE0FFF1FEE55F84FD9
:102850008081918197FF02C081589F4F880F892FF7
:10286000881F990BE82F181624F0882321F0E19592
:1028700002C080E801C080E0E8300CF0E7E0F0E062
:10288000E85DFC4FE491EE2319F099E0909370011C
:102890008E2B0895833021F0811103C083E001C0A5
:1028A00080E0E82FF0E0EE0FFF1FE35CFA4F80813D
:1028B00091810895FF920F931F93CF93DF93F12C93
:1028C000C0E0D0E08F2D0E944A14092F10E0C00F05
:1028D000D11FF39484E0F812F5CFCE01DF91CF91B0
:1028E0001F910F91FF9008950E944A14209118059E
:1028F00020FF03C0919581959109089578941F92C6
:102900000F920FB60F9211248F93809144018F5F25
:10291000809344018F910F900FBE0F901F901895D8
:1029200078941F920F920FB60F9211242F938F93CA
:102930009F93EF93FF93F89487B78F7B87BF78942B
:10294000209191018091930190912105882359F064
:1029500090FF07C08091740D820F8093740D87FFE4
:1029600002C01B9A01C01B9891FF2AC08091570892
:10297000811126C0E8E2FDE086A1823009F583A13D
:10298000882311F081501BC021A1C79A82A180FD2C
:1029900009C02D7F84A195A196FD2260880F991F03
:1029A00095A384A381E082278BBB81A3C79882A1D2
:1029B000815082A3811104C083E086A385E083A3B4
:1029C000F89487B7806487BF7894FF91EF919F91C7
:1029D0008F912F910F900FBE0F901F9018957894A4
:1029E0001F920F920FB60F9211242F933F934F9384
:1029F0005F936F937F938F939F93AF93BF93EF9367
:102A0000FF9381B7845681BF8FE891E00E94F069FF
:102A10000E9461618091950C82608093950CEBE03F
:102A2000F1E08081815011F0808307C084E68083CB
:102A300081818F5F818381E082838381815011F066
:102A4000838304C08AE0838381E08483FF91EF91D4
:102A5000BF91AF919F918F917F916F915F914F91B6
:102A60003F912F910F900FBE0F901F901895789463
:102A70001F920F920FB60F9211242F933F934F93F3
:102A80005F936F937F938F939F93AF93BF93EF93D6
:102A9000FF932091800030918100F89480917D0017
:102AA0008F7D80937D0078948091360590913705D5
:102AB000A901481B590BCA01969587953093370594
:102AC000209336059C01215A3F402F3D3E4220F481
:102AD00081E0809345012FC0E09145012FEF2E0F3B
:102AE000283048F59C01215233402737354008F5FE
:102AF00021E02E0F20934501F0E0EE0FFF1FEC5B6D
:102B0000FE4FAC014C5D554020911C05332727FD3D
:102B10003095265F3F4F429FC001439F900D529FCB
:102B2000900D11246AE070E00E94806F71836083D1
:102B300002C010924501F89480917D0080628093DC
:102B40007D007894FF91EF91BF91AF919F918F910C
:102B50007F916F915F914F913F912F910F900FBE99
:102B60000F901F9018959C0155E0359527955A9523
:102B7000E1F7280F391FAC01440F452F441F550BB7
:102B8000241B350B892F990F990B8595820F931F65
:102B900008959DE7980F9B3FA0F08E57282F30E0B7
:102BA000220F331FF901E456FB4F8081861714F47E
:102BB0006083862F48172CF4F901E456FB4F4083BD
:102BC000842F089544E66CE90C94C91520911605EC
:102BD000217092E0921B21E0981320E0822F08954B
:102BE0009091F60194FF08C00E94E61591E08111D2
:102BF00001C090E0892F089580E0089549E28402A1
:102C000090011124359527953595279587FD815C91
:102C100086FB880F880B80F9A901481B510987FDA5
:102C20005395CA0108954F925F926F927F928F924F
:102C30009F92AF92BF92CF92DF92EF92FF920F934B
:102C40001F93CF93DF93782E642E25E0241708F48A
:102C5000D4C0882309F4CFC036E1831721F08AEE6F
:102C6000781203C0CAC081E0CCC096E197150CF47D
:102C7000C4C0872D992787FD909597FF03C0919534
:102C8000819591098A3040F4825F0E940161171496
:102C90000CF4B7C091E01CC026EF280FE22EF12CF7
:102CA000E701CC0FDD1FCE0DDF1DC55CDB4F8A8138
:102CB0008F7009F4A2C0F701EA58FE4F6F01F5E0EA
:102CC0006F1208C0F601908117140CF492C081E0D5
:102CD000892797C0588049800E94A00F811109C0A0
:102CE0008FEF850D0E9422118C0189810E94FE15B3
:102CF00010C0823051F48FEF850D0E9422118C019B
:102D0000898181500E94221104C080E090E000E09F
:102D100010E02A812F70822E912CF4013197EE3031
:102D2000F10508F06CC0EA5BFF4F0C94D56F17FFFC
:102D300037C011950195110933C017FF35C01195A2
:102D40000195110931C001E0060D402F60E0852D8D
:102D50000E941316182F402F60E0842D0E94131636
:102D60002A812F70253061F4112309F448C088238B
:102D700009F445C08A81982F907F69F591E036C0AB
:102D8000263019F41111F6CFF2CF982F912720C0D9
:102D900008171907A1F5EECF0817190759F72FC023
:102DA000801791073CF32BC0081719071CF327C0A5
:102DB00008171907FCF623C080179107DCF61FC01F
:102DC000F701EE57FE4F90819095991F9927991F13
:102DD0009111D0CF0BC082958F7089300CF08F5F2E
:102DE00041E0460D60E00E941316982FF601908393
:102DF0006BCF892F06C0862F04C080E002C090E010
:102E0000F5CFDF91CF911F910F91FF90EF90DF9061
:102E1000CF90BF90AF909F908F907F906F905F907A
:102E20004F90089540E060E0809103050E941316E2
:102E3000811114C08091570190915801892B71F430
:102E40001092480D8091590C90913C05981751F0C3
:102E500080933C0588E29DE00C946F1381E08093A1
:102E6000480DF0CF08952091570130915801211558
:102E7000310511F021503109882319F080911A058C
:102E800001C080E090915601992329F0909122058C
:102E9000891708F4892F4AEF849FC0011124880FF5
:102EA000991F8217930708F4C901909358018093E2
:102EB00057010C941217CF92DF92EF92FF920F936B
:102EC0001F93CF93DF93F89480915A0C90915B0CF1
:102ED000789441E020913A0530913B0582179307A1
:102EE00009F440E04093590190933B0580933A05E3
:102EF00060E08BE597E00E949E368091590188231F
:102F000009F4BFC28091720190917301A091740184
:102F1000B0917501AC01BD014F5F5F4F6F4F7F4FA7
:102F20004093720150937301609374017093750123
:102F3000443651056105710598F083569109A10940
:102F4000B1098093720190937301A0937401B093BF
:102F5000750180917001882319F081508093700170
:102F6000E1EBF7E0878980FF0DC0808D91E0980F3D
:102F7000908F943638F08356808F85899689019694
:102F8000968B858B80E00E94B7570E940D5C0E9453
:102F90009560182F082F0F700650C091F701C430AC
:102FA00021F0C33019F4C4E001C0C8E0083008F0D3
:102FB0009FC0F02EF6948091320580FF03C083E01D
:102FC0008F19F82E6F2D80914D050E94F111E82E7A
:102FD0006F2D0E9414129C01C1110DC0AC0197FF0E
:102FE00004C044275527481B590B559547955595BF
:102FF0004795C1E0C40F8091160580FBCC24C0F832
:10300000D12C42E050E04C195D098F2D90E048171B
:10301000590761F48091F60180FF31C281E0C4E07C
:103020009091180590FF03C0C19501C080E0DD2795
:10303000C7FDD09500FF03C0C20FD31F04C0A90174
:103040004C1B5D0BEA01209721F09D2F932797FFE2
:1030500011C081110FC0232B69F040E050E06F2DAB
:103060008E2D0E941C12812F0E94526186E10E94C7
:103070003F6C3DC0CE0184589F4F893F910580F43D
:10308000AE016F2D8E2D0E941C12D7FF03C0D1956B
:10309000C195D109D595C795D595C7954C2F21C018
:1030A0001C161D061CF44DE750E002C043E85FEF1C
:1030B0006F2D8E2D0E941C12CE0183589F4F8B3F87
:1030C0009105A8F4D7FF03C0D195C195D109D7FDCB
:1030D0002396AE0155954795559547955195419540
:1030E0005109445C65E18FE891E00E94C16A10E0FB
:1030F000EAE5F1E08091AE079091AF072081318140
:10310000281B390B37FF02C0215E3F4FC5E03595C4
:103110002795CA95E1F72115310561F024813581A4
:10312000281B390B37FF02C02F5F3F4F359527957E
:1031300091838083958384838091180585FF02C0E5
:1031400020E030E033832283C8ECD1E02D818981F7
:10315000821B8F3F09F480E087FD8F5F859588870C
:10316000982F990F920F9D83812B0E943317E09126
:103170006501F0E0EE0FFF1FEA59FE4F808191815B
:103180008D569F43B9F488858823A1F02E81992715
:1031900087FD9095820F911D27FD9A958E37910599
:1031A00014F08DE705C08338EFEF9E070CF483E839
:1031B0008E83188680911E0587FF3BC08091710128
:1031C0008823B9F1809170018823A9F18091390594
:1031D00087FD03C08F5F8093390582E00E941C1435
:1031E000982F9F7789F020913905921720F510923A
:1031F0003905111120C0182F1095111F1127111F0B
:1032000083E6811B182F17C083E00E941C14982F9F
:103210009F7789F020913905921768F4109239054B
:10322000111109C0182F1095111F1127111F1C59BA
:1032300002C01092700181E0809371017DE9E72E58
:1032400074E0F72ECCE9D4E0EAE0CE2ED12CF701E1
:103250008081882309F462C0853068F40E94696225
:10326000E82FF0E0EE0FFF1FEF5FFE4F0190F081BF
:10327000E02D808104C0853021F48091CE018883C7
:103280004DC08A30B8F485500E946962E82FF0E0A2
:10329000EE0FFF1FE056F84F8081918197FD079652
:1032A00043E0959587954A95E1F78338FFEF9F07AF
:1032B000DCF015C08D30D0F4E82FF0E0EE0FFF1FEA
:1032C000EA56F84F8081918197FD079623E0959506
:1032D00087952A95E1F783382FEF92072CF08D37E9
:1032E00091056CF28DE7CBCF83E8C9CF8D31B0F477
:1032F000E82FF0E0EE0FFF1FE859F84F8081918131
:10330000B6010E94806F63384FEF74072CF06D3761
:1033100071051CF06DE701C063E8688352E0E50EBB
:10332000F11C22968BEAE81684E0F80609F08FCFAC
:103330008091E3019091E401009761F060E00E94C8
:10334000A7110E94556D882399F01092E401109204
:10335000E3010EC01093C701E0916501F0E0EE0FAC
:10336000FF1FEA59FE4F0190F081E02D812F099552
:103370000E942360C09165008FE891E00E94DC69A3
:10338000882311F084E105C08091760D882321F017
:1033900081508093760D06C0809163008695817080
:1033A0008093750D8091750D8093E101882309F458
:1033B00064C080911E0585FD60C0CF7EC09365000E
:1033C0008091590C8F71823009F054C080914B0567
:1033D00090914C05AC0114E0440F551F1A95E1F78C
:1033E00097FD0796BC01D3E075956795DA95E1F7EF
:1033F00020910205332727FD30952A5F3F4F629FBA
:10340000C001639F900D729F900D1124840F951F32
:103410002091180526FD05C0609100017091010101
:1034200002C060EF70E00E946C6F80910201680F33
:10343000711D6F5F7F4F7595679560930201809155
:103440003805805F80933805811114C08091010593
:10345000681780F4623370F06EE281E10E94456C7F
:103460008091180583FF06C082E390E09093580195
:10347000809357011092560104C0C0619FCF80E035
:10348000CFCDDF91CF911F910F91FF90EF90DF9003
:10349000CF900895CF93DF93C62F2091E20122238E
:1034A00029F09093E4018093E30133C060E00E942F
:1034B000A711C11103C08091000501C089E10E94DC
:1034C000106067E182E10E94456C0E945811D1E0D2
:1034D0000E94556D81111DC08091950C833019F4A7
:1034E000A8951092950C40E060E0809103050E9441
:1034F0001316811106C080911A05811102C0CC23D8
:1035000029F0D093480D0E941217E2CF1092480D77
:10351000FACFDF91CF91089590916501911103C089
:10352000811106C017C0811103C08FEF890F01C040
:1035300080E08093650187E10E943F6CE091650126
:10354000F0E0EE0FFF1FEA59FE4F0190F081E02DF1
:103550008EEB099460E08EEB91E00C944A1ACF93C5
:10356000DF93EC0180916501843038F060E081EBFD
:1035700091E0DF91CF910C944A1A87E10E943F6C51
:10358000A0916501AF5FA0936501B0E0AA0FBB1FDA
:10359000AA59BE4FCD93DC938FEBFE01DF91CF9103
:1035A00009941F93CF93DF93C2EBD4E090E088811E
:1035B00011E0190F882341F040E060E00E941316EB
:1035C000882311F0812F05C0912F2A96143079F7A6
:1035D00080E0DF91CF911F910895DF92EF92FF92EB
:1035E0000F931F93CF93DF9380914401C2B79091C3
:1035F00044018913F9CFD0E0D82B60E1F62E8091F9
:103600006104F81A0E94880F1EE517B90E94F4138E
:103610000E945B1717B9369A3699FECF84B195B1DF
:103620000496409100015091010167E0649F900170
:10363000659F300D1124820F931F53E09695879557
:103640005A95E1F790930101809300018091950CC8
:10365000833019F4A8951092950C2091440182B7FB
:10366000909144012913F9CF90E0922B8C1B9D0B74
:103670002091AC063091AD062817390720F49093BD
:10368000AD068093AC0680910C01823078F4809175
:103690000F01882309F4F1C080913305909134051E
:1036A0000196909334058093330589C010920C01E4
:1036B000809135058F5E982F977F903618F4909300
:1036C000350503C0877080933505C5EED1E0E12C48
:1036D000EF14E9F28E0103581D4FF8018081982FF5
:1036E000907C9034C9F4880F880F40E060E08595A5
:1036F00085950E941316882379F08091210580FF1B
:1037000005C0FE01E258FD4F608101C061E046E462
:103710008FE891E00E94C16AF8018081982F907C27
:103720009038D1F5880F880F85958595873114F1EC
:10373000992787FD909547978130910549F0823010
:10374000910561F0892B41F580913505837003C0A7
:1037500080913505807F81111FC005C0809135059E
:1037600087708230C9F4FE01E258FD4F80810E94CB
:10377000791D12C09091350590FD0EC040E060E0CB
:103780000E941316882341F0FE01E258FD4F80810C
:10379000805890E00E944913E394229699CF0F2D10
:1037A00010E0E801CC0FDD1FCE59DB4F8881E82EF9
:1037B000E294E69447E0E4228F7129F4F394FFE069
:1037C000FF1568F758C040E060E00E941316D82E3D
:1037D00080910F010F521E4F823009F449C08E2D87
:1037E000857051F4F8018081811106C0DD2021F03F
:1037F000898190E00E9449138FEF8E0D823060F432
:10380000F80180818130A1F5D11032C08981F2E0C8
:10381000EF122BC08F5F29C085E08E1550F4F801A0
:103820008081811125C0DD2019F189810E94791DD7
:103830001FC0F2E0FE15E0F4DD20D1F084E0E816D0
:1038400031F095E0E91631F066E970E005C06CE210
:1038500071E002C068E572E0809133059091340513
:103860000E946C6F892B21F4898190E00E9449139A
:10387000F801D082A3CF10920F0180910D0188230F
:10388000D1F110920D010BE314E0C2E8D1E0EE2477
:10389000EA94F801F2808F2D8F700E94A00F833080
:1038A00019F59881911104C0F8018081809508C0B4
:1038B00097FF08C09F5F9883911106C0F80181812E
:1038C000888302C0915098838F2D807F69F08F2D5F
:1038D00082958F7089300CF08F5F40E060E00E942D
:1038E0001316811101C0E8820D5F1F4F2196F1E090
:1038F000CE38DF0771F6DF91CF911F910F91FF90C6
:10390000EF90DF9008951F93CF93DF93182FD62F5A
:10391000C42F8091B007811101C0C2E04D2F50E04B
:103920002C2F60E08FE70E945F5FDA3010F0DFE657
:1039300001C0D5E72C2F4FE260E08D2F0E945D5C27
:10394000412F50E04F5F5F4F2C2F60E08FEF8D0FC6
:10395000DF91CF911F910C945F5F1F93CF93DF9303
:10396000D82F162FC42FB9010E94685D112329F0AA
:103970006FE08C2F0E941C13C82F4C2F50E0212F7A
:103980006D2F80E60E945F5F8C2FDF91CF911F919A
:103990000895813649F40E94526181E00E948C1A98
:1039A00086E395E40E94AF1A6CE27EE080E10E941B
:1039B000685D66E17EE080E20C94685DFF920F93A3
:1039C0001F93CF93DF93182FF62E0AE08AE0189FFB
:1039D000E0011124C150DE4F2FE130E0211B3109FD
:1039E000029FA001039F500D1124BE01CE010A9633
:1039F0000E94EA6FFF2049F0BE016A5071094AE057
:103A000050E0CE010E94EA6F0AC0FE0111920A95B1
:103A1000E9F78091F3078883898384E68A8310938A
:103A2000F507DF91CF911F910F91FF9008959C01B1
:103A3000220F331F280F391F9595879595958795E8
:103A4000280F391F95958795959587959595879515
:103A5000820F931F0895429643E7489F9001499F24
:103A6000300D1124C901E6E095958795EA95E1F7B7
:103A7000089581E00895E82FFF27E7FDF095E65BC4
:103A8000FD4EE491862F992787FD909583589F4F8F
:103A9000EE5FE23038F42AE0AC01249FC001259F9C
:103AA000900D11240895E82FFF27E7FDF095E65BC0
:103AB000FD4EE491ED3F4CF4EE0FFF0BE055FB4F54
:103AC0008081992787FD90950895ED3F59F074F016
:103AD000EF3F09F05CF4EE0FFF0BEB54F84F8389D6
:103AE000948908958091020190E0089580E090E02B
:103AF0000895CF92DF92EF92FF92F82E0E94531D0D
:103B0000EF2DFF27E7FDF095E65BFD4EE491ED3FDD
:103B100009F15CF4E63FDCF0EE0FFF0BE055FB4FE4
:103B20008081992787FD909512C0EF3F09F07CF4C2
:103B30006CE370E00E94806F6B017C0146E260E004
:103B4000C6010E944E6CC70160E045E305C060E01D
:103B500040E002C061E044E2FF90EF90DF90CF9040
:103B60000C944E6CBF92CF92DF92EF92FF920F9324
:103B70001F93CF93DF93F82ED62EC42EE901102F7A
:103B80008E2D8170B82EE0FE12C000E021E0240FDF
:103B900044E552E18F2D0E94345D12FD03C088E19F
:103BA0008F0D06C08CE18F0D98EFD90E01C08F2DBF
:103BB0009E2D9870E3FC1F7BEC2DFF27E7FDF09511
:103BC000E65BFD4EC49022E02C0D223088F412FFFB
:103BD0008450B110865F1770012F212FAE016D2D1B
:103BE00086500E94BC0FC3E3CC0D8AEFF80E0AC0CA
:103BF000992311F08DE38F0D212FAE016D2D0E94C1
:103C00005F5FC0E28E2D867069F0E2FE04C08AE03C
:103C10008F0D1B7F02C08091580C212F4C2F6D2DD2
:103C20000E945D5C8C2FDF91CF911F910F91FF90CF
:103C3000EF90DF90CF90BF900895DF92EF92FF92C8
:103C40000F931F93CF93DF93D82F162FC42FD22E0D
:103C50008E2D8370F82EA1F08091C701803881F4F9
:103C60008DE7840F8B3F40F0E42FF0E0EE0FFF1F55
:103C7000E056FC4FC08101C0CEE782E00E94A5570C
:103C80008DE78C0F2E2D8B3FE0F043E151E1612F4A
:103C90008EEE8D0F0E94485D2E2D43EB4C0F612F51
:103CA0008AEF8D0F0E945D5CFF2009F122E042E85F
:103CB00050E06EE770E08C2F90E00E945A12C82FFF
:103CC00016C04C2F552747FD5095612F8D2F0E9410
:103CD0005F5FFF2061F0402F6D2D8C2FDF91CF9122
:103CE0001F910F91FF90EF90DF900C9419138C2F80
:103CF000DF91CF911F910F91FF90EF90DF9008958A
:103D0000CF93DF939EE0899FE0011124CB51DE4FDA
:103D1000FE01EA54FE4F40E060E080810E941316ED
:103D2000882359F0C954DE4F40E060E088810E944A
:103D30001316811104C081E003C080E001C082E05D
:103D4000DF91CF910895EF92FF920F931F93CF933E
:103D5000DF93F82EE62EC42FD42FD695062F0D1BF9
:103D6000182F1D1B602F812F0E94035E6D2F6E0D7B
:103D70004C2F812F0E94005E4C2F602F8D2F8F0DB6
:103D80000E94035E4C2F602F812FDF91CF911F91F6
:103D90000F91FF90EF900C94005E21E0AC0160E089
:103DA00080E00C94485D1F93CF93DF93182FC0E100
:103DB000D1E080E598E00E94CD1E1136B1F068F4A4
:103DC0001036D1F48FEF888319821092AD061092CD
:103DD000AC0687E10E943F6C0FC0123619F0133613
:103DE00021F00AC087ED9FE102C08DE69FE3DF91DD
:103DF000CF911F910C94331361E478E088E00E9426
:103E0000685D4981469550E068E084E50E946E5FF8
:103E100062E378E080E10E94685D4881469550E069
:103E200060E184E50E946E5F63E278E088E10E94D1
:103E3000685D498150E08881481B510957FF02C0E5
:103E40004F5F5F4F5595479568E184E50E946E5F2F
:103E50006AE178E080E20E94685D8091AC06909112
:103E6000AD0629E1289FA001299F500D11245695E8
:103E700047955695479520E360E284E50E945F5F91
:103E800067E078E088E3DF91CF911F910C94685D43
:103E9000FF920F931F93CF93DF93C82F82E098E098
:103EA0000E94CD1EC13659F40E942B6D8DE69FE312
:103EB000DF91CF911F910F91FF900C94331303E585
:103EC0001DE0C3E6DDE08CE0F82EF80141918F01A2
:103ED00020E168E18F2D0E945D5C499120E160E264
:103EE0008F2D0E945D5CF6E0FF0E8CE6F812EDCFA0
:103EF0008091520D882309F454C00E94296D83E0FB
:103F00000E940161882351F080912801909129013C
:103F1000807D9927909329018093280182E00E9457
:103F20000161882351F08091280190912901807BC3
:103F30009927909329018093280185E00E940161CF
:103F4000882351F080912801909129018077992749
:103F5000909329018093280184E00E9401618823C5
:103F600051F08091280190912901807E99279093AA
:103F70002901809328011092520D8091280190917F
:103F800029010E94316DEFE9FFE03197F1F700C0A0
:103F900000000E94276D80EF90E0909329018093AC
:103FA0002801DF91CF911F910F91FF9008950F93FA
:103FB0001F93CF93DF93182FC1EBD7E08DEF97E0DE
:103FC0000E94CD1E113678F0133628F0133659F4BE
:103FD00083ED9EE102C08DE69FE3DF91CF911F91BB
:103FE0000F910C94331364EF77E088E00E94685DD2
:103FF0004A815B8100E020E068E08AE20E94BC0F19
:104000004C815D8120E068E08EE40E94BC0F6BEE85
:1040100077E080E10E94685D4E815F8120E060E191
:104020008AE20E94BC0F4885598594E056954795D1
:104030009A95E1F720E060E18EE40E94BC0F66EE05
:1040400077E080E00E94685D4881598120E060E06F
:104050008EE40E94BC0F4EE76CE382E00E94005E9B
:1040600043E26CE185E00E94035ECBE043E06BE35A
:104070008C2F0E94035ECA5FC338C1F71091AF0650
:104080008091AE06893710F4C0E001C0C12FD6E0A0
:104090000CE3EC2FF0E0E055F94F4081602F641BFA
:1040A0008D2F0E94035ECF5FC83708F0C0E0C117B4
:1040B00019F0DF5FDE3769F7DF91CF911F910F9124
:1040C000089591E0211101C090E0442319F041E5E9
:1040D00053E002C045E553E0292F0C94485D0F934F
:1040E00001E0211101C000E0242F4BE051E10E94CA
:1040F000345D0F9108956F927F928F929F92AF924D
:10410000CF92DF92EF92FF920F931F93CF93DF93A3
:10411000EC01162F842F4901602FD0905A07609030
:10412000AA077090AB07A091AC07B091AD07EAE584
:10413000F1E0268137812619370937FF02C0215C5B
:104140003F4F76E0359527957A95E1F7422F2093FA
:104150007D07208531852A1B3B0B37FF02C0215C80
:104160003F4F56E0359527955A95E1F7922F2093CA
:104170007B07442311F077826682992311F0B1877F
:10418000A08790917C07911104C09091180595FF2C
:1041900006C010927D0710927B0710927C079091C9
:1041A0007D07911108C020917B07211104C0228155
:1041B0003381232B61F020911A054AEF249F90014F
:1041C0001124220F331F309358012093570181147B
:1041D0009104B1F02881211177C12091B0072223E9
:1041E00009F47BC1213009F48AC191118FC11536C0
:1041F00009F4AFC1143609F4B6C141E00E94831C32
:10420000E114F10451F098818C2D9C1508F4892F4C
:10421000F701E80FF11DE49101C0E0E08091B007E3
:10422000813081F58091D00118166CF4DE1610F4FF
:10423000D39411F588818A1518F48F5F888301C0A3
:104240001882D12C19C08823B9F0D11014C08881EC
:10425000882319F08150888301C0A882E114F104F9
:1042600059F098818C2D9C1508F4892FF701E80FDF
:10427000F11DD49001C0DA941092D0011E3249F49D
:1042800083E005C0833029F41E3219F481E0809365
:10429000B007E114F10451F098818C2D9C1508F4BD
:1042A000892FF701E80FF11D549101C050E0809172
:1042B0008007811145C080917B07882301F14881E7
:1042C000481B47FD40E08A2D90E0242F332727FD2F
:1042D0003095281739070CF04A2D4883E114F10472
:1042E00059F0C41608F44C2DF701E40FF11DE491C8
:1042F000ED1518F4DE2E01C0D12C10927B07288119
:104300002223F1F080917D078823D1F0D81AD7FCC1
:10431000D12C8D2D992787FD9095E114F10479F02A
:104320003C2D2C1508F4322FF701E30FF11DE49119
:104330002E2F30E0821793071CF0DE2E01C0D12C07
:10434000103669F190F4123409F473C028F4113274
:10435000A9F11E3221F197C0143409F446C008F4C3
:1043600076C0153409F451C08EC0153609F451C019
:1043700040F4133609F46EC0D8F5123609F45CC067
:1043800082C01E38C1F01F3B31F0113809F07BC0EC
:104390001092800721C018821092800738C088814F
:1043A000882309F470C081E090918007911180E02A
:1043B0008093800768C08EE80E94526180918007D8
:1043C000882319F0109280075EC08881882311F03D
:1043D000892831F41092B00780E00E948C1A53C0F3
:1043E00087E10E943F6C18824EC0D51609F44BC07D
:1043F000EF2809F448C080918007811144C0D51688
:1044000010F4D39411C0D12C0FC0D11002C0D12C04
:104410003AC0EF28C1F180918007811134C0DD20BE
:1044200011F0DA9401C0D52E552369F11092C7011D
:104430002AC088818A1539F180918007811123C0B3
:1044400088818A1510F48F5F0DC018820EC0888194
:104450008823C9F080918007811115C08881882345
:1044600019F08150888301C0A882E114F10479F227
:1044700088818C1508F4C82EF701EC0DF11DE4902D
:10448000ED1408F4DE2C8091800781110AC021E030
:1044900080915C0190915D01892B09F420E0822FCD
:1044A00001C081E080937F07D0925A07DF91CF91BE
:1044B0001F910F91FF90EF90DF90CF90AF909F9062
:1044C0008F907F906F90089590918007911103C015
:1044D00091E09093B00740E091CE2091D001121668
:1044E00024F0222319F015E601C014E61092D00141
:1044F0001E3209F07ACE21E02093B00705C01E32AB
:1045000009F073CE1092B00710E06FCE20918007B3
:1045100021116DCEE82FE91BE7FDE0E0462F50E0CA
:104520002E2F332727FD30952417350714F0EFEF92
:10453000E60FFF27E7FDF095282F30E0E217F3079D
:1045400029F0EE0FFF1FE80DF91D1DC010927D0729
:104550004ECE811101C0862FF401E80FF11DE80F46
:10456000F11D329710C0282F30E070E061507109C2
:104570002617370714F48F5F01C080E0880E911C66
:10458000880E911CF40185919491DF91CF911F9138
:104590000F91FF90EF90DF90CF90AF909F908F9012
:1045A0007F906F900C943313AF92CF92EF92FF9263
:1045B0000F93AE2CC12CE12CF12C0E947B200F918B
:1045C000FF90EF90CF90AF900895EF920F93E42E6D
:1045D00000E020E030E040E00E94D4220F91EF9014
:1045E0000895BF92CF92DF92EF92FF920F931F93A5
:1045F000CF93DF93C82F83EB9AE00E94CD1EEE2469
:10460000E39406E027E231E144E06C2F87ED97E088
:104610000E94D422B090D70710927101C2EAD7E06D
:1046200010E000E0C12CE4E0DE2EE12CF12C41E4AE
:10463000612F88E10E940F5D41E3400F612F8EE101
:104640000E940F5D802F0E944A14AC01612F8AE204
:104650000E94715D073081F0A881B98124E630E0C5
:104660000E94426FA70196010E94B66FA901612FB7
:104670008AE50E946E5F0AC081E0B81611F040E240
:1046800001C041E2612F8AE50E942C100F5F185F84
:104690002296083061F622E040EB5AE068E28CE6B0
:1046A0000E94425D409100015091010160E388E762
:1046B0000E946E5F81E0B8120AC0B0927C074FE79B
:1046C00061E8809102050E94211380930205DF9129
:1046D000CF911F910F91FF90EF90DF90CF90BF90FF
:1046E0000895EF920F931F93CF93DF93C82F8BEA18
:1046F0009AE00E94CD1EE12C06E027E231E143E082
:104700006C2F86ED97E00E94D422D0E0C0E0C43048
:1047100018F018EF1D0F01C01D2F8FE08C0F0E94A5
:104720000161082FCF5F20E04C2F612F8AE20E94A9
:10473000831040E3400F202F612F84E40E945D5CD2
:10474000D85FC93021F7D8E3C0E08C2F0E94016107
:10475000182F00E02C2F4BE85AE06D2F80E00E94CC
:10476000345D40E3410F212F6D2F80E20E945D5C9C
:10477000CF5FD850C63049F743E85AE068E184E596
:104780000E946E5D16E0C0E2D0E02D2F4BE451E1B7
:104790006C2F84E50E94185C812F0E94016140E328
:1047A000480F282F6C2F8CE60E945D5C81E0810F02
:1047B0000E94016140E3480F282F6C2F88E70E9478
:1047C0005D5CDF5FC85F1E5FD430F9F6DF91CF918B
:1047D0001F910F91EF900895EF920F93CF93C82FF1
:1047E0008BE79AE00E94CD1EE12C06E027E231E142
:1047F00042E06C2F85ED97E00E94D4226BE877E0D1
:1048000080E10E94685D6BEB77E088E10E94685D63
:104810006AEA77E080E20E94685D6BE977E088E20F
:104820000E94685D6BE777E080E3CF910F91EF9096
:104830000C94685D4F925F926F927F928F929F92DD
:10484000AF92BF92CF92DF92EF92FF920F931F939E
:10485000CF93DF93C82F85EC90E10E94CD1EA7E097
:10486000AA2ECC24C394B3ECEB2EB0E1FB2E0CE0CB
:1048700023E331E14BE06C2F8BEE97E00E947B202D
:104880006090EB0780905A07CDE9EC2EC4E0FC2E37
:10489000CCE9D4E0AA24A394B12C18E0712C99247B
:1048A00087FC9094C12CD12CF0E34F2E4A0C0C2D98
:1048B00060EC70E1812F0E94685D442D612F8CE0D7
:1048C0000E940F5D6A147B0449F48C149D0431F43A
:1048D00080918007811105C021E001C020E0512CAA
:1048E00003C022E055245394013099F0022FF701C0
:1048F000208147E650E1612F88E40E94345D552015
:10490000C1F06CE1F70180810E941C13F7018083E4
:1049100010C04881552747FD5095612F8CE60E94B5
:104920005F5F552031F04DE763E888810E941913DD
:104930008883FFEFCF1ADF0A82E0C816D10409F09E
:10494000B6CFE2E0EE0EF11C2296185FFFEFAF1A31
:10495000BF0A103409F0A6CFDF91CF911F910F91BC
:10496000FF90EF90DF90CF90BF90AF909F908F908F
:104970007F906F905F904F9008957F928F929F925B
:10498000AF92BF92CF92DF92EF92FF920F931F935D
:10499000CF93DF93D82E83E79AE00E94CD1E56E096
:1049A000A52E65E0C62E7DE6E72E7AE0F72E06E01E
:1049B00027E231E141E06D2D84ED97E00E947B20FC
:1049C000C090D40780905A078091630081FF04C093
:1049D00066E67AE088E1FCC0CA948091800788236B
:1049E00019F043E0942E02C099249394CCE0D5E0D2
:1049F000B12C10E1AA24A394AB0C20E04A2D612F26
:104A000080E00E943110F12CCB1002C08F1411F005
:104A100000E001C0092D802F8270782E92E0F916F7
:104A200009F444C0E3E0FE1609F455C0F1E0E98062
:104A3000FF16D1F0E294E694E69433E0E3222E2DC3
:104A40004BE55AE0612F88E10E94345D772009F43C
:104A50005AC062E08E2D0E9424138295880F880F21
:104A6000807C99819F731FC0EE0CEE0CE594E59459
:104A70008E2D9DE08902F0011124F7FD3396AF01E0
:104A80005595479555954795202F612F82E40E94B3
:104A90005F5F7720C1F14FE161EE8E2D0E942113FF
:104AA0008F739981907C982B99832DC0E880EE2D8F
:104AB000E770EE2E2E2F4DE45AE0612F88E40E941D
:104AC000345D772001F163E08E2D0E9424138770FE
:104AD0009881987F16C0E880E594E594E594202FAE
:104AE0004E2D612F8AE50E948310772061F046E108
:104AF0006AEE8E2D0E942113880F880F880F9881EF
:104B00009770982B9883F394F4E0FF127DCF185F91
:104B10002296AF1611F0BA2C6DCF62E47AE080E3F2
:104B20000E94685D84E0C8120AC048E266EF809186
:104B30001C050E94211380931C0521E201C020E284
:104B400040911C05552747FD5095465F5F4F60E338
:104B50008EE40E945F5FEE24E39495E0C912E12C9D
:104B60002E2D4EE35AE068E380E00E94485D06E4A3
:104B700011E0C4E0D5E090E3F92EF80141915191A4
:104B80008F0169917991461B570B440F551F20E205
:104B900068E38F2D0E945F5FF8E1FF0E80E9F81255
:104BA000ECCFEE2091F090E6D9120FC088E0E6E459
:104BB000F1E0A4E0B5E001900D928A95E1F781E083
:104BC0000E94A55787E10E943F6C6EE27AE088E080
:104BD000DF91CF911F910F91FF90EF90DF90CF90D9
:104BE000BF90AF909F908F907F900C94685DFF92E4
:104BF0000F931F93CF93DF93F82EEB018A0147E1C8
:104C00006CE20E94A31E43E06BE28F2D0E94035EC4
:104C100043E06CE28FEF8F0D0E94005EC8016FE8E9
:104C20007FEF0E94806F2CE2260FCE0161E770E0DB
:104C30000E94806F862F45E0622F8F0DDF91CF910C
:104C40001F910F91FF900C94A31ECF92DF92EF92D1
:104C5000FF920F931F93CF93DF93C2EAD7E04A816D
:104C60005B81688179818AE20E94F7254C815D81B0
:104C70006E817F8186E50E94F7252896EAE3FE2E65
:104C80000DE510E0F7E3CF2E899199919C5FB80173
:104C90000E94806FDD24D394D60EEC2CE61A4D2DA5
:104CA0006E2D8F2D0E94035E4D2D6E2D81E08F0D98
:104CB0000E94035E4D2D6E2D82E08F0D0E94035EDB
:104CC00085E0F80E89E4F812DFCFDF91CF911F91D4
:104CD0000F91FF90EF90DF90CF900895DF92EF92C9
:104CE000FF920F931F93CF93DF93F82E88EE9AE0F5
:104CF0000E94CD1EEE24E39406E027E231E145E078
:104D00006F2D88ED97E00E94D4221092D807CBE354
:104D1000D7E010E0812F0E944A14488159818417FE
:104D200095070CF4AC01499359932C853D852817C0
:104D300039070CF49C013D872C87143060F0FE018C
:104D40007097240F351F37FF02C02F5F3F4F3595F7
:104D50002795318320831F5F1730E1F68091570735
:104D600080937C0790E2F91621F08FEBF8120EC0C9
:104D70000BC08F5F80935707833041F487E10E9417
:104D80003F6C81E00E94A55710925707809157070A
:104D90008130E1F0A8F0823009F07BC010927101FF
:104DA00067EB7AE080E10E94685D46E151E168E1ED
:104DB00082E10E946E5DC3EDD4E0EBE3F7E028C032
:104DC00067ED7AE088E10E94685D63C069EC7AE093
:104DD00080E10E94685D46E151E168E182E10E9464
:104DE0006E5DCDE2D7E0D12C18E9E12E1AE3F12E69
:104DF00008E615ECFF86EE861D8F0C8F8D2D0E9428
:104E00004A1489939993D39497E0D912F3CF41C070
:104E100061917191848595859B01281B390B37FF22
:104E200003C0319521953109233331053CF1DF0170
:104E300050974D915C91598348839A01261B370BFB
:104E4000B90137FF02C0615C7F4FB6E07595679589
:104E5000BA95E1F7261B370B3F872E87841B950BEE
:104E60009C0197FF02C0215C3F4FA6E03595279536
:104E7000AA95E1F7821B930B9D8F8C8F229687E07A
:104E8000E934F80729F60E940E569093FE048093A9
:104E9000FD04DF91CF911F910F91FF90EF90DF9074
:104EA0000C942526FF920F931F93CF93DF93182F17
:104EB000062FEA01F22E222321F061E00E94241342
:104EC000182FBE01802F0E94685D2F2D412F602F6B
:104ED00086E60E946120812FDF91CF911F910F9173
:104EE000FF900895FF920F931F93CF93DF93182F96
:104EF000062FEA01F22E222321F061E00E941C130A
:104F0000182FBE01802F0E94685D2F2D412F602F2A
:104F100086E60E946120812FDF91CF911F910F9132
:104F2000FF9008951F93CF93DF93D62F122F0E94E7
:104F30007227C82F212F482F6D2F86E60E946F20E1
:104F40008C2FDF91CF911F910895CF93482FCAE006
:104F50002AE0829FC001112481509E4F2FE130E052
:104F6000241B3109C29FA001C39F500D1124BC0115
:104F7000665F7F4F0E94EA6FE5E3F3E0DF011D9279
:104F8000CA95E9F782E00E94A557CF910C94445846
:104F90000F93CF93C42F0E948310002339F046E172
:104FA0006AEE8C2FCF910F910C9419138C2FCF9107
:104FB0000F9108950F931F93CF93DF93D82F162F40
:104FC000C42F022F47FF08C041E28AEF8D0F0E94D5
:104FD0005D5C86E08C1BC82F2C2F41E05FE0612FC9
:104FE0008D2F0E94345DDF91CF911F910F91089515
:104FF0000F931F93CF93DF93162F8132C0F581114A
:1050000003C0611108C033C0803219F4662329F04F
:105010002EC0662311F001E001C00FEF080F0E94BF
:10502000AE0FEC01802F0E94AE0FFC0198818FEF34
:10503000890F8031E0F420812131C8F4291302C0A6
:105040008BE009C0112329F0903188F49F5F988389
:105050000EC088830CC0815029F090812881219353
:105060009993F9CF82E00E94A5570093F407DF914E
:10507000CF911F910F91089580913503882329F0D6
:1050800089EC9CE10E94AF1A81E008956EE07EE019
:1050900088E20E94685D6FEF7DE080E30C94685DBC
:1050A000CF93C82F813669F08F3B39F0803699F461
:1050B00080912C070E94A52704C080E00E943F6CCD
:1050C0000AC08C2F0E94526181E00E948C1A86E3F4
:1050D00095E40E94AF1A63EF7DE088E00E94685D6E
:1050E000CF910C9446280F93CF93C82F8091290716
:1050F000882319F065E57DE002C068E47DE088E082
:105100000E94685D4FE06DE277E0809128070E9481
:10511000705600E12AE04DE257E060E181E00E9434
:10512000125D4FE360E182E40E940F5D0E94462819
:10513000C13609F44EC0CF3B21F0C03609F055C04E
:1051400005C080E0CF910F910C943F6C80912907AE
:105150008823A9F086E39DE00E94C9118091280769
:105160000E94DE56882339F087E10E943F6C82E07E
:10517000809329072CC080E00E943F6C28C080915A
:10518000FF048F5F0E949559C091FF0481E08C0F4E
:105190000E946559811109C0C150C13108F0CFE0AA
:1051A0008091FF04C813F2CFC0E0C093FF0481E0F8
:1051B0000E94A5570E9444588091FF040E94A75660
:1051C0008091EF010E945F1382E080930F0180E6DF
:1051D00001C081E60E94526181E00E948C1A8EE635
:1051E00090E3CF910F910C94AF1ACF910F91089546
:1051F0009091D00181E0191624F0911101C080E056
:1052000081951092D0010895CF93C82F0E94F8285D
:1052100090912B072091C701223671F028F4203697
:1052200039F02136A9F006C0233661F02E3611F48C
:1052300081E00FC0181624F49C1730F49F5F04C05F
:10524000882311F09111915090932B0780E001C0B9
:1052500082E0CF91089569EE7DE088E00E94685D6C
:105260006FED7DE080E10E94685D65ED7DE088E1A5
:105270000E94685D6BEC7DE080E20E94685D61ECFD
:105280007DE088E20E94685D2AE240E367E082E117
:105290000C94715FCF93DF9380E00E942B2984E010
:1052A0000E940429D82FC0912B076C2F660F660F20
:1052B000660F685F20E044E288E10E94965DD1308D
:1052C000B9F5C13089F40E943C2881110FC0C09308
:1052D000F2078091F5078F5F8093F50760E00E94E9
:1052E000DE1C10922A0702C0C23018F482E192E458
:1052F0000EC08091F507C43069F480932C0780912B
:10530000C7010E9452611092C70180E598E20E9495
:10531000AF1A0BC0C23031F48F5F8093F50761E0A4
:105320000E94DE1C81E080932A07109259070AC070
:10533000D23041F4109259078091C7010E94526106
:105340001092C7018091F5078093F407DF91CF9108
:105350000895CF92DF92EF92FF92CF93DF93FC01FB
:10536000EB019C01DC010E94336F9B01AC01DE016B
:105370000E94496F272F382F492F5527DF010E94A0
:10538000496F6B017C013CE0F694E794D794C79495
:105390003A95D1F724E630E02C1B3D0B0E94336F89
:1053A0006E5C7F4F8F4F9F4F6C0D7D1D8E1D9F1D1F
:1053B00024E630E040E050E00E94946FC901DF91A4
:1053C000CF91FF90EF90DF90CF9008951F93CF93F0
:1053D000DF936115710529F1192F111F1127111F75
:1053E00019F091958195910977FF10C0719561959C
:1053F0007109C0E0D4E09E01281B390BC9010E944D
:10540000A9299E01281B390BC90102C00E94A929A4
:10541000112329F022273327281B390B01C09C01B7
:10542000C901DF91CF911F9108956F927F928F9262
:10543000AF92CF92EF920F93CF93DF93CDB7DEB7BA
:10544000382F562F822F602F9C2D442321F0552377
:1054500029F022E00AC020E000E008C0E0915C01F1
:10546000F0915D0121E0EF2BB9F301E0442311F04D
:10547000311121E03EE0E39E30011124A3014157A8
:105480005C4F3A01933639F4FA0144850E94C827EB
:10549000F30184872AC0923639F4FA0145850E94C7
:1054A000C827F301858721C04A2D50E0490F511DBF
:1054B000490F511D440F551F480D511D460D571DD5
:1054C000FA013F01A11007C04081E22E04E62CE959
:1054D0000E941D1E08C040814C59E22E04E620E0C7
:1054E0000E941D1E8456F3018083DF91CF910F919E
:1054F000EF90CF90AF908F907F906F9008952F9204
:105500003F924F925F926F927F928F929F92AF9253
:10551000BF92CF92DF92EF92FF920F931F93CF93A0
:10552000DF9300D000D000D0CDB7DEB7182F8EEAC1
:105530009DE00E94CD1E93E0A92EC12C2DEAE22E03
:105540002DE0F22E00E020E030E040E0612F85EE1B
:1055500097E00E947B20109271014091F1074F5F0C
:1055600020E060E080E30E943110F090E507809138
:10557000F1070E94801E182F8091F107E82FF0E0BC
:10558000EE0FFF1FEE55F84F208131812A31310592
:105590001CF01092E40706C0273E3F4F1CF491E038
:1055A0009093E4070E94F01581111092E40768EAD5
:1055B0007DE080E10E94685D41E0F11040E0809074
:1055C000E407A12CC12EE090F10700E126E361E0A1
:1055D00081E00E94152A61EA7DE088E10E94685D11
:1055E00041E0F41240E08090E407AA24A394C12E85
:1055F000E090F10708E126E361E081E00E94152ACE
:105600006BE97DE080E20E94685D41E0E2E0FE122D
:1056100040E0812CA12C83E6C82EE090F10700E247
:105620002EE161E081E00E94152A65E97DE088E2D3
:105630000E94685D41E0F3E0FF1240E0812CA12C64
:1056400002E6C02EE090F10708E22EE161E081E081
:105650000E94152A113029F0123031F467E87DE0FC
:1056600005C06EE87DE002C06FE77DE080E30E9448
:10567000685D2091F1078EE0289F9001112494E04D
:10568000199F200D311D11242B513E4FF901E65574
:10569000FE4FD901A555BE4F1C91D901A455BE4F4F
:1056A000FC9084E6F80ED901A355BE4F0C910C591D
:1056B00080810E94E215682E812F0E94E215382E0B
:1056C00044E660E08F2D0E94C915782E44E660E024
:1056D000802F0E94C915582E8091F1070E94F01565
:1056E000E62DFF27E7FDF095FE83ED83E72CFF24F1
:1056F000E7FCF094882309F464C0812C912C5401B8
:1057000010E0A4E6CA2ED12CB0E44B2E6D817E8130
:10571000D501C401B595A795979587950E94E6296F
:10572000880F991F61E270E00E94806F6E9DC0013A
:105730006F9D900D7E9D900D11240FE3010FB6011A
:105740000E946C6FF42DF61B6F2F802F0E94B35DAB
:10575000812F837051F46FE3802F0E94B35D612F1E
:105760006695605E8FE30E94B35D1F5F21E2820E4B
:10577000911CA11CB11C1E3349F6E091F107F0E029
:10578000EE0FFF1FEE55F84F008111814801AA244A
:1057900097FCA094BA2CC501B40121E230E040E0AE
:1057A00050E00E94B66F4EE361E08EE5820F0E94EA
:1057B000035E8091F1070E94F015882309F4ABC0C5
:1057C0006CC000E010E0912C31E2C32ED12C44E6F5
:1057D000A42EB12C50E2252E832D992787FD90957C
:1057E0009A838983E52DFF27E7FDF095FC83EB8302
:1057F0006D817E81C8010E94E629B6010E94806FFA
:105800006E9DC0016F9D900D7E9D900D11242EE523
:10581000822E890CB5010E946C6FF22DF61B6F2F42
:10582000882D0E94B35D292D2370422E49F460E239
:10583000882D0E94B35D60E2690D8EE50E94B35D24
:1058400069817A81C8010E94E629B6010E94806FB1
:10585000EB81FC816E9FC0016F9F900D7E9F900D2C
:105860001124BEE58B2E8918B5010E946C6F605E15
:10587000882D0E94B35D411009C060E2882D0E940E
:10588000B35D622D69198EE50E94B35D93940F5D3F
:105890001F4FFFE19F12ACCF70CFC501B4017C5FF9
:1058A0008F4F9F4F22E030E040E050E00E94B66F03
:1058B0006D817E81C9010E94E6299C01220F331F60
:1058C000A72D77FCAD5FA595A595BB27A7FDB09546
:1058D0000E942B6F29E130E040E050E00E94B66F5B
:1058E00069017A01CA01B9012FED3FEF4FEF5FEF78
:1058F0000E94B66F60E4620F4EE38FE30E94005E89
:10590000C701B60122E030E040E050E00E94B66FEF
:1059100069017A0135C0181419041A041B040CF02B
:10592000632C662D772767FD7095C8010E94E629D4
:10593000181419041A041B0414F4A72D01C0A52D72
:10594000A7FDAD5FA595A5959C01BB27A7FDB095CB
:105950000E942B6F29E130E040E050E00E94B66FDA
:1059600069017A01CA01B9012FED3FEF4FEF5FEFF7
:105970000E94B66F60E2620F4EE38FE30E94005E0A
:1059800029E130E0D8010E94426F412C512C3201B4
:105990005394A30192010E94B66FA90160E382E7CC
:1059A0000E946E5FA9E1B0E0A70196010E94496FD5
:1059B000A30192010E94B66FA90168E084E50E94EC
:1059C0006E5F181419041A041B045CF46D817E8147
:1059D000C80144970E94E6299601281B390BC9018A
:1059E0000AC0632D772767FD7095C80144960E9411
:1059F000E6298C199D0945E0489F9001499F300D8B
:105A00001124442737FD4095542FE3E0EE2E00E3A8
:105A100060E184E50E944F5E26960FB6F894DEBFE3
:105A20000FBECDBFDF91CF911F910F91FF90EF90EF
:105A3000DF90CF90BF90AF909F908F907F906F90AE
:105A40005F904F903F902F9008952F923F924F92EA
:105A50005F926F927F928F929F92AF92BF92CF92FE
:105A6000DF92EF92FF920F931F93CF93DF93CDB707
:105A7000DEB72B970FB6F894DEBF0FBECDBF182F41
:105A800087E79DE00E94CD1EF4E0AF2ECC24C394A6
:105A9000A5E7EA2EADE0FA2E0CE023E331E144E085
:105AA000612F83EE97E00E947B208091E307FF2423
:105AB000FA94F80E20915A072983811110927101EE
:105AC000103871F480E80E9452611092C701F7FC0F
:105AD00052C18FE79AE20E94AF1AF092F1074BC1D0
:105AE00045E65DE068E085E10E946E5D7FED672E32
:105AF00077E0772E82EA97E09F838E8310E11B8602
:105B00001A86EEE05E2EEF2DFF27E7FDF095FB8372
:105B1000EA83BA848B2D0E94801E982E84E0989E82
:105B2000900111243D832C83EA85FB855E9EC00194
:105B30005F9E900D1124820F931F8B519E4FDC01AD
:105B4000A355BE4FFC01E455FE4F3C91208132131A
:105B50000DC0FC01E555FE4FDC01A655BE4F31E0FE
:105B600020818C91281330E0432E01C0412CEE811E
:105B7000FF8181919191FF83EE839C01275E3F4FCE
:105B80002333310508F0412C79866886F301F080D3
:105B90008A31910534F4873E9F4F24F4FF24F39417
:105BA00001C0F12C8B2D0E94F015882319F0F12CE7
:105BB00044244394F301F08220E041E04B0D612F37
:105BC00080E00E94311033243394F110312C809105
:105BD000800781110AC021E080915C0190915D01F4
:105BE000892B09F420E0D22E02C0DD24D3942A812F
:105BF0003B818A859B852817390731F481E099819B
:105C0000911180E0282E01C0212CF3018080A12C6D
:105C1000C92CEB2C012F27E2422D6D2D80E00E9434
:105C2000152A2220C9F0DD20B9F04420A9F02A85E8
:105C30003B85529EC001539E900D1124EC81FD8145
:105C40008E0F9F1F81579C4FFC01EF0DF11D20818E
:105C5000FC01E30DF11D20832A813B818A859B8510
:105C60002817390739F481E09981913009F080E0F3
:105C7000282E01C0212CEFEF6E1A7E0AE885F985E7
:105C80008080AA24A394C92CEB2C012F29E3422D58
:105C90006D2D80E00E94152A2220C9F0DD20B9F088
:105CA0004420A9F02A853B85529EC001539E900D49
:105CB0001124EC81FD818E0F9F1F8F569C4FFC019C
:105CC000EF0DF11D2081FC01E30DF11D20832A81E0
:105CD0003B818A859B852817390721F441E099810A
:105CE000923009F040E0812CA12C63E6C62EEB2C0B
:105CF000012F2FE36D2D80E00E94152AEA81FB81A0
:105D00002A853B85E217F30721F441E039813330DE
:105D100009F040E0812CA12C52E6C52EEB2C012F7E
:105D200027E56D2D80E00E94152A411004C0FF2058
:105D300029F04FE701C04DE28AE302C04EE78BE352
:105D4000612F0E940F5D81E0981629F092E0991270
:105D500004C04CE403C04DE401C048E4612F85E772
:105D60000E940F5DEA85FB853196FB87EA87185F05
:105D7000103309F0CECE2B960FB6F894DEBF0FBECF
:105D8000CDBFDF91CF911F910F91FF90EF90DF90EA
:105D9000CF90BF90AF909F908F907F906F905F90CB
:105DA0004F903F902F90089590E0E92FFF27E7FD57
:105DB000F095E95FFD4EE491E81302C0892F089544
:105DC000EE2311F09F5FF1CF80E00895823430F42C
:105DD000E82FF0E0E95FFD4E8491089580E2089598
:105DE000FF920F931F93CF93DF93C82FD62FF42EDC
:105DF000122F622F842F0E94CE11FC01E53F81E01B
:105E0000F80794F09BE09E0F9F1510F09CE09E0F0A
:105E100040E3490F202F6D2F8C2FDF91CF911F91E1
:105E20000F91FF900C945D5C212F43EA5BE06D2F96
:105E30008C2F0E94345DDF91CF911F910F91FF90C5
:105E40000895BF92CF92DF92EF92FF920F931F932C
:105E5000CF93DF93C82F86E89BE00E94CD1E06E01B
:105E6000E02E0CE023E331E143E06C2F8CED97E072
:105E70000E94D422B090DC07C03611F0CE3669F40F
:105E80008FEF8B0D843048F48093F7078C2F0E949E
:105E900052618FE89FE20E94AF1A6DE77BE088E0D5
:105EA0000E94685DC5EED1E010E1F12E11E0CC2436
:105EB000C3941B11C12C6AE77BE08F2D0E94685DA3
:105EC00040E3410F6F2D8CE00E940F5D2C2DFE01F1
:105ED000E353FD4F40816F2D8AE20E948310BAE5A3
:105EE000DB2EE12C0C2D2E2D412F6F2D8D2D0E94A0
:105EF000F02EE39486E0D80E84E0E812F3CF1F5F23
:105F000088E0F80E2A96153091F6DF91CF911F9117
:105F10000F91FF90EF90DF90CF90BF9008956F9218
:105F20007F928F929F92AF92BF92CF92DF92EF9229
:105F3000FF920F931F93CF93DF93C82F8090F707A3
:105F40002AE0829E40011124C40186559B4F4C01DA
:105F50008BE99BE00E94CD1EAA24A394CC24C39479
:105F600029E9E22E2BE0F22E00E020E030E040E0D4
:105F70006C2F8DED97E00E947B204091F7074F5CDE
:105F800060E080E30E940F5DC090DD0760908007B5
:105F900018E0E12CF12CDD24C7FCD0948E2DCE141A
:105FA000DF0429F416142CF492E0A92E04C0A12CCD
:105FB00002C0AA24A394813081F062E97BE0812FA2
:105FC0000E94685D0A2D2A2DF4014085612F80E32F
:105FD0000E94C827F401808751C06CE87BE0812FC4
:105FE0000E94685D80E3782EB12C80915A078B1552
:105FF00011F000E001C00A2D4091F7074F5F2B2DF3
:10600000612F872D0E94F02EAA2091F120915A072E
:106010002B112EC0161434F080915C0190915D011B
:10602000892B31F1E401C20FD11DC20FD11DE881CE
:10603000F981CF018B509E4F843FF1E09F0714F40C
:1060400084EF91E022E048EF51E064EF71E00E94BC
:106050005A12AC0180916401882351F0443F21E041
:10606000520711F440E050E0455F514059834883A6
:10607000B39486E0780E94E0B912B7CFEFEFEE1A42
:10608000FE0A185F183109F089CFDF91CF911F9177
:106090000F91FF90EF90DF90CF90BF90AF909F90C7
:1060A0008F907F906F900895CF93C62F0E9452617A
:1060B0000E944458C093FF048C2F0E94A7568091E1
:1060C000EF010E945F1382E080930F0181E00E9444
:1060D000A5570E94445881E0CF910895BF92CF9276
:1060E000DF92EF92FF920F931F93CF93DF93D82FFE
:1060F0008AEF9AE00E94CD1E80918007811110C026
:10610000E0917D07E7FF0CC0E195EC3008F0EBE093
:10611000F0E0EE0FFF1FED5CFE4E859194915BC0A9
:106120001091DA074FE06D2F8AED97E00E94E5228B
:1061300064EF7AE080E00E94685D0E94B858AC018C
:1061400060E086E60E946E5F41E06CE080E00E94C5
:10615000831CC091DA0780912907823021F41092C4
:10616000D90710922907D63638F4D436F0F4D03651
:10617000E9F1D13659F05EC0D13809F440C0DF3BB7
:1061800009F44FC0D03809F055C03DC08091D907FF
:10619000882359F01092D90787E10E943F6C6091E3
:1061A000DA0781E60E94543045C08091FF048C17C5
:1061B00039F06C2F8D2F0E94543081E00E943F6C8B
:1061C000D53629F48AE194E20E94331333C0D436E1
:1061D00089F58CEB9DE4DF91CF911F910F91FF909A
:1061E000EF90DF90CF90BF900C94331381E08093B9
:1061F000D9071092800787E10E943F6C1BC081E0A5
:106200000E948C1A17C08091D907882399F081E0E9
:1062100080932907C093280783E798E20E94AF1A6A
:1062200009C01092D9078091FF048093DA0781E0BA
:106230000E94B7578091D907882341F01C1731F08D
:1062400061E06C0F81E0810F0E947359DD27C7FD6B
:10625000D095809181079E01281B3109C90118162C
:1062600019065CF0CE01019797FF02C080E090E034
:106270008093810710E1B12C0BC025303105D4F398
:10628000CE0104978B3091059CF38AE090E0F0CF2B
:10629000F0908107FB0CCF2CD12CCC15DD0511F42F
:1062A00001E101C000E196012F5F3F4F442737FD18
:1062B0004095542F62E0E62E612F82E10E944F5EEE
:1062C0008091FF04F81205C04AE2612F81E00E942C
:1062D0000F5D4FE06DE277E08F2D0E947056CC1578
:1062E000DD0531F48091D907882311F001E101C067
:1062F00000E12FE04DE257E0612F88E10E94125D3E
:10630000B394185F36E0B312C3CFDF91CF911F91E2
:106310000F91FF90EF90DF90CF90BF900895DF92A4
:10632000EF92FF920F931F93CF93DF93E82E00918C
:10633000F001C1EBD7E010916004202F332727FD37
:10634000309537FF03C0319521953109253231054C
:1063500054F12D853E854F855889242B352B4B854F
:106360005C85242B352B8989282B8A89282B232B84
:1063700029F4802F881F8827881F8A8B101614F411
:106380008CED01C084E2800F40E060E00E941316B3
:10639000882341F09A89911105C091E02989211142
:1063A00090E0998B8A8B112339F040E060E0812FD7
:1063B0000E941316882319F0FF24F39402C0F12CD5
:1063C000E12C2D853E852F5F3F4F3E872D872F8502
:1063D00038892E0D311D388B2F87F89420915A0C57
:1063E00030915B0C78948B859C85281B390B243667
:1063F000310508F423C18C599F4F9C878B872F85CB
:106400003889ED85FE85C901BF010E946C6FE62EBB
:10641000D62E6E9FC0016F9F900D1124281B390B43
:10642000388B2F871E861D868FE0800F8F3110F4EA
:10643000198A0DC094E2900F993448F4101614F4A0
:1064400081EF800F40E060E00E941316898B20915D
:10645000F001332727FD309537FF03C03195219593
:106460003109622F88819981019699838883EA8115
:10647000FB813196FB83EA83DD2029F08E819F81A9
:1064800001969F838E83613009F4698B8989882303
:1064900041F0FF2031F04C815D814F5F5F4F5D83A4
:1064A0004C83E694488559854E0D511D5987488780
:1064B000E090F201F090F301FC8AEB8A611102C0D6
:1064C0001A8620C0613031F4111114C0C7018E1B2F
:1064D0009F0B16C0603170F420FF06C0E4E05695B3
:1064E0004795EA95E1F702C04E815F81C701841BA1
:1064F000950B06C08C819D819701281B390BC90122
:106500009C8B8B8B8A850B891C89813049F018F014
:10651000823069F017C08091F001882399F010C093
:1065200017FF10C0E114F10469F082E00AC0053CD5
:106530003FEF130714F483E08A87E114F10411F4A8
:1065400081E08A87898D9A8D8017910709F46AC046
:106550008A85813009F057C08091180582FF31C0CB
:10656000E114F10471F10E31110519F469E289E1C8
:106570000BC00431110519F46AE28AE105C00A3042
:10658000110531F46BE28BE10E94456C81E00DC096
:10659000063011054CF417FD03C0602F8CE1F4CFD9
:1065A0008CE10E943F6CF2CF80E09091180593FF40
:1065B00008C0882331F082E390E0909358018093E3
:1065C00057018091F10180FF04C0C701801B910B2E
:1065D00001C0C8016CE370E00E94806FDC01CB0158
:1065E0004091180541FF1EC0AB2BE1F440912105FD
:1065F00041FF07C0009761F046E260E00E944E6CE8
:1066000007C080E003C0823069F48CE10E943F6CD7
:106610008091180583FF06C082E390E090935801B3
:10662000809357018B899C899A8F898F2091F101E2
:1066300020FF04C0E81AF90AFC8AEB8ADF91CF91A7
:106640001F910F91FF90EF90DF9008959091F001CE
:1066500097FD91958EEF890F8E3020F5892F8595C6
:106660009A3024F40E94696290E003C0992787FD64
:1066700090950197FC01EE0FFF1FEE55F84F20811A
:1066800031818091F00187FF05C080E094E0821B9A
:10669000930B02C0C9019C5F26E0969587952A95C9
:1066A000E1F702C080E090E00E948F3183E00E9419
:1066B0006962E82FF0E0EE0FFF1FE056F84F80818F
:1066C00091819C5FB6E096958795BA95E1F7209108
:1066D000F10122FF0AC08530910538F02091C807EA
:1066E000211103C023E02093C8072091D1073091E6
:1066F000D2072F5F3F4F3093D2072093D1072091CD
:10670000CF073091D007280F391F3093D00720933F
:10671000CF07F89480915A0C90915B0C789420915B
:10672000CD073091CE07AC01421B530B9A01283E96
:106730003340D8F19093CE078093CD078091F40138
:10674000823039F440E060E085E10E941316811147
:1067500028C08091CF079091D0076091D1077091A8
:10676000D2070E946C6F1092D0071092CF07109240
:10677000D2071092D1078091AE06893718F48F5F47
:106780008093AE06E091AF0681E08E0F8093AF0656
:10679000F0E0E055F94F6083883738F01092AF068B
:1067A000089587E00E943F6CD4CF0895E1EBF7E0B5
:1067B0001286138212821782168215821482118623
:1067C00010868091F2019091F301928F818F08954C
:1067D000CF92DF92EF92FF92CF93DF936B017C0118
:1067E000C0E1D0E040E050E8E0E0F0E89A01DA01F2
:1067F0000E94336FC616D706E806F90610F44E2736
:106800005F27F695E7952197209719F04E2B5F2B80
:10681000EDCFCA01DF91CF91FF90EF90DF90CF9045
:1068200008951F9341E0262F30E0683050F440E097
:1068300055E0529FF001539FF00D1124E553FC4F9A
:106840000AC02850310959E0529FF001539FF00DC2
:106850001124ED50FC4F9C5F97FD0DC0811528E081
:10686000920784F0442319F088E090E002C084E0AD
:1068700090E0E80FF91F2081332727FD3095322F54
:10688000222725C0442329F0492F9927880F991FD3
:1068900003C0492F46959170242F30E0E20FF31F7B
:1068A000608140E052E0481B590B559547956403C1
:1068B0009001659F300D11241181BC01759567957C
:1068C0001603A001179F500D1124240F351FC90175
:1068D00069E170E00E94806FCB011F9108953F92A3
:1068E0004F925F926F927F928F929F92AF92BF92E0
:1068F000CF92DF92EF92FF920F931F93CF93DF938C
:10690000982EBB24B3948091F607883008F4B12CFC
:1069100085E091E10E94CD1EBB2011F08AE001C00C
:1069200086E0A82ECC24C394F3E0EF2EF1E1FF2EF5
:1069300000E020E030E040E0692D8FEE97E00E941B
:106940007B204091F60750E04F5F5F4F21E060E011
:1069500084E20E945F5FC091F607BB2061F08C2F3C
:1069600090E0089729E0289FE001299FD00D11248D
:10697000CD50DC4F06C025E0C29FE0011124C55375
:10698000DC4F6090EF076A94A0905A0741E6941696
:1069900081F0491538F054E49516E1F085E4981635
:1069A00089F02EC0E4E69E16A9F0F5E69F1651F098
:1069B00027C0AA2029F110925A0781E60E9452614D
:1069C000A12C1EC0809180078823D1F01A14C4F432
:1069D0008FEF13C080918007882391F02A2D3327F1
:1069E00027FD3095BB2019F089E090E002C085E0DA
:1069F00090E02817390724F481E08A0D80935A0724
:106A000080915A07809380078C2E7D2ECC2EDD2E10
:106A100005E010E0E0E15E2EE62CFF24E7FCF094B8
:106A2000F60141916F0121E0C8010597E816F906CA
:106A300009F020E0552747FD5095652D88E10E941B
:106A40005F5FBB2091F0093081F021E0E016F10694
:106A500009F020E0FE01E00FF11F4081552747FDBE
:106A60005095652D80E30E945F5FF8E05F0E0F5F39
:106A70001F4F28E35212D4CF4FEF641202C021E01F
:106A8000A11020E04CEF50E168E08CE00E94485DEE
:106A9000BB2019F089E090E002C085E090E021E0A1
:106AA000E816F90609F020E045EF50E168E38CE0D4
:106AB0000E94485DBB2019F089E090E002C085E0AB
:106AC00090E0E816F9066CF467FC50C0EC0EFD1E71
:106AD00044E66CE9F70180810E941913F701808375
:106AE00045C016140CF042C020E044E06CEF8091E9
:106AF000EE070E940D138093EE0790916401992395
:106B0000A9F1BB2021F090E164E049E003C098E0E6
:106B100062E045E0F4E68F028001112470E0719597
:106B200061957109582F56039001579F300D11241C
:106B300084E6829F6001839FD00C1124E82DF72DFD
:106B400020E030E0E92EF12CC9018C0D9D1DB7012C
:106B50000E94806F6193200F311F8E2F8819841738
:106B600098F382E00E94A5570E94445880918007C4
:106B7000882309F459C0712C7CE9E72EFF24FA948C
:106B8000CA2CDD24C7FCD094892D8F7DA82EEEEB76
:106B9000AE0E40C0C90155E0880F991F5A95E1F724
:106BA000BB2009F44AC064E070E00E94806F462E6A
:106BB0004E01820E931EF4018081F0E28F02C0012B
:106BC0001124B7010E94806F662E40E2542E560EAB
:106BD0002F5F3F4F052D10E0C216D30609F05EC0AF
:106BE000023411056CF12FE3251530F045E0652DD9
:106BF0008AE3840D0E94005E0F331105A4F1809199
:106C00005C0190915D01892B09F03FC051E05A155C
:106C1000E0F57394272D30E0BB2061F089E090E02F
:106C2000281739070CF4B6CFC0E0DCEF10E060E2C3
:106C3000F62E52C085E090E0F3CF62E070E0B5CF71
:106C40003AE3332E340C45E06EE1660D832D0E944D
:106C5000005E0134110539F245E06FE1660D832DC8
:106C60000E94005EC0CF4AE3440E45E061E2660D3B
:106C7000842D0E94005E0E33110509F262E2660D5A
:106C800045E0842D0E94005EBACF44E66CE9F40131
:106C900080810E941913F4018083BBCFFBE34F0E68
:106CA0000134110534F443E06FE1660D842D0E9438
:106CB000005E2FE3251528F043E0652D842D0E940A
:106CC000005E0F3311050CF0A4CF61E2660D43E0C6
:106CD000842D0E94005E9DCF6091F607CE010E9438
:106CE00011340CE3010F25E0969587952A95E1F77D
:106CF0006F2D681B802F0E94B35D812F837021F45C
:106D000060E2802F0E94B35D1F5FA096103421F7D0
:106D100040E460E08CE5DF91CF911F910F91FF90EF
:106D2000EF90DF90CF90BF90AF909F908F907F902B
:106D30006F905F904F903F900C94035E2F923F9224
:106D40004F925F926F927F928F929F92AF92BF927B
:106D5000CF92DF92EF92FF920F931F93CF93DF9327
:106D6000CDB7DEB76E970FB6F894DEBF0FBECDBFBE
:106D70008D8F9E8F698780915901882309F44EC0B9
:106D800080917E07882319F0815080937E070E94AE
:106D90005A1420916706309168068217930761F0B4
:106DA000909368068093670610926A0610926906AF
:106DB00081E08093560132C060911705665F71F1E2
:106DC00080910201823350F180916B068F5F809336
:106DD0006B06803118F18091690690916A060196E0
:106DE00090936A068093690610926B0647E751E01C
:106DF000649F9001659F300D11242817390770F4A6
:106E00008F719927019751F486EF9FEF0E944913E4
:106E10006DE280E10E94456C0E9467130E94D11AC6
:106E200080934D0580911605282F2170822E839422
:106E300081FF02C0612C02C033E0632E4091FD014E
:106E40004423F1F1E82DF0E0EE0FFF1FEE55F84F6F
:106E5000A081B181E62DF0E0EE0FFF1FEE55F84F57
:106E60000190F081E02D9D010E942B6F6B017C0150
:106E70009F01DF010E942B6FC60ED71EE81EF91E70
:106E8000642F70E080E090E02AE0660F771F881F93
:106E9000991F2A95D1F724E630E040E050E00E94A7
:106EA000B66FCA01B9010E945C6F6C157D058E0535
:106EB0009F0530F4C701B6010E94E8337C0102C08F
:106EC000E12CF12C9701A4E6B0E00E94336F6D8BAA
:106ED0007E8B8F8B988FB3ED4B2EB4E05B2E4EE004
:106EE00056E05C874B87BE016F5F7F4F7E876D8763
:106EF00082EA97E09A8B898BC12CD12C712C9985D1
:106F00009170998FA985AE70AA8FB985BA70BB8F21
:106F1000E985E670EC8F9C2C8C2D0E944A1492011E
:106F20002E5F3F4F388B2F87D2012D913C91821BD2
:106F3000930B9C01BC01882777FD8095982FAAE0D0
:106F4000660F771F881F991FAA95D1F7EF85F889DB
:106F5000121613061CF4228D338D02C0248535854C
:106F60002436310514F424E630E0442737FD4095FB
:106F7000542F0E94B66F89012130FCEF3F073CF08F
:106F8000011524E012072CF000E014E002C000E03C
:106F90001CEF8091180580FF11C08091160581704B
:106FA0008B8B1C8A82E090E04B895C89841B950B5B
:106FB000C816D90619F4119501951109A989BA893C
:106FC0000D931D93BA8BA98B580117FF03C0BFE027
:106FD000AB0EB11CF4E0B594A794FA95E1F73A2C06
:106FE000E4E0CE16D1045CF481E0890D0E94696270
:106FF000815091E001C0990F8A95EAF706C091E0AF
:107000000C2C01C0990F0A94EAF737FE02C03A2C03
:107010003194F1E0F31544F0311002C0892F03C020
:10702000809166068923782A23E0291508F422C175
:10703000398D31114DC08091F10181FF49C052015C
:1070400049E3A40EB11CF5018181807C09F440C0A4
:10705000F20181AD40E061E08595859585950E94BE
:1070600013168823A9F1D501EC91E770F0E0DF0158
:10707000AA0FBB1FAA5BBE4FEE0FFF1FEC5FFA4FBC
:107080008D919C9120813181821B930B97FD0196FC
:10709000AC0155954795F5012181322F330F330F00
:1070A000359535953403C001359F900D11246FE15E
:1070B00070E00E94806F660F771F660F771F229522
:1070C000269526952370213009F08FC6060F171FCD
:1070D000E114F104C1F0981411F0961014C020913D
:1070E000FD0130E0D8010E94426FEAE0660F771F91
:1070F000881F991FEA95D1F72D893E894F89588DB0
:107100000E94B66F8901892D0E94801EA82E892DAC
:107110000E94F015EA2DF0E0882311F1EE0FFF1F19
:10712000EE0FFF1F2EE02C9DC0012D9D900D112410
:10713000E80FF91FE157FC4F80810E94E215682F8C
:10714000772767FD7095C8019C5F97FD019695951F
:1071500087950E94E6298C01000F111FB12C24C0D5
:1071600081E0101611060CF480E0B82E3EE03C9D44
:10717000C0013D9D900D1124EE0FFF1FEE0FFF1F6C
:107180008E0F9F1F8B519E4F8B0D911DFC01E6555D
:10719000FE4F80810E94E215682F772767FD70956A
:1071A000C8010E94E6298C014EE04C9DC0014D9D16
:1071B000900D112454E0A59E800D911D11248B513A
:1071C0009E4F8B0D911DFC01E455FE4F808144E6DE
:1071D00060E08C590E94C9159801A82FBB27A7FD14
:1071E000B0950E942B6F24E630E040E050E00E9412
:1071F000B66F8901892D0E94F01581111450892DD7
:107200000E94E615811106C0692D80914D050E94EE
:1072100014122AC08091F60180FFF6CF692D80916B
:107220004D050E941412282F8091180580FD21958C
:10723000332727FD3095432F532F23583F4F4F4F70
:107240005F4FA0E0B4E0A01BB10B0E94546F20E0A0
:1072500038E040E050E00E94B66F211568E0360744
:107260004105510589F2C901880F991FAD85BE8579
:107270008D939C93EB85FC8511830083FA8DFF230E
:10728000F9F023E02915E0F0892D0E94E61581111F
:1072900013C03B8D332349F0065F1F4F05311105A5
:1072A00020F0AB85BC851D921C92BC8DBB2321F0C8
:1072B000ED85FE8511821082EB85FC85118E108E86
:1072C000FFEFCF1ADF0A2B853C852E5F3F4F3C87AF
:1072D0002B874D855E854E5F5F4F5E874D8757E0FC
:1072E000C516D10419F04F84588815CE1091FA01B3
:1072F0001721809166068095812319F088E10E940C
:107300003F6C1093660680E094E090931D06809396
:107310001C0690931F0680931E0682E10E94016165
:10732000811108C083E10E940161882331F080E06F
:1073300090E005C080E09CEF02C080E094E0909374
:1073400057068093560626E431E006E216E0E4E0B4
:10735000F5E060E0D9018D919D919D01643020F4AC
:1073600040815181841B950B880F991FD8018D9303
:107370009D938D016F5F3296683061F726E336E0AA
:10738000ECE6F6E04191519161917191D9014D93F3
:107390005D939D01B6E0EC3AFB07A1F7ECE9F4E060
:1073A000A8E5B6E0808128E08202C00111248D9317
:1073B0009D93329634E0EA3AF307A1F7A090FD01DD
:1073C000AA2009F46EC0E82CF12CEE0CFF1CA701DA
:1073D000425F594F7A01DA01CD90DC90062D10E022
:1073E000000F111F025F194FF80140815181960172
:1073F000D6010E942B6F1B012C019A01DA010E9419
:107400002B6F260E371E481E591E6A2D70E080E035
:1074100090E0EAE0660F771F881F991FEA95D1F781
:1074200024E630E040E050E00E94B66FCA01B901A6
:107430000E945C6F621573058405950590F5C20185
:10744000B1010E94E8339C01A4E6B0E00E94336FD2
:107450001B012C01B12C9501D6010E94426F2AE03C
:10746000660F771F881F991F2A95D1F7A2019101F6
:107470000E94B66FD7012D933C93F801A081B18192
:1074800095010E94426F3AE0660F771F881F991F8F
:107490003A95D1F7A20191010E94B66FD8012D93C0
:1074A0003C936091FB01862F807E09F4F8C08985AA
:1074B0008A7089F4E82DF0E0EE0FFF1FE25FF94FCC
:1074C00020813181E62DF0E0EE0FFF1FE25FF94FE2
:1074D0008081918104C080E090E020E030E0498527
:1074E0004670A1F4FE013196E80DF11DE80DF11D85
:1074F00040815181240F351FFE013196E60DF11DAB
:10750000E60DF11D40815181840F951FE091FC0132
:10751000EE2341F0F0E0EE0FFF1FE45FF94F4081F2
:10752000518102C040E050E062FF03C031952195D7
:10753000310963FF03C091958195910964FF03C0F0
:10754000519541955109629566956770623009F4CD
:1075500051C018F46130E1F0A2C0633009F489C071
:10756000643009F09CC0FA01E21BF30BF093210692
:10757000E09320069A01280F391F309323062093A9
:107580002206481B590B509325064093240687C0BA
:10759000BC0197FF02C0695F7F4FB3E075956795A7
:1075A000BA95E1F7FC01E61BF70BBC0197FF02C09F
:1075B00061587F4F660F672F661F770BE61BF70B2F
:1075C00097FF02C081509E4FBC01672F770F770B4A
:1075D0006595CF01861B970BBA01621B730B7093E5
:1075E00021066093200637FF02C02F5F3F4F35957D
:1075F000279546C0B90137FF02C0695F7F4F13E08E
:10760000759567951A95E1F7F901E61BF70BB90136
:1076100037FF02C061587F4F660F672F661F770BD9
:10762000E61BF70B37FF02C021503E4FB901672F11
:10763000770F770B65959F01261B370BBA01681BE7
:10764000790B709321066093200697FD019695951E
:107650008795840F951FAC01420F531F509323064B
:1076600040932206821B930B909325068093240659
:1076700016C0BA01621B730B70932106609320063B
:10768000240F351FA901480F591F5093230640931B
:107690002206281B390B309325062093240680915F
:1076A000590181110E94263380E4ECE6F6E0DF0107
:1076B0001D928A95E9F787EC93E0909304018093FB
:1076C000030188EC93E0909306018093050189EC17
:1076D00093E090930801809307018AEC93E09093E4
:1076E0000A0180930901EEEEF5E0FA87E9872EE8BA
:1076F00035E0388B2F874EE455E05E874D87312C7F
:10770000212C832D0E94AE0F7C01FC0182810E94FE
:10771000E2158B87D7018C918150803108F06AC2C5
:1077200040E061E0F70183810E941316811116C0C9
:10773000A985BA85DC901C92F701918188EF890FA9
:10774000823008F041C287818670843009F43CC2DF
:10775000993009F047C000E01CEF46C0DD24D39407
:10776000A985BA858C918111D12C81E0E985FA85B2
:107770008083F70121818FEF820FA82FB0E0FD01F8
:10778000EE0FFF1FE25FF94F00811181843150F04D
:10779000831540F4AA0FBB1FAA0FBB1FA459B94FF2
:1077A0000D911C91F7013781832F807361F0832F36
:1077B00082958370815041E050E002C0440F551F14
:1077C0008A95E2F7242A36FF0FC0253068F4E22FAD
:1077D000F0E0EE0FFF1FEF5FFE4FC70108969183A9
:1077E000808302C000E010E0F7018781887459F4BB
:1077F0008085882341F04DE763E80E94C9150E9407
:10780000FE15080F191FF701F681FB8B2B85332717
:1078100027FD30953A8B298BF11105C0F701858141
:10782000882309F4F0C0AD85BE85AD90BC90EF858E
:10783000F88980819181A2819C014A2F552747FDBB
:10784000509529013A01D1100AC0BB2757FDBA95BE
:10785000A52F942F832F6801C81AD90A3EC0F701BB
:10786000878186708430D9F4E081F0E0EE0FFF1F4D
:10787000EC5CF94FA081B18120E034E60E94426FB8
:107880002B013C01FB85FF2351F02F2F332727FDD0
:107890003095432F532F0E94B66F29013A01C3013F
:1078A000B20120E031E040E050E00E94B66F509518
:1078B0004095309521953F4F4F4F5F4F6801C20E65
:1078C000D31EC114D10449F0F7018581D7FE8295FA
:1078D0008F70F4E68F9F50011124A114B10491F030
:1078E00080915901882331F021E0A21AB108A11436
:1078F000B10441F0332777FC3A95272D162D052D3D
:10790000C12CD12CAD85BE85AD92BC92C114D104E1
:1079100009F474C04801AA2497FCA094BA2CBB892E
:10792000BB2309F467C080915901882309F443C03F
:10793000EB85EE23A1F029893A8937FF03C0319501
:1079400021953109442737FD4095542F60E070E0C0
:1079500080E293E00E94B66FCA01B90104C060E002
:1079600070E080E293E0F70126811C141D0444F0CE
:1079700090958095709561957F4F8F4F9F4F229581
:107980002F7030E02115310591F0E4E6E29FA0016F
:10799000E39F500D11249A01442737FD4095542F41
:1079A0000E94B66F420E531E641E751E04C044240E
:1079B000582C692C7A2CBB2777FCBA95A72D962DCD
:1079C000852D1C141D0434F488169906AA06BB06DE
:1079D00034F009C088159905AA05BB0524F4442490
:1079E000582C692C7A2C332777FC3A95272D162DA5
:1079F000052D04C04424582C692C7A2CAF85B889F5
:107A00004D925D926C92F701878187FF28C044E612
:107A10006CE984810E94C915A82FBB27A7FDB095EA
:107A20001A161B0644F417FF6AC024E630E02A1B2E
:107A30003B0BD90109C0109709F461C0101611065B
:107A40000CF05DC0AC59BF4F98010E942B6F24E62B
:107A500030E040E050E00E94B66F890150C0F7016D
:107A60006481862F992787FD9095A92FB92F87309C
:107A7000910590F5FC01EC5AFF4F0C94D56FF7017E
:107A80008181893021F417FD35C012500BC017FFDA
:107A900036C01BC0F7018181893039F410161106F8
:107AA00064F11E5F000F111F2AC0101611066CF042
:107AB00026C017FF24C011950195110920C010168A
:107AC0001106DCF002C017FD15C000E010E017C081
:107AD0001016110694F00EC067FF06C011950195AF
:107AE0001109F6E0F61B6F2F6750C8010E94113490
:107AF0008C0105C000E01CEF02C000E014E0F701BB
:107B0000478140FD10C081819FEF980F943058F459
:107B1000FE013196E80FF11DE80FF11D32978081CB
:107B20009181080F191F9801A989BA890E942B6FAA
:107B30004B015C014874483051F4F701808588237B
:107B400031F04DE763E80E94C9150E94FE15D70188
:107B50000C9110E001501109F7018781869583701F
:107B6000000F111F000F111F813071F0823029F1B9
:107B7000F801E459F94F80819181A281B381880E87
:107B8000991EAA1EBB1E19C0C501B40124E630E02F
:107B900040E050E00E94B66FF801E459F94F60816F
:107BA0007181828193810E945C6F20E034E040E02B
:107BB00050E00E94B66F49015A01F801E459F94FAB
:107BC00080829182A282B382339429853A852F5F85
:107BD0003F4F3A8729874F8558894D5F5F4F588BB4
:107BE0004F876D857E856E5F7F4F7E876D8770E2E4
:107BF000371287CD1091590C20FE05C0111103C01A
:107C00008EE10E943F6C21FE07C0812F877F803468
:107C100019F48FE10E943F6C22FE09C0812F877FFB
:107C2000803811F0103919F480E20E943F6C82E82C
:107C300097E09E878D879D8D9987AE8DAA8733E6C5
:107C4000232E34E0332EECE6F6E0FC87EB87E12CC4
:107C5000F12CEF86AB85BC854D905D906D907C904E
:107C6000C301B20124E630E040E050E00E94B66F6C
:107C7000EB85FC852193319341935193FC87EB87EE
:107C8000AD85BE852D933D93BE87AD878E2D0E9419
:107C9000B50F4C01FC01838194812181FAE02F0210
:107CA0006001112428E1C21A2CEFD20AD4012C91D0
:107CB000BAE02B0250011124E8EEAE1AE3E0BE0A4E
:107CC0003C2D2D2D8C159D0514F4382F292F032FB5
:107CD000122F0A151B050CF485014114510461048F
:107CE0007104A9F077FE04C0D801AA19BB0903C02A
:107CF000D601A01BB10BA30192010E94546F20EA90
:107D000036E841E050E00E94B66F29013A01C8010F
:107D10000E94B3158C01040D151DC6010E94B315F8
:107D20006C01C5010E94B315C016D1060CF4860182
:107D3000081719070CF48C01F4018281882319F0CB
:107D400011950195110980916104F0E1F81B2F85CF
:107D50002F17F8F4F701EE0FFF1FEE59FB4F90813C
:107D6000892F880F880F8595859599F0929596951E
:107D7000969593709D5F9370923058F040E060E06C
:107D80000E941316882329F0D1018C910E94FE15C0
:107D90008C01F894E985FA8501931193FA87E987B4
:107DA0007894FFEFEF1AFF0A22E0220E311C30E137
:107DB000E316F10409F04DCF6E960FB6F894DEBFCE
:107DC0000FBECDBFDF91CF911F910F91FF90EF902C
:107DD000DF90CF90BF90AF909F908F907F906F90EB
:107DE0005F904F903F902F900895223009F070C916
:107DF0008B016EC9FF920F931F93CF93DF93CDB783
:107E0000DEB7C054D1090FB6F894DEBF0FBECDBFA8
:107E100063E0CE0181960E949E3661E0CE0101961C
:107E20000E949E36E1E4F3E09E012F5D3F4F8E01FC
:107E30000F5F1F4F418152818081882329F0D90132
:107E40008D919C91D80104C0D8018D919C91D9014C
:107E50006D917C91861B970B840F951F883EB3E034
:107E60009B073CF489314CEF94073CF0482F892F55
:107E700002C048EE83E0942F02C098E18CEF91831A
:107E8000828335962E5F3F4F0E5F1F4F83E0E139AF
:107E9000F80781F607EC13E0F12C8F2D0E94E61510
:107EA000811102C0D8011C92F3940F5F1F4FB4E000
:107EB000FB12F3CF86E00E94A55781E00E943F6C41
:107EC000C05CDF4F0FB6F894DEBF0FBECDBFDF91B1
:107ED000CF911F910F91FF9008959F92AF92BF9203
:107EE000CF92DF92EF92FF920F931F93CF93DF9386
:107EF000C82F80911405282F2F70F22E80731092B6
:107F00007101C038E9F198F4C33209F462C030F469
:107F1000C03261F1C23209F46BC0ACC0C53209F4A1
:107F20004DC008F441C0C13609F484C0A3C0C438B0
:107F300081F158F4C23809F469C008F487C087EDAC
:107F40009FE10E94331383E868C0CE38C9F0CF3B6D
:107F500009F482C0C53809F08DC081E080937C07A8
:107F60008CEF96E40E94AF1A85E81BC043E024130F
:107F700081C08091C80791E089278093C8076AC0B3
:107F800081E080937C070E9429130E94AF1A8C2FF6
:107F900008C081E080937C078EE690E30E94AF1AD0
:107FA00084E80E94526166C052E0251363C080914C
:107FB000F0078F5F833054F080E008C082E0281320
:107FC00059C08091F007815087FD82E08093F007CF
:107FD00051C0F39493E09F1508F4F12C8F298093FE
:107FE000140581E00E94A55783E10E943F6C42C0C6
:107FF000222311F0FA9402C003E0F02E8F2980931F
:10800000140581E00E94A55784E1EFCF0E942E6DF8
:1080100088E49FE10E94331382E8DF91CF911F91A2
:108020000F91FF90EF90DF90CF90BF90AF909F9017
:108030000C9452618091BB07823021F483E08093DD
:10804000BB0708C0E3E02E1315C002C00E94D63360
:108050000E94421387E1C9CF81E00E94526183E010
:108060000E94526182E00E94526181E08093CC07BD
:108070001092F00740E060E08091F9010E94131631
:10808000C82F882331F08091CC07811102C00E9453
:10809000FA3EC093CC079091020180910105981798
:1080A00010F4C6E001C0C4E080E00E9491114C2FA2
:1080B000406860E185E20E942C1046E568E186E2B6
:1080C0000E940F5D8091BB078823A1F0823011F4DC
:1080D00026E001C024E04091C4075091C507022F5B
:1080E00060E18DE50E94BC0F20E040E068E183E3A1
:1080F0000E94B81000E02091F70145ED57E060E1E3
:1081000086E20E94345D8091F60180FF06C041ED59
:1081100057E060E188E30E946E5DC0E0D0E01FE1BF
:10812000D12EEC2EFE01E353F84F14916C2F809169
:108130004D050E94141297FD03969C0135952795D5
:1081400035952795243E0CF424EE022F2D310CF0AA
:108150000CE18FEF8E0D46E38230E0F464E0812F76
:108160000E94035E809116058E2580FD04C08091DB
:10817000F60180FD0CC043E06EE18FEF810F0E949D
:10818000035E43E06EE181E0810F0E94035E6D2D8E
:10819000601B14C06BE385EE810F0E94005EEE242D
:1081A000EA94E10E43E06AE38E2D0E94005E43E014
:1081B0006CE38E2D0E94005E100F6BE347E0812F71
:1081C0000E94A31E2196C430D10509F0AACFF1E088
:1081D000FF1508F47FC00BE517E0E12CF9E1DF2E75
:1081E000ABE1CA2EF801C191D1918F018E2D837020
:1081F000F1E0FF1641F19E01D7FF02C0215E3F4F23
:10820000E5E035952795EA95E1F7AE01421B530B62
:108210009A01D7FF02C0C158DF4FAE01440F452F6E
:10822000441F550B420F531F6E2D66956695660FC2
:10823000660F660F685D8C9D802D112420E28F5D96
:108240000E945F5F42C053E05E1518F062E2962E16
:1082500002C05EE5952EB82EBB0CBB0CB80E9E017D
:10826000D7FF04C0222733272C1B3D0BD29EA00131
:10827000D39E500D11249A013E5FA32EA594A59480
:1082800089E18A1514F449E1A42E25E543E366E269
:108290006B0D87EE890D0E94D05D45E064E26B0DA9
:1082A000892D0E94035E1C161D0614F4939401C0D0
:1082B0009A1867E26B0D4A2D892D0E94005E6B2D86
:1082C0006B5D4A2D892D0E94005EE39498E0E912CF
:1082D00089CF7CC0E2E0FE126FC00E94252680910B
:1082E000F007882329F0982F990F890F880F8D5F49
:1082F000182FC82FDD27C7FDD0956E01F2E0CF0EF5
:10830000D11CE12EFF24E7FCF094CE14DF04FCF036
:10831000BB24B394B10E40E060E08B2D0E94131695
:10832000082F0E94B510AC0123E01202400D511D30
:108330001124B7016C1B7D0B6C5F7F4F660F660FBE
:10834000660F23E08AE00E94125D1B2DDACF809138
:10835000F0078F5F182F110F180F110FC12FDD2796
:10836000C7FDD0956E0142E0C40ED11CE12EFF2462
:10837000E7FCF094CE14DF044CF1BB24B394B10EAF
:1083800040E060E08B2D0E941316082F0E94B5106C
:10839000AC01E3E01E02400D511D1124B7016C1B1E
:1083A0007D0B6C5F7F4F660F660F660F23E084E6E0
:1083B0000E94125D1B2DDACF4091C6075091C7076E
:1083C00004E024E068E28CE30E94BC0FDF91CF91CF
:1083D0001F910F91FF90EF90DF90CF90BF90AF90E3
:1083E0009F900895982F809181071916BCF4292F2A
:1083F000332727FD3095281B3109462F50E04217BF
:1084000053071CF4892F861B0AC0465051092417B4
:1084100035072CF4892F861B8A5F01C080E080938A
:1084200081070895BF92CF92DF92EF92FF920F9350
:108430001F93CF93DF93C82E4EE0682F87EE97E00F
:108440000E94E5228091F207882319F085EF9EE0D3
:1084500002C08BEE9EE00E94CD1E182F8091F50782
:108460000E94AE0FEC0120E0488160E086E0810FC1
:108470000E946110D090E70766E08D2D0E94F241C6
:1084800018E0F12CBB24B394409181074F0DEE24EA
:10849000E394D412E12C50E04F30510508F045C16F
:1084A000FA01E55AFF4F0C94D56F63EE7EE0812F01
:1084B0000E94685D2E2D20614981612F84E50E9414
:1084C0003110EE2009F431C14CE261E089810E9453
:1084D000191389832AC16BED7EE0812F0E94685DAC
:1084E0000DE723E84A81612F80E60E941D1E8A83E2
:1084F0001CC18F8186FF03C041ED5EE002C04AECE3
:108500005EE0612F8CE00E946E5D0DE723E84885F8
:10851000612F80E60E941D1E888707C18F812E2D46
:108520004EEB5EE0612F83FB882780F90E94722763
:108530009F8180FB93F90DC08F812E2D42EB5EE071
:10854000612F86FB882780F90E9472279F8180FB1C
:1085500096F99F83EAC08F8181702E2D4CEA5EE0F0
:10856000612F9B2D981B892F0E9472279B2D981B92
:108570008F8190FB80F98F83D8C00F8107FB002784
:1085800000F9002319F046EA5EE002C040EA5EE02E
:108590002E2D612F8CE00E94485DEE2059F08F81D6
:1085A00087FB882780F961E00E941C139F8180FB74
:1085B00097F99F838F8187FB882780F9081709F433
:1085C000B4C01C82B2C08F8187FF09C004E62CE9C9
:1085D0004C81612F80E60E941D1E8C83A6C02E2D2B
:1085E0004C81612F82E10E94DA27EE2009F49DC0C0
:1085F00046E160EF8C810E9419138C8387300CF464
:1086000094C090E6C91291C087508093F6078FE618
:1086100094E30E94AF1A89C068E97EE0812F0E942E
:10862000685D0E2D2E2D4B81612F8EE40E94C82790
:108630008B837BC06FE87EE0812F0E94685D0F8195
:108640000295037049F0402F50E02E2D2064612FD9
:1086500084E50E945F5F07C02E2D45E553E0612F42
:108660008EE40E94485DEE2009F45FC063E0802F35
:108670000E941C1383708295807F9F819F7C1CC009
:1086800067E87EE0812F0E94685D2F812695237028
:108690000E2D4DE65EE0612F8EE40E94345DEE20EB
:1086A00009F443C08F81869562E083700E941C1399
:1086B0008370880F9F81997F982B4BCF4D81429576
:1086C0004F7021E63EE06E2D812F0E94AD1C8295F9
:1086D000807F9D819F700BC04D814F7027E53EE0EC
:1086E0006E2D812F0E94AD1C8F709D81907F982BE5
:1086F0009D831BC04E8142954F702BE43EE06E2D52
:10870000812F0E94AD1C8295807F9E819F700BC03F
:108710004E814F7021E43EE06E2D812F0E94AD1CF2
:108720008F709E81907F982B9E83F394185F87E0D3
:10873000F812AACEDF91CF911F910F91FF90EF9089
:10874000DF90CF90BF9008956F927F928F929F920B
:10875000AF92BF92CF92DF92EF92FF920F931F934F
:10876000CF93DF93C82F8EEE90E10E94CD1E40E1A3
:10877000E42E0CE023E331E147E06C2F8DEE97E02F
:108780000E94D422E090ED07EA9466E08E2D0E94CC
:10879000F241C03611F0C43641F4E7FC06C0E09265
:1087A000F6078FE694E30E94AF1AA12CB12CCC24DB
:1087B000C39498E0D92EFF24E7FCF09425E0922E94
:1087C00039E0832EC0918107CA0D0C2F10E0D1E053
:1087D000E016F10609F0D0E077247394C83028F44D
:1087E000712C87E08C1528F45FC0E6E0EC1508F4E6
:1087F0005BC0B11002C0BD2E02C0BB24B3942D2FAC
:108800004BEE50E16D2D80E00E94485DA8014F5F66
:108810005F4FC93010F482E101C087E12D2F6D2D2B
:108820000E945F5F772051F008501109809EE0019F
:10883000819ED00D1124CD50DC4F07C0909EE001E9
:10884000919ED00D1124C553DC4F8E018AE2682E13
:10885000F80141918F01552747FD50956D2D862DCB
:108860000E946E5FF5E16F0E83E96812F1CF08E0B8
:108870000D0D711002C0C39411C025961AE24991E2
:10888000552747FD5095602F812F0E946E5F1B5E1C
:108890001E37A9F700E10D0DC394C394A394E7E03C
:1088A000AE1611F0D02E8ECFB11005C08091810789
:1088B0008F5F80938107DF91CF911F910F91FF9080
:1088C000EF90DF90CF90BF90AF909F908F907F9070
:1088D0006F900895BF92CF92DF92EF92FF920F9325
:1088E0001F93CF93DF93C82F8DE590E10E94CD1E9B
:1088F000FAE0EF2E0CE023E331E14AE06C2F8AEE40
:1089000097E00E94D4221091EA07115066E0812F6F
:108910000E94F241B82EC03899F480E80E9452615A
:1089200089E180937E07193019F40E94096205C01D
:10893000183018F4812F0E94766281E00E943F6C0B
:10894000E8E0FE2EC12EDD24C7FCD09488E0B812EA
:1089500005C080917E07882389F134C0CB2DD0E0FB
:10896000CC16DD0611F401E101C000E19E012F5F8C
:108970003F4F442737FD4095542F72E0E72E6F2D6F
:1089800082E10E944F5E80917E07811104C021E048
:10899000CC16DD0609F020E0FE01EE0FFF1FE655C4
:1089A000F34E459154916F2D88E10E94485D88E017
:1089B000F80EB39480E4F812C9CF4EC0DD24D394EE
:1089C000183009F0D12C6EE470E18F2D0E94685DA3
:1089D0005AE5C52EC6E0D0E0E0911B05F0E0E75A6D
:1089E000FC4F449150E00C2E02C0559547950A94D7
:1089F000E2F743705527475B5F4E0D2D21E06F2D49
:108A00008C2D0E94125D229786E0C80E82E7C81264
:108A1000E3CFDD2039F067E180911B050E9424132C
:108A200080931B0568E06F0D6933B0F480917E0779
:108A3000811103C021E0193009F020E045E350E145
:108A400086E0DF91CF911F910F91FF90EF90DF9023
:108A5000CF90BF900C94485DDF91CF911F910F9103
:108A6000FF90EF90DF90CF90BF9008952F923F92AC
:108A70004F925F926F927F928F929F92AF92BF922E
:108A8000CF92DF92EF92FF920F931F93CF93DF93DA
:108A900000D000D0CDB7DEB7282E8BEB9DE00E9432
:108AA000CD1E80912A07882321F00E94F828182FD4
:108AB00001C010E08091590781110BC0E090580768
:108AC0000CE023E331E145E0622D86EE97E00E9461
:108AD000D4226090E6078091C701803621F08F3B59
:108AE00031F08E32A1F490912A07992319F0109257
:108AF0002A070DC090915907911109C00E94526137
:108B00001092C701611007C010922A0702C06620A8
:108B1000D9F3198202C081E0898367E0862D0E9423
:108B2000F241382E8091590781111092C70180912E
:108B30002A07882369F011160CF456C1111156C189
:108B40008091C701823609F44FC1833609F44EC1C2
:108B50004424439411E0512CA32CB12C852D0E9468
:108B6000AE0F7C01311678F4612F70E06A197B0931
:108B70006830710544F4660F660F660F20E0442DDF
:108B800081E00E9461109FE1951508F4C8C0F701CB
:108B9000F081FA83F411C3C0C7010A969C838B83CA
:108BA000F52CCB80DC809AE0C91AD108311608F088
:108BB000A3C0812F90E08A199B09883091050CF0A1
:108BC0008CC0782E770C770C770C80912A07811156
:108BD00013C0611211C0F092F507EA81E093F30728
:108BE000F981FF2359F010922B0781E080935907F8
:108BF000EE24E394212C04C0E12C02C0EE24E39483
:108C00005F1459F0F60127812695237000E046EBAA
:108C10005DE0672D83E10E94345D20E1EB81FC8102
:108C200039974081672D80E30E9431100DE723E8DA
:108C30008B809C80F8E08F1A9108F4014081672DA9
:108C40008DE20E941D1EF4018083EB81FC81379729
:108C50004081442329F020E0672D88E40E9483109E
:108C6000EB81FC8136974081442379F0F6018781BE
:108C700020E087FF06C044E6672D80E60E945D5C29
:108C800004C0672D80E60E94DA27F60186818111F3
:108C900002C040E201C043E5F6018581882329F046
:108CA000433511F44AE201C044E4672D89E70E948C
:108CB0000F5D80912A078823F9F08091F4078F11C6
:108CC0001BC020E046E6672D88E10E94965DF09289
:108CD000F5071093E607612E0FC0089769F480919D
:108CE0002A07882349F08091F4078F1105C08091ED
:108CF000E6078F5F8093E6071F5FF394F0E2FF16AD
:108D000009F448C08B819C810A969C838B83FC016B
:108D10003A9780819A81891709F443CF3BC0611249
:108D200037C04092F3075092F507662D6A19660F17
:108D3000660F660F615029E049E180E00E94715F93
:108D4000E981EE2329F10E943C28811121C060E0D5
:108D50008091F5070E94DE1C10922A0782E192E4BE
:108D60000F900F900F900F90DF91CF911F910F9167
:108D7000FF90EF90DF90CF90BF90AF909F908F903B
:108D80007F906F905F904F903F902F900C94AF1A10
:108D90001F5FF52C4394F1E14F1611F05F2CDECEEE
:108DA00080915907882331F02092C7010E944A29F7
:108DB000109280071150109358070F900F900F904A
:108DC0000F90DF91CF911F910F91FF90EF90DF9067
:108DD000CF90BF90AF909F908F907F906F905F905B
:108DE0004F903F902F90089561E001C060E0809126
:108DF000F5070E94F827ACCE6F927F929F92BF92A8
:108E0000CF92DF92EF92FF920F931F93CF93DF9356
:108E1000D82E82E29AE00E94CD1E1EE1E12E06E0ED
:108E200027E231E140E06D2D83ED97E00E94D422EE
:108E30001091D307E0905A0767E0812F0E94F2411A
:108E4000F82E87E1F81208C01A3110F48FEF01C034
:108E500081E0D7E1FD2EF80E91E6D916B1F09D150F
:108E600058F084E4D81661F18D1520F092E4D916FB
:108E7000E0F541C085E406C094E6D91609F1D9169B
:108E8000A0F185E6D81659F036C080918007882376
:108E900091F11092800781E60E9452612CC011303E
:108EA00039F4EE2041F180918007882321F104C03C
:108EB000163109F5EE20F9F080915A0781500CC067
:108EC000113069F498E09E15B0F0809180078823F6
:108ED00091F080915A078F5F80935A070CC016312A
:108EE00051F486E08E1538F0F4CF8091800781111F
:108EF00002C010925A07F1107EC067E17AE088E064
:108F00000E94685D113031F480918007811102C0A8
:108F100001E101C000E12AE043E255E068E082E4BB
:108F20000E94125D8091800781110BC080917D07A6
:108F300087FF07C081E08093800710927D07109221
:108F40005A0780918007882381F020917D0733277D
:108F500027FD30958E2D90E08217930734F4109200
:108F6000800710927D0710925A07113009F071C4E2
:108F700080918007882309F46CC480915A079091EE
:108F80007D07891B87FD03C080935A0702C010929A
:108F90005A0780915A078A301CF089E080935A075B
:108FA00010927D07CE2DD0E0CE52DB4FFE01EF5A5E
:108FB000FF4F80810E94D42E20915C0130915D0191
:108FC000232B29F49D2D9F7D9254923018F461E457
:108FD0000E9424130E94E62ECF5ADF4F88839E2DD5
:108FE000990F9E0D990F21E0482F68E082E4890FC8
:108FF0000E945D5C2EC491E09F1548F1D8E0C091BD
:109000001505C695C695C695C77060E17AE08D2FA7
:109010000E94685D123089F466E08C2F0E94241350
:10902000C82F8770880F880F880F90911505977C3F
:10903000982B9093150501E001C000E02C2F44EE21
:1090400059E06D2F8CE50E94345DD85F04C082E04A
:10905000F8121DC0D8E0C091210569ED79E08D2F8F
:109060000E94685D133049F463E08C2F0E94241342
:10907000C82F8093210501E001C000E02C2F4FEAAA
:1090800059E06D2F82E40E94345DD85F04C093E004
:10909000F91231C0D8E0C0912E05C95F68EA79E0C5
:1090A0008D2F0E94685D143039F467E08C2F0E9488
:1090B0002413C82F21E401C020E44C2F50E06D2F71
:1090C00086E60E945F5F40912E05552747FD50952B
:1090D0002C2F332727FD309527503109421753078E
:1090E00029F0C750C0932E050E946713C8E0CD0F2A
:1090F000C93328F0B0C384E0F8121EC0C8E069E9A3
:1091000079E08C2F0E94685D153051F444E661E0EF
:1091100080911F050E94211380931F0521E401C047
:1091200020E440911F0550E06C2F86E60E945F5FAF
:10913000C85FC93328F08FC395E0F9121DC0C8E09D
:1091400068E879E08C2F0E94685D163049F465E08C
:10915000809120050E9424138093200521E401C002
:1091600020E44091200550E06C2F86E60E945F5F6E
:10917000C85FC93328F06FC386E0F81220C0C8E08A
:109180006FE779E08C2F0E94685D173061F44DE243
:109190006AE0809100050E942113809300050E94DF
:1091A0001F6021E401C020E44091000550E06C2FD5
:1091B00086E60E945F5FC85FC93328F04CC397E022
:1091C000F9121DC0C8E06FE679E08C2F0E94685D3F
:1091D000183051F448E768E2809101050E9421139C
:1091E0008093010521E401C020E4409101056C2F2A
:1091F00086E60E941610C85FC93328F02CC388E0A9
:10920000F81222C0C8E06CE579E08C2F0E94685DFE
:10921000193051F44EE666EF809117050E94211334
:109220008093170521E001C020E0409117055527E4
:1092300047FD5095465F5F4F6C2F80E70E945F5F50
:10924000C85FC93328F007C399E0F91217C0C8E016
:1092500021E01A3009F020E0809118054BE459E034
:109260006C2F81700E9452279091180580FB90F915
:1092700090931805C85FC93328F0EDC28AE0F81250
:1092800018C0C8E021E01B3009F020E080911805EB
:109290004FE359E06C2F869581700E945227909180
:1092A000180580FB91F990931805C85FC93328F021
:1092B000D2C29BE0F91219C0C8E021E01C3009F0CD
:1092C00020E08091180540E359E06C2F82FB88274D
:1092D00080F90E9452279091180580FB92F9909393
:1092E0001805C85FC93328F0B6C28CE0F81219C05F
:1092F000C8E021E01D3009F020E08091180542E22D
:1093000059E06C2F83FB882780F90E9452279091A7
:10931000180580FB93F990931805C85FC93328F0AE
:109320009AC29DE0F9121DC0C8E065E179E08C2F7A
:109330000E94685D1E3051F446E16AEE809103059B
:109340000E9421138093030521E001C020E0409199
:1093500003056C2F80E60E948310C85FC93350F06C
:109360007AC28EE0F81629F0D8E000E0C0E1BC2E09
:109370004CC0C8E021E01F3009F020E080911E05BC
:1093800044E059E06C2F86FB882780F90E94522721
:1093900090911E0580FB96F990931E05D8E0DC0F96
:1093A000D93318F358C2011133C064EF78E08D2F20
:1093B0000E94685D01112FC0C0911A051B112EC0BB
:1093C00068E78C2F0E942413C82F21E0CC2341F1A1
:1093D000206495E0C99FA00111246D2F86E60E94AC
:1093E0005F5F43E76D2F8091580C0E940F5D011164
:1093F0001EC0C0931A05D85FD93308F02CC281E093
:109400008B0D0F5F8231B1F0B82EFB14C0F7CBCFBC
:1094100064EE78E0CCCFC0912205D0CF20E0D6CF4B
:1094200045E553E06D2F86E60E94485DE0CFC0938E
:109430002205E1CF81E18F15E0F021E0123109F042
:1094400020E08091180582958170C1E046ED58E0DA
:109450006D2F9C2F981B892F0E945227C81B80912B
:109460001805C0FB84F980931805D85FD93308F03C
:10947000F2C182E08B0DF816D8F421E0181320E039
:1094800080911E0582958170C1E04AEC58E06D2FF5
:109490009C2F981B892F0E945227C81B80911E0564
:1094A000C0FB84F980931E05D85FD93308F0D3C17F
:1094B00083E08B0DF816D0F421E0181320E08091A2
:1094C00015058170C1E049EB58E06D2F9C2F981B6A
:1094D000892F0E945227C81B80911505C0FB80F977
:1094E00080931505D85FD93308F0B5C184E08B0DA2
:1094F000F816D8F421E0181320E080911505869520
:109500008170C1E042E852E16D2F9C2F981B892F9A
:109510000E945227C81B80911505C0FB81F98093DA
:109520001505D85FD93308F096C1B5E0CB2ECB0C2A
:10953000FC1408F079C06EEA78E08D2F0E94685D17
:10954000AEEF6A2EA1E17A2EC2E499249394809121
:109550002D05892101E009F400E021E0A3016D2F30
:109560008C2F0E94125D990CCA5F8FEF681A780ADF
:10957000C23769F71C1154C080915A0790917D073A
:10958000891B87FD03C080935A0702C010925A07B7
:1095900080915A078A301CF089E080935A07109214
:1095A0007D074E2D50E042505E4E8E2D880F8E0D61
:1095B000880F02E021E06D2F8E5B0E94125D90E625
:1095C000D91649F08EE6D81631F080915C01909161
:1095D0005D01892B29F18D2D0E9452611092800727
:1095E00021E030E002C0220F331FEA94E2F74091FD
:1095F0002D054227C90188739927892B19F44093B7
:109600002D0509C0842F822319F0276C242301C063
:10961000242B20932D0581E00E94A5570E944458D9
:10962000D85FD93308F017C186E08B0DF816E0F447
:1096300021E0181320E08091150582FB882780F92E
:10964000C1E04FE958E06D2F9C2F981B892F0E9495
:109650005227C81B80911505C0FB82F98093150520
:10966000D85FD93308F0F7C087E08B0DF816E0F427
:1096700021E0181320E08091150587FB882780F9E9
:10968000C1E041E958E06D2F9C2F981B892F0E9463
:109690005227C81B80911505C0FB87F980931505DB
:1096A000D85FD93308F0D7C088E08B0DF816E0F406
:1096B00021E0181320E08091180585FB882780F9A8
:1096C000C1E047E858E06D2F9C2F981B892F0E941E
:1096D0005227C81B80911805C0FB85F98093180597
:1096E000D85FD93308F0B7C089E08B0DF816B8F40D
:1096F00021E0181320E080911E0587FB882780F960
:109700004BE758E06D2F0E94522790911E0580FB79
:1097100097F990931E05D85FD93308F09CC08AE072
:109720008B0DF816E0F421E0181320E08091180565
:1097300086FB882780F9C1E043E758E06D2F9C2F16
:10974000981B892F0E945227C81B80911805C0FBC7
:1097500086F980931805D85FD93308F07CC08BE078
:109760008B0DF816B8F421E0181320E080911E0547
:1097700045E658E06D2F85FB882780F90E94522727
:1097800090911E0580FB95F990931E05D85FD93303
:1097900008F061C08CE08B0DF816A8F421E01813D6
:1097A00020E0809132054BE558E06D2F81700E94DA
:1097B00052279091320580FB90F990933205D85F43
:1097C000D93308F048C08DE0B80EFB1408F043C050
:1097D00046E558E06D2F86E00E946E5DD83328F094
:1097E00008E00D0F093378F036C004E2C0E02C2FFA
:1097F0004BE451E16D2F802F0E94185CCF5F085E13
:10980000C430A9F7EDCF1B110DC0809180078823CC
:1098100059F063E0809116050E9424138093160589
:1098200022E003C020E001C021E0409116054F5C1A
:10983000602F82E10E945D5CD4E2C0E0CF5F20E057
:109840004C2F602F8D2F0E943110D85EC430B1F79D
:1098500002C0D0E1D4CBDF91CF911F910F91FF9047
:10986000EF90DF90CF90BF909F907F906F90089582
:109870008F929F92AF92BF92CF92DF92EF92FF9220
:109880000F931F93CF93DF93C82F8CEB9FE00E9421
:10989000CD1E6CE0A62ECC24C3947AEBE72E7FE09D
:1098A000F72E0CE023E331E148E06C2F88EE97E0DF
:1098B0000E947B20C090E807CA94F0905A0766E0A7
:1098C0008C2D0E94F241A82E18E0DD24C7FCD09414
:1098D0002A2D30E0C216D30639F480918007882300
:1098E00029F052E0B52E04C0B12C02C0BB24B394C1
:1098F000E901CC0FDD1FC20FD31FC55CDB4F67EB47
:109900007FE0812F0E94685D88E08A1510F448E3AB
:1099100001C041E34A0D612F8CE00E940F5DFF20E2
:1099200011F000E001C00B2D2A812F704CE45FE0A4
:10993000612F83E10E94345D8A818F700E94A00FA5
:10994000982E81E091102EC0F81611F020E001C091
:109950002B2D4881612F8DE30E9431108881853243
:10996000B4F09BED892E880E6981882D0E943B1DE5
:109970009C0182E0F81611F000E001C00B2D82E09E
:10998000E82E482D612F8AE60E94B21D62C082E057
:10999000F81611F020E001C02B2D4981552747FD15
:1099A000509553C0981216C0F81611F020E001C06F
:1099B0002B2D4881612F8DE30E94831082E0F816E1
:1099C00011F020E001C02B2D4981612F84E50E9418
:1099D00083103FC082E0981217C081E0F81611F0A2
:1099E00020E001C02B2D4881612F8DE30E943110B2
:1099F00082E0F81611F020E001C02B2D4981612F83
:109A000087E50E94311025C068E47FE0812F0E9425
:109A1000685D81E0F81611F020E001C02B2D48812F
:109A2000552747FD50954F5F5F4F612F8FE40E9490
:109A30005F5F82E0F81611F020E001C02B2D498114
:109A4000552747FD50954F5F5F4F612F8CE60E9471
:109A50005F5F4A8142954F7049300CF04F5F83E061
:109A6000F81203C02B2D286001C028E0612F89E681
:109A70000E94831080918007811107C080915C0152
:109A800090915D01892B09F465C0BB2009F462C087
:109A900081E0F81639F1F816A0F082E0F81609F422
:109AA0003EC083E0F81256C08A816FE082958F70C5
:109AB0000E941C138295807F9A819F70982B9A83B5
:109AC00049C08A816EE08F700E941C138F709A814A
:109AD000907F982B9A830E94A00F9816D9F1188234
:109AE000198238C081E0981661F0981640F082E043
:109AF000981651F083E098122DC063E60BC06EE219
:109B000009C046E16AEE02C04EE260E088810E9430
:109B1000191303C088810E941C1388831BC081E035
:109B2000981669F0981640F082E0981671F083E07C
:109B3000981210C063E60AC04DE763E802C046E130
:109B40006AEE89810E94191304C06EE289810E9425
:109B50001C138983A394185F103409F0B9CEDF91E8
:109B6000CF911F910F91FF90EF90DF90CF90BF901A
:109B7000AF909F908F900895AF92BF92CF92DF9257
:109B8000EF92FF920F931F93CF93DF93B82E80E352
:109B90009DE00E94CD1EB3E1AB2ECDE0CC2ED2E2F3
:109BA000ED2EDDE0FD2E0CE023E331E141E06B2DF5
:109BB0008EED97E00E947B201091DE07D0905A072F
:109BC00067E0812F0E94F241C82F2091FF0430E00E
:109BD0002F5F3F4F442737FD4095542F02E0E02E82
:109BE00001E160E08AE20E944F5EC1113BC06DE17D
:109BF0007DE088E00E94685D00E12AE045EE51E0EA
:109C000068E082E40E94125D113009F0AEC329E0E1
:109C100040E467E08AE30E94715F8D2D880F8D0D0F
:109C2000880F2091800746E068E0845C0E94965D82
:109C300080918007882309F498C3CD2DD0E0CB51C3
:109C4000DE4F88810E94D42E61E40E941C130E9482
:109C5000E62E9881981709F488C3888382E00E94D1
:109C6000A55783C3C23020F5C8E06CE07DE08C2F9F
:109C70000E94685D123081F420E6B21204C0809127
:109C8000EF010E945F1361E38091EF010E941C13BA
:109C90008093EF0121E001C020E04091EF0150E00E
:109CA0004C5F5E4F6C2F88E50E945F5FC85F03C00A
:109CB000C23091F4C8E068EF71E18C2F0E94685DBA
:109CC000133009F0B1C381E0D81251C380918007ED
:109CD0008111ACC301E0ABC3C330D1F4C8E064E090
:109CE0007DE08C2F0E94685D143051F449E367ECED
:109CF0008091F0010E9419138093F00141E001C0AE
:109D000040E021E06C2F8CE30E94B810C85F03C0D4
:109D1000C430E1F4C8E06BEF7CE08C2F0E94685DFA
:109D2000153051F445E16BEE809160040E941913E7
:109D30008093600441E001C040E022E06C2F8CE39E
:109D40000E94B810C85FC93320F073C3C53021F535
:109D5000C8E068EF71E18C2F0E94685D163071F4E5
:109D60008091F10161E081700E941C139091F101DA
:109D700080FB90F99093F10101E001C000E0209197
:109D8000F101217045EE5CE06C2F8CE30E94345DA4
:109D9000C85FC93320F04DC3C630B9F4C8E021E034
:109DA000173009F020E08091F6014EED5CE06C2F59
:109DB00081700E9472279091F60180FB90F9909338
:109DC000F601C85FC93320F034C3C730C1F4C8E01E
:109DD00021E0183009F020E08091F60147ED5CE0C9
:109DE0006C2F829581700E9472279091F60180FB02
:109DF00094F99093F601C85FC93318F01AC3C830BC
:109E0000E9F46EEC7CE08C2F0E94685D193049F417
:109E100064E08091F7010E941C138093F70101E038
:109E200001C000E02091F7014EEA5CE06C2F8CE36A
:109E30000E94345DC85FC93320F0FBC2C930D1F441
:109E4000C8E066EA7CE08C2F0E94685D21E01A3051
:109E500009F020E0022F4091F9016C2F86E30E9467
:109E6000C8278093F901A8E0EA2EEC0E88E38E154E
:109E700030F4DFC2CA3009F050C0F8E0EF2E6DE9CF
:109E80007CE08E2D0E94685DECE3CE2EC0E0D0E039
:109E9000DC1202C01B3061F02091FA0130E00C2E80
:109EA00002C0359527950A94E2F7022F017001C090
:109EB00002E0AE014B56534F21E06E2D8C2D0E94D7
:109EC000125D219626E0C20E86E6C812E1CF1B3055
:109ED000F9F420E6B21631F020915C0130915D0179
:109EE000232BB1F08B2D0E9452611092800721E04C
:109EF00030E00D2C01C0220F0A94EAF78091FA019C
:109F000082278093FA0182E00E94A5570E9444585C
:109F1000C8E0CE0DC93328F08CC2CB3009F0DAC0CE
:109F2000C8E06FE87CE08C2F0E94685D1C3041F433
:109F3000D11006C080918007882321F002E003C081
:109F400000E001C001E04091F40186E0489FA001DB
:109F500011244059534F26E06C2F84E20E94125D79
:109F60008091F401882359F09DEF980F9230F0F51D
:109F700066E67CE08C2F0E94685DD8E406C06AE645
:109F80007CE08C2F0E94685DDCE31C3049F421E00A
:109F9000D21206C080918007882321F002E003C01E
:109FA00000E001C001E02091F5012E5F48E45CE093
:109FB0006C2F8D2F0E94345D1C3049F482E0D81242
:109FC00006C080918007882321F022E003C020E0B2
:109FD00001C021E04091F80182E34802A001112470
:109FE000445D5E4F6C2F88E28D0F1EC08130F1F40E
:109FF00061E47CE08C2F0E94685D1C3049F421E014
:10A00000D21206C080918007882321F022E003C08D
:10A0100020E001C021E04091F501552747FD509512
:10A020004F5F5F4F6C2F8EE70E945F5F1C3009F01F
:10A030004DC080918007811107C020915C01309153
:10A040005D01232B09F442C0D091F40180911E05DB
:10A0500085FF02C064E001C063E081E0D81661F0D2
:10A06000D81620F022E0D216F1F02BC08D2F0E94DE
:10A070001C138093F40125C0DD2321F08DEF8D0F9B
:10A08000823038F444E06EEF8091F5010E9419139C
:10A0900007C0D130B1F46CE78091F5010E941C1328
:10A0A0008093F5010EC0DD2321F08DEF8D0F8230FE
:10A0B00040F44AE06CEF8091F8010E9419138093FC
:10A0C000F8018091F4018D131092F501C85FC93336
:10A0D00028F0AFC1CC3009F077C0C8E08091F4011E
:10A0E000882321F09DEF980F923010F562E37CE019
:10A0F0008C2F0E94685D1D3011F421E201C020E226
:10A100004091FE0185E04802A00111244F515F4FAC
:10A110006C2F8CE40E945F5F1D3009F051C044E158
:10A120006CEE8091FE010E9419138093FE0148C0DD
:10A130008130B9F4D1E01D3009F0D0E02D2F4CE191
:10A140005CE06C2F80E00E94485DDD23C9F120E8CF
:10A15000B21236C081E08093930C80E00E943F6C85
:10A160002FC063E17CE08C2F0E94685D4091F50177
:10A1700047FD04C043301CF042E001C040E0409382
:10A18000F5011D3031F480918007882321F002E031
:10A1900003C000E001C001E089E04802A0011124F1
:10A1A0004950544F29E06C2F8CE30E94125D1D3002
:10A1B00039F462E08091F5010E941C138093F5014F
:10A1C000C85FC93320F035C1CD3051F5C8E06AEE23
:10A1D0007BE08C2F0E94685D1E3099F48091F6011F
:10A1E00067E08295869587700E941C138295880F80
:10A1F000807E9091F6019F71982B9093F60121E05B
:10A2000001C020E04091F6014295469547704F5CB1
:10A210006C2F82E70E945D5CC85FC93320F009C1E2
:10A22000CE3021F5C8E060EE7BE08C2F0E94685DA7
:10A230001F3071F48091FB0161E081700E941C135A
:10A240009091FB0180FB90F99093FB0101E001C02C
:10A2500000E02091FB01217048ED5BE06C2F8CE366
:10A260000E94345DC85FC93320F0E3C0CF30C1F431
:10A27000C8E021E0103109F020E08091FB014EECB4
:10A280005BE06C2F869581700E9472279091FB0194
:10A2900080FB91F99093FB01C85FC93320F0C9C0DE
:10A2A000C031C1F4C8E021E0113109F020E0809113
:10A2B000F10146EC5BE06C2F869581700E9472275D
:10A2C0009091F10180FB91F99093F101C85FC9333E
:10A2D00020F0AFC0C131D1F4C8E021E0123109F063
:10A2E00020E08091F1014DEB5BE06C2F82FB882731
:10A2F00080F90E9472279091F10180FB92F990936E
:10A30000F10168E06C0F693328F093C0C23109F0A5
:10A3100090C068E080917E07811103C021E0133175
:10A3200009F020E049EA5BE080E00E94485D1331DB
:10A3300009F07FC020E8B2127CC01092800789E14A
:10A3400080937E0780E80E9452611092290783E77C
:10A3500098E2DF91CF911F910F91FF90EF90DF90E6
:10A36000CF90BF90AF900C94AF1AC0E17ECCD110CB
:10A370005BC08091800700E0882311F022E001C0DB
:10A3800021E04091F2015091F3016C2F87E40E948B
:10A39000BC0F133009F046C080918007811106C0C0
:10A3A00020915C0130915D01232BE1F16CE370E0C1
:10A3B0008091F2019091F3010E94806F962FD82F27
:10A3C000DD2021F021E0D21691F02CC06BE3892F23
:10A3D0000E941C132CE38202C00111248D0F911DD9
:10A3E000D7FD9A959093F3018093F2011BC04EE341
:10A3F00061E082E08D0F0E941913D81BDE5F20916F
:10A40000F2013091F3012D1B3109D7FD339537FD52
:10A4100005C03093F3012093F20104C01092F301C0
:10A420001092F201C85F5BCC00E001C002E020E0C6
:10A43000A8CFDF91CF911F910F91FF90EF90DF9008
:10A44000CF90BF90AF900895AF92CF92EF92FF92CE
:10A450000F93CF93DF93C82F8FE69BE00E94CD1E12
:10A4600086E0A82EC12C9EE6E92E9BE0F92E0CE09A
:10A4700023E331E142E06C2F8BED97E00E947B20DB
:10A48000C091DB0767E08C2F0E94F241D091FB0165
:10A49000D295D695D77063E67BE088E00E94685D30
:10A4A000C13089F464E08D2F0E941C13D82F982F9F
:10A4B0009295990F907E8091FB018F71892B8093EB
:10A4C000FB0101E001C000E02D2F43E45BE068E008
:10A4D00084E50E94345D68E37BE080E10E94685D72
:10A4E000C23049F464E28091FC010E941C13809305
:10A4F000FC0121E001C020E04091FC0160E184E525
:10A500000E9431106DE27BE088E10E94685DC330FB
:10A5100049F464E68091FD010E941C138093FD01C3
:10A5200021E401C020E44091FD0150E068E184E5B0
:10A530000E945F5F21E0C43009F020E08091FB01C0
:10A540004FE15BE060E282FB882780F90E9492275E
:10A550009091FB0180FB92F99093FB0121E0C530C3
:10A5600009F020E08091FB0141E15BE068E283FBC0
:10A57000882780F90E9492279091FB0180FB93F934
:10A580009093FB0121E0C63009F020E08091FB01AF
:10A5900043E05BE060E3829581700E949227909196
:10A5A000FB0180FB94F99093FB01DF91CF910F9118
:10A5B000FF90EF90CF90AF9008955F926F927F924F
:10A5C0008F929F92AF92BF92CF92DF92EF92FF92C3
:10A5D0000F931F93CF93DF93D82E84EE90E10E94C8
:10A5E000CD1EB1E1AB2ECC24C394C2EEEC2EC0E163
:10A5F000FC2E0CE023E331E146E06D2D8CEE97E07C
:10A600000E947B20C090EC07CA94B0905A0766E085
:10A610008C2D0E94F241982E80E8D81227C09FE02E
:10A620009C1520F14C2D552747FD5095FA01E9194D
:10A63000F109EE0FFF1FE55AF84F20813181B1106B
:10A6400015C085E0849FF001859FF00D1124E15C29
:10A65000FC4F8281882319F031952195310934838B
:10A66000238382E00E94A5570E944458E8E0AE2E62
:10A67000EC2CFF24E7FCF09480E1981609F4BEC0AE
:10A68000892D0E94B50FEC01092D10E0F801EE0FA5
:10A69000FF1FE55AF84F208131818A81EB81FC81CF
:10A6A000882319F0F195E195F1092E1B3F0B233317
:10A6B00031051CF081110AC09EC02E3C3F4F1CF496
:10A6C000882321F098C06DE2862E02C05FE7852EB8
:10A6D000939420E0492D6A2D80E00E946110482D5E
:10A6E0006A2D8BE40E940F5D8091FB0181FF03C006
:10A6F0004DE7642E02C034E6632E812C562C519413
:10A70000E016F10641F4B81006C08091800781116F
:10A7100005C021E004C020E0712C09C022E0809136
:10A720007F078823C9F3772473941092710182E024
:10A73000881691F193E0891609F443C081E08816E8
:10A74000B1F020624B815C816A2D80E30E945F5FE3
:10A75000772009F446C022E048EE53E068E17CEF40
:10A760008B819C810E945A129C838B833AC04881C2
:10A770004456552747FD50956A2D88E40E945F5F37
:10A78000772079F188818456888349E1652D0E947C
:10A7900019138C59888325C049814C59552747FD89
:10A7A00050956A2D86E60E945F5F7720D1F08981FF
:10A7B0008C598983462D67EE0E941913845689832C
:10A7C00010C04A816A2D8CE60E946F20772049F0E4
:10A7D00061E08A810E941C1391E0811101C090E028
:10A7E0009A83839494E089128BCF88E08A0D803419
:10A7F00091F1A82E41CF2EE7822E6ACFC1E090E1E1
:10A80000C912C0E080917E07811123C02C2F41ED39
:10A8100050E16A2D82E10E94485DCC23E1F080E89E
:10A82000D81219C089E180937E0780E80E945261A6
:10A83000DF91CF911F910F91FF90EF90DF90CF901C
:10A84000BF90AF909F908F907F906F905F900C948F
:10A85000FA3E20E0DCCFDF91CF911F910F91FF9066
:10A86000EF90DF90CF90BF90AF909F908F907F90B0
:10A870006F905F9008956F927F928F929F92AF92A8
:10A88000BF92CF92DF92EF92FF920F931F93CF93DD
:10A89000DF93C82F85E290E10E94CD1E41E1A42EF6
:10A8A00052E0C52E62E2E62E60E1F62E0CE023E3D4
:10A8B00031E149E06C2F89EE97E00E947B20A09067
:10A8C000E907AA9490905A0766E08A2D0E94F24107
:10A8D000B82E18E0CA2CDD24C7FCD094B11020C0DB
:10A8E00062E170E1812F0E94685DA1100FC080912C
:10A8F0008007882311F0C2E001C0C1E060E18091CF
:10A9000061040E941C138093610401C0C0E0409167
:10A91000610450E02C2F612F8CE60E945F5F59C1CB
:10A9200080E18B1508F455C100E180916104081B9A
:10A93000EB2CF12CE701CC0FDD1FC05ADB4F20E0E0
:10A940004B2D612F80E00E9461100B1508F4C3C0ED
:10A95000812CCE14DF0441F4981006C0809180074A
:10A96000811105C001E004C000E0712C07C002E0C5
:10A9700080917F078823C9F377247394888181109D
:10A9800021C0807C803421F0803821F446E503C06A
:10A9900041E401C043E5202F612F8EE10E945D5C00
:10A9A000772009F493C0888162E082958695869528
:10A9B00083700E941C138295880F880F807C988179
:10A9C0009F7330C091E0891230C0982F907C9038EE
:10A9D00019F026E1622E02C099E1692E482F440F3A
:10A9E000440F4595459547314CF029EE240F4BEF28
:10A9F0005FE0612F8AE20E94345D05C0202F612F45
:10AA00008AE20E948310772009F460C08881880F51
:10AA1000880F462D6AEE859585950E9419138F73D0
:10AA20009881907C982B988351C0982F907C498175
:10AA3000903491F447FD03C04F3024F401C040E04E
:10AA4000242F01C02FE0298346E951E1612F80E6E0
:10AA50000E94345D4FE017C0903841F5880F880F91
:10AA600089359CF047FD04C049301CF049E001C025
:10AA700040E0498321E0240F44E552E1612F80E664
:10AA80000E94345D49E060E01BC04F360CF04FE699
:10AA90004983552747FD509540585F4F202F612F20
:10AAA00080E60E945F5F4FE660E80AC0552747FDD9
:10AAB0005095202F612F80E60E945F5F4DE763E88D
:10AAC000772021F089810E9419138983839483E080
:10AAD00088123FCF7EC068EF7FE0812F0E94685DC3
:10AAE000812CCE14DF0441F4981006C080918007B9
:10AAF000811105C001E004C000E0712C07C002E034
:10AB000080917F078823C9F377247394888181100B
:10AB100013C0482F4F71202F612F8EE10E948310A8
:10AB2000772009F452C0888165E18F710E941C135F
:10AB30008F719881907E1BC091E089121BC0282FD5
:10AB40002295269527704CEC5FE0612F8CE30E94E4
:10AB5000345D7720D1F1888166E082958695877093
:10AB60000E941C138295880F807E98819F71982B7C
:10AB700098832BC082958695877090E049810697CF
:10AB800074F0493008F049E0498321E0240F44E59E
:10AB900052E1612F80E60E94345D49E00BC04A3FDC
:10ABA00008F04AEF498350E0202F612F86E60E948B
:10ABB0005F5F4AEF772049F050E0898122E060E052
:10ABC00070E090E00E945A128983839483E0881297
:10ABD00088CFB394185F103409F080CEDF91CF9105
:10ABE0001F910F91FF90EF90DF90CF90BF90AF90AB
:10ABF0009F908F907F906F9008951F93CF93DF93D6
:10AC0000EC011AE088810E94D42E0E94E62E8993DE
:10AC10001150C1F7DF91CF911F910895E3EDF4E05A
:10AC200080E090E021913191820F931F24E0EB3E70
:10AC3000F207C1F7089581E6E2EDF4E0DF011D922D
:10AC40008A95E9F78AE08093D20489E18093000530
:10AC50008AE58093010581E080931605E3EDF4E039
:10AC600020E032E080E891E021933193958784875A
:10AC7000938F828FB4E0E13EFB07B1F74AE050E0EA
:10AC80006DEC72E183E295E00E94DB6F0E940E564C
:10AC90009093FE048093FD040895CF93C82F2DEE6A
:10ACA00032E0E5EEF1E0DF01C9011D920197E9F71D
:10ACB0004AE050E062EC72E1CF010E94DB6F8C2F22
:10ACC00090E06AE070E001960E94806F605D6093A2
:10ACD000EA01805D8093EB0180E0CF910C94766275
:10ACE0000F931F93CF93DF93EB01042F803138F53F
:10ACF00061E0680F8BE098E00E94BE5910E0A80167
:10AD000060E270E0CE010E94FC6F4AE050E0BE01BC
:10AD10008BE098E00E94425A0A9789F48BE098E011
:10AD20000E94B059C00FD11F009749F06AE070E04F
:10AD30000E94806F805D8A93862F972FF5CFDF91D9
:10AD4000CF911F910F9108958F5F0C946559CF9308
:10AD5000C82F803188F561E0680F8BE098E00E9491
:10AD6000BE592DEE32E0E5EEF1E0DF01C9011D92A2
:10AD70000197E9F74DEE52E0BF018BE098E00E94A9
:10AD8000425A8F3F910509F018F48C2F0E944D56BE
:10AD900085EE91E00E94FD5580918D04811107C0E0
:10ADA0008091F601869583708E5F80938D040E945A
:10ADB000D633CF910C944213CF910895FF920F9305
:10ADC0001F93CF93DF93CDB7DEB72F970FB6F894CD
:10ADD000DEBF0FBECDBF01E0080F102F1031C8F449
:10ADE000FF24F394F10E8F2D0E94655981110FC03D
:10ADF000602F8BE098E00E94BE5961E0610F28E56A
:10AE000032E042E082E098E00E942A5B06C01F2DFB
:10AE1000E5CF103169F780E01AC04FE050E0BE0185
:10AE20006F5F7F4F8BE098E00E94DB59882351F0E1
:10AE3000482FBE016F5F7F4F82E098E00E94A75AC3
:10AE4000A895EBCF82E098E00E94555B81E02F96B9
:10AE50000FB6F894DEBF0FBECDBFDF91CF911F912B
:10AE60000F91FF900895EF920F931F93CF93DF936D
:10AE70000E945259882381F10E94C85887FD2CC036
:10AE800060E08BE098E00E94BE5981E6E2EDF4E0DC
:10AE9000DF011D928A95E9F741E650E0BF018BE0A2
:10AEA00098E00E94425A83E295E00E94FD5580910D
:10AEB000D2048A3028F480918E01816080938E01C3
:10AEC0008AE08093D204C091FD04D091FE040E94D8
:10AED0000E56C817D90781F161E082EB92E10E941A
:10AEE0004A1A80EA92E10E94C9110E942D590E94DB
:10AEF0001B5688ECE82E01E610E022ED34E041E03C
:10AF000060E08BE098E00E94865B8136910529F035
:10AF100060E081E992E10E944A1A80E00E944D5669
:10AF200098ECE92E0DEE12E025EE31E042E061E012
:10AF30008BE098E00E94865B8091FF04DF91CF91C7
:10AF40001F910F91EF900C94A756882379F0909160
:10AF50001608982B90931608F89480915A0C9091AB
:10AF60005B0C789490931508809314080895EF92E1
:10AF70000F931F93CF9340911608442309F47FC089
:10AF8000811110C0F89480915A0C90915B0C7894C8
:10AF90002091140830911508821B930B843691057B
:10AFA00008F46DC08091F807811169C0C42FC47086
:10AFB00042FD02C081E001C083E08093F807109257
:10AFC000160840FF26C034E1E32E01E610E022ED32
:10AFD00034E041E061E189EF97E00E94865B8136D1
:10AFE000910519F461E180E029C08091FF0782306A
:10AFF00051F48091160881602BC08091FF07823048
:10B0000001F1C1113AC060E088ED92E10E944A1A54
:10B0100034C041FF32C024E1E22E0DEE12E025EEF5
:10B0200031E042E061E189EF97E00E94865B8D3E6E
:10B03000924019F78091FF0461E18F5F0E9473597C
:10B040001CC080911608C11102C0826001C08660D8
:10B0500080931608F89480915A0C90915B0C789428
:10B060008456910990931508809314088091950C4B
:10B07000833019F4A8951092950C1092F807CF918F
:10B080001F910F91EF90089580911608882359F031
:10B0900081E00E94B7578091950C8330A9F7A8955D
:10B0A0001092950CF1CF089540E450E060E070E01C
:10B0B00087E198E00C945D6041E050E062E070E070
:10B0C00089E198E00C945D60CF93DF931F92CDB738
:10B0D000DEB7698390E1899FB001112441E050E01F
:10B0E000CE0101960E945D600F90DF91CF9108958F
:10B0F000CF93DF931F92CDB7DEB790E1899FB00168
:10B10000112441E050E0CE0101960E940370898134
:10B110000F90DF91CF910895CF93DF93D82FC82F51
:10B120008C2F0E947858882329F08C2F0E94785801
:10B13000C82FF6CF609119088C2F0E946458D093C5
:10B140001908DF91CF910C945C58CF93C0911908E6
:10B15000CC2359F08C2F0E947858809319080E94B4
:10B160005C5860E08C2F0E9464588C2FCF9108951A
:10B17000CF93DF9380911908C0E0D0E0882321F0BD
:10B180002F960E947858FACFCE01DF91CF91089583
:10B19000DF92EF92FF920F931F93CF93DF9380E89C
:10B1A000E5EEF1E0DF011D928A95E9F7CBE1D8E009
:10B1B000F12CB4E1FB1205C08091190809E118E0F7
:10B1C00002C08E01888190E0E12CDD24D394DF0C55
:10B1D000009701F19C01245031092C37310530F4DE
:10B1E000FC01EB51FE4F2081222371F0EE2029F06B
:10B1F00060E08E2D0E94645804C0F80110820E9405
:10B20000545880E090E0E4CFD082E82E0E94785835
:10B2100090E0DECFF3942396F5E1FF12CACFC4E0AD
:10B22000D0E0FE01EB51FE4F8081811109C0609199
:10B2300019088C2F0E946458C09319080E945C580A
:10B240002196C038D10569F780E0DF91CF911F9139
:10B250000F91FF90EF90DF900895CF9380E4E7E1A6
:10B26000F8E0DF01982F1D929A95E9F794E090930A
:10B2700017088093180880E180931A0884E0C1E0E1
:10B28000C80F6C2F0E946458CF3711F08C2FF7CF66
:10B2900060E08FE70E94645884E080931908CF91A2
:10B2A0000C94545840E450E060E070E087E198E08E
:10B2B0000E94037080911708843029F481E09091F6
:10B2C0001808903409F080E0089590E0FC01EE0F3A
:10B2D000FF1FE80FF91FE95EF74F81E0948191119C
:10B2E00001C080E00895CF93DF9390E0EC01CC0F94
:10B2F000DD1FC80FD91FC95ED74F8C819D81AE81DC
:10B3000070E0FB01EE0FFF1FE60FF71FE95EF74F3E
:10B310002481358146812C833D834E8384839583AC
:10B32000A683DF91CF910C945458CF9390E09C0169
:10B33000220F331F280F391FF901E95EF74FC4812F
:10B34000F901E55EF74F1082118212820E94545873
:10B35000CC2321F08C2FCF910C948C58CF91089551
:10B36000FC01808190E0FC01EE0FFF1FE80FF91F48
:10B37000E45EF74F918180819F700895CF93DF93B2
:10B38000FC0160831282118270E0CB01880F991F4B
:10B39000860F971FEC01C95ED74F2C81238314823F
:10B3A00015821682FC01E35EF74F808182958F70D3
:10B3B000DF91CF910895AF92BF92CF92DF92EF923B
:10B3C000FF920F931F93CF93DF931F92CDB7DEB7FA
:10B3D0008C01FC01808190E0FC01EE0FFF1FE80F63
:10B3E000F91FE45EF74F80812181922F9F70F80151
:10B3F00021813281821B930B7A018417950708F40F
:10B400007C015B016701C114D10429F1F80183813A
:10B41000882309F164816F5F648370E0F0E18F9F9E
:10B42000600D711D112441E050E0CE0101960E9493
:10B4300003708981F50181935F01F80184818F3068
:10B4400030F0148283810E947858F8018383F1E000
:10B45000CF1AD108D8CFF801818192818E0D9F1D1E
:10B460008C199D09928381838E2D8C190F90DF9109
:10B47000CF911F910F91FF90EF90DF90CF90BF90F1
:10B48000AF9008957F928F929F92AF92BF92CF928A
:10B49000DF92EF92FF920F931F93CF93DF934C01B4
:10B4A0006B018A01C0E0D0E05C0125E0A20EB11C76
:10B4B000C017D107E8F5F40185818F7781F0F40199
:10B4C0004581F42FFF777F2E2F2F30E0C8018C1B92
:10B4D0009D0B8217930760F4702E7C1A09C041E01F
:10B4E00050E0B501C4010E94DB59813041F320C016
:10B4F000E72CF12CC6018C0F9D1F47FF06C0A7014A
:10B5000060E070E00E94FC6F0CC0A701BC01C401A8
:10B510000E94DB59871529F0FE01E80FF11DCF01CC
:10B5200008C0CE0DDF1DF401858187198583C0CF4A
:10B53000CE01DF91CF911F910F91FF90EF90DF909F
:10B54000CF90BF90AF909F908F907F900895AF92D3
:10B55000BF92CF92DF92EF92FF920F931F93CF9300
:10B56000DF93EC018B01D42E8B81811111C0898175
:10B570009A81892B69F4E880F12C0E94A5588B836D
:10B58000F701EE0FFF1FEE0DFF1DE95EF74F8483FD
:10B59000CD2C8FE0A82ECC2009F445C02F81388512
:10B5A000F89480915A0C90915B0C7894281B390B7D
:10B5B00037FF02C082E004C08B81811103C081E0AB
:10B5C0008E8331C09C819F3078F01C820E94785815
:10B5D000811106C00E94A558682F8B810E94645873
:10B5E0008B810E9478588B838B81882341F36C81F7
:10B5F0009A2D961BBC2C9C1508F4B92EEB2CF12C23
:10B6000070E090E1899F600D711D11246F5F7F4F85
:10B61000A701C8010E945D600E0D1F1D8C818B0D5E
:10B620008C83CB18B8CF6D2D70E06C19710929810E
:10B630003A81260F371F3A8329838D2D8C19DF918C
:10B64000CF911F910F91FF90EF90DF90CF90BF901F
:10B65000AF900895EF92FF920F931F93CF93DF93D4
:10B66000EC01F62EE42E89010E94BE596F2D70E088
:10B67000FB01EE0FFF1FE60FF71FE45EF74F10828E
:10B68000E29430EFE322E182F89440915A0C509119
:10B690005B0C7894400F511F58874F83DF91CF91F7
:10B6A0001F910F91FF90EF9008951F93CF93DF9319
:10B6B000EC01888190E0FC01EE0FFF1FE80FF91FFD
:10B6C000E45EF74F898180839A819F708181807FBA
:10B6D000892B81838B81882329F00E947858182F29
:10B6E00081110BC010E00E945458112359F0812F92
:10B6F000DF91CF911F910C948C5860E08B810E9458
:10B700006458F1CFDF91CF911F9108957F928F926E
:10B710009F92AF92BF92CF92DF92EF92FF920F93E0
:10B720001F93CF93DF931F92CDB7DEB76C01590102
:10B730002E2D30E00E942A5B19824501E12CF12C6C
:10B7400077247394F40181914F019981811108C08C
:10B7500071104EC08081811105C0772473941CC084
:10B7600071100AC080E09F3718F4E016F10679F5F1
:10B77000772089F0782E01C0712C992341F19068CF
:10B78000998341E0BE016F5F7F4FC6010E94A75AB7
:10B790008130E1F027C0782E9923C9F041E0BE0145
:10B7A0006F5F7F4FC6010E94A75A8130D9F449814B
:10B7B000B701641B71096A0D7B1DC6010E94A75A5F
:10B7C0009981891719F0981B99830CC01982898176
:10B7D0008F5F8983FFEFEF1AFF0A0E151F0508F030
:10B7E000B1CF08C089818F778701081B110902C07A
:10B7F000872DB9CFC6010E94555BC8010F90DF911C
:10B80000CF911F910F91FF90EF90DF90CF90BF905D
:10B81000AF909F908F907F90089580E094E0E8E54E
:10B82000F8E0DF019C011D9221503040E1F70895BE
:10B83000FF920F931F93CF93DF93FA017491319688
:10B84000A491B0E0179693E0B595A7959A95E1F786
:10B850001A2FDA011396FA0132964491249FA00D13
:10B86000B11D112466956695669590E0F0E86F9F8E
:10B87000800D911D112420E030E060E0885A974F40
:10B88000472F50E0611798F40A2FEC01C20FD31F25
:10B89000FD01FE2EF01AF71620F4F490F99231967D
:10B8A000F8CFA40FB51F6F5F20583F4FEBCFDF914C
:10B8B000CF911F910F91FF900895FF920F931F93C7
:10B8C000CF93DF9346312CF4842F880F840F880F99
:10B8D000A0C076E0780FA42FBB27A7FDB09520FD70
:10B8E00008C021FD02C090E005C09091590C96FF60
:10B8F000FACF91E0669566956695C82FD0E030E85E
:10B90000639FC00DD11D1124C85AD74FFE0122FFDD
:10B9100053C04E3211F07CE0780F8AE04802F0010B
:10B920001124E054F1409D012052310937FF03C03A
:10B930009D0121513109A90124E0559547952A958A
:10B94000E1F780EA849F9001859F300D11242E0F2E
:10B950003F1F25513D4E85E0882381F0F901049178
:10B96000E056FF4F6491A9014F5F5F4FFA011491B8
:10B97000F901EF55FF4FF4909A0104C010E060E028
:10B9800000E0F12C2F5F3F4F992321F00095109597
:10B990006095F094DE01AF57BF4FFCE0A835BF07BC
:10B9A00040F408831983FE01E058FF4F6083FC9246
:10B9B0002296815088F62CC023FF08C02196292F9B
:10B9C0002195208375E0780F51E001C050E025E01B
:10B9D0004202F0011124E253F64E85E044915523D2
:10B9E00011F0843059F03CE0C835D30738F49E019B
:10B9F0002F5F3F4F911140954883E9018150319667
:10BA00008111ECCF4CE0C835D40710F491959883A0
:10BA1000872FDF91CF911F910F91FF90089520E024
:10BA20000C945D5CEF92FF920F931F93CF93DF9383
:10BA3000F62E122F902F9071E92EEA01112369F052
:10BA4000EE2011F0488102C0FE014491202F6F2D9D
:10BA50000E945D5C11502196F1CFDF91CF911F9133
:10BA60000F91FF90EF9008950F93FA0194914F5F1B
:10BA70005F4F929F400D511D1124292F0E94125D8E
:10BA80000F9108950F9300E00E94125D0F910895A9
:10BA9000FF920F931F93CF93DF93062F122F922FB6
:10BAA0009071F92EFA01FF2011F0408101C04491FC
:10BAB000EF012196442331F0212F602F0E945D5C1D
:10BAC000FE01F1CFDF91CF911F910F91FF9008956B
:10BAD000AB0120E0682F80E00C94485D20E00C94DE
:10BAE000485DFF920F931F93CF93DF93082FF62E9D
:10BAF000EA0114E1180F15504C2F4F704A301CF01A
:10BB0000495C28E002C0405D20E06F2D812F0E943B
:10BB10005D5C34E0D695C7953A95E1F71013EBCF0D
:10BB2000DF91CF911F910F91FF900895222321F073
:10BB30009091590C96FD0895480F66956695669507
:10BB4000E82FF0E090E8699FE00DF11D1124E85A1C
:10BB5000F74F8E1B982F9E0F941720F4908190958D
:10BB60009193F8CF0895962F969596959695E82FF0
:10BB7000F0E080E8989FE00DF11D1124E85AF74F9E
:10BB80008CE0E835F80758F4677081E090E0062E05
:10BB900001C0880F0A94EAF790819827908308954E
:10BBA00047FF02C0840F4195962F969596959695DE
:10BBB000E82FF0E080E8989FE00DF11D1124E85A8D
:10BBC000F74F677031E001C0330F6A95EAF74423FD
:10BBD000B1F08CE0E835F80790F4822F90E020FF78
:10BBE00008C020812327208395958795282F2068DA
:10BBF00003C095958795282F41503196E8CF089539
:10BC00002FEF0C94D05D962F969596959695282FAC
:10BC100030E0F90180E8989FE00DF11D1124E85A09
:10BC2000F74F962F940F96959695969580E8989F46
:10BC3000200D311D1124285A374F862F8770A1E01F
:10BC4000B0E001C0AA0F8A95EAF7A1958081A827E4
:10BC5000A083E217F30750F4E058FF4F8CE0E8357B
:10BC6000F807E0F4908190959083F3CF8CE0E8356D
:10BC7000F807A0F4842F992787FD9095860F911DD2
:10BC800068E070E00E94806F21E030E001C0220F88
:10BC90008A95EAF7219580818227808308953F92D3
:10BCA0004F925F926F927F928F929F92AF92BF92CC
:10BCB000CF92DF92EF92FF920F931F93CF93DF9378
:10BCC000182FB62E802F05FF04C004FF04C002E029
:10BCD00003C000E001C001E0982F9F77C92EE7FE66
:10BCE00004C0E1946624639401C0612C57FF0AC02C
:10BCF00050954095309521953F4F4F4F5F4F77249A
:10BD0000739401C0712C82FF06C09CE09093580C84
:10BD1000CAE0DC2E05C096E09093580CB5E0DB2E0F
:10BD200086FF28C071101D0D283E83E038074105AD
:10BD3000510514F01D0D05C024363105410551058E
:10BD400014F01D0D05C02A303105410551050CF0D8
:10BD50001D0D002381F0023031F4243631054105F8
:10BD600051054CF41D0D2A303105410551051CF4D7
:10BD70001D0D01C01D198091580C810F8093580C26
:10BD8000023011F490EFC90E88248394F2E09F2EC4
:10BD9000A12CFF24E7FCF094A6E05A2E5B0CE82DC2
:10BDA000F0E0EE16FF060CF460C06AE070E0C90136
:10BDB0000E94806F382EEB01E0E34E2E480E2C2DB2
:10BDC000442D6B2D812F0E945D5C081131C0C2FE95
:10BDD0001AC08FEF830D833008F49394CE016AE08C
:10BDE00070E00E94806F823011F08430E9F484E3C7
:10BDF000481204C0AA24A394A10E17C0AA24AA948E
:10BE0000A10E939412C07EEF472E410E8FEF810F4B
:10BE1000C0FE05C047E06B2D0E94035E03C0652D88
:10BE20000E94B35D142D01C0A12E209709F000E0FF
:10BE30009E01442737FD4095542F211531054105BA
:10BE4000510581F4002331F0023059F491E0981546
:10BE500040F008C0C4FE09C0611004C080EFC80EE5
:10BE600001C000E01D1983949ACFAA2061F0492DEA
:10BE70006CE06B0D8A2D0E94005E492D6DE06B0D0C
:10BE80008A2D0E94005E772039F02C2D4DE26B2D1B
:10BE9000812F8D190E945D5C80E0DF91CF911F9111
:10BEA0000F91FF90EF90DF90CF90BF90AF909F9059
:10BEB0008F907F906F905F904F903F900895EF929A
:10BEC0000F93022F9A01442737FD4095542F95E098
:10BED000E92E0E944F5E0F91EF90089520E00C94A0
:10BEE0005F5F0F931F93CF93DF93182FC62F042FFD
:10BEF000D22F422F0E94035E023038F04D2F6C2F5C
:10BF00008FEF800F810F0E94035E02501F5F6FEF63
:10BF10006C0F6D0F402F812F0E94005E402F6C2F01
:10BF2000812FDF91CF911F910F910C94005E0F93A1
:10BF30001F93CF93DF93182FC62FD22FE42FF0E05B
:10BF40003297053608F004E60E9FC0010F9F900D52
:10BF5000112464E670E00E94806F062F2D2F6C2F55
:10BF6000812F0E94715F002369F0D150DC0FCF5FF9
:10BF70001F5FCD1738F4402F6C2F812F0E94005E79
:10BF8000CF5FF7CFDF91CF911F910F910895A998BF
:10BF9000AB98AC988BBBAD9AAD98AB9AA99A089523
:10BFA00081E080935708AA9825E02A95F1F70000D0
:10BFB00085E08A95F1F70000AA9A8CED95E025E0DE
:10BFC0002A95F1F7000001970097C9F782EE0E94C9
:10BFD000C75F8EEA0E94C75F81EA0E94C75F86EA58
:10BFE0000E94C75F84EA0E94C75F82EA0E94C75F1F
:10BFF00080EC0E94C75F8FE20E94C75F85E20E94CB
:10C00000C75F81E80E94C75F82E20E94C75F8FEA34
:10C010000E94C75F82E2809300051092570808953E
:10C02000CF93C82F81E08093570881E80E94C75FB3
:10C030008C2F0E94C75F10925708CF91089580916E
:10C0400000050C9410601F93CF93DF9381E08093E1
:10C05000570810E0C8E5D8E084E00E94C75F80E19F
:10C060000E94C75F812F806B0E94C75FA998AB9A1F
:10C07000AC98FE01CE0180589F4F20812BBBAD9A1A
:10C08000AD9821812BBBAD9AAD9822812BBBAD9A87
:10C09000AD9823812BBBAD9AAD983496E817F9077C
:10C0A00061F7EF01AB9AA99A1F5F1830A9F61092B9
:10C0B0005708DF91CF911F910895BF92CF92DF92E1
:10C0C000EF92FF920F931F93CF93DF937B018A012F
:10C0D000080F191FEC01E81AF90A6701CC0EDD1EE2
:10C0E000C017D107C1F0B9908091F8078270E19B29
:10C0F00005C08823E1F30E94ED1AF6CFDFBACEBA6D
:10C10000E09A8DB3B81649F3BDBA8FB7F894E29AA6
:10C11000E19A8FBFE2CFDF91CF911F910F91FF90F6
:10C12000EF90DF90CF90BF9008958091890C10928E
:10C13000890C0895FC0180818F70880F61118160E6
:10C140008F709081907F982B908381818F5F818306
:10C150008281882351F09F7041F4833621F0842F2F
:10C1600080628093890C118212828281883069F109
:10C1700048F4813091F188F0823039F1843009F04F
:10C180003FC023C08F35C1F018F48031F1F008951D
:10C19000813649F0823671F1089580818F708F3039
:10C1A00079F581E62BC040664093890C10926A06AF
:10C1B000109269068FE522C08181803211F44068B7
:10C1C00016C08832E9F480E119C09181903328F0DB
:10C1D00090E09595879582831182828190E0019706
:10C1E000218130E082239323892B51F440644093D2
:10C1F000890C08958181803418F088E0828311824F
:10C200000895282F30E02F3031056CF4F901EE0F3E
:10C21000FF1FE20FF31FE45AF34F90819F7081E0FC
:10C220009F3071F52EC090E0FC013F97E930F10599
:10C2300038F5E659FF4F0C94D56F91B194701DC03D
:10C2400093B390781AC090916300917016C090914A
:10C2500063009095987011C08091630083FF10C0B7
:10C2600091B102C091B19095907407C091B1907155
:10C2700004C093B3F9CF91B1907281E0911101C0E4
:10C2800080E008958F7090E08F30910551F0FC01AF
:10C29000EE0FFF1FE80FF91FE45AF34F82E6828387
:10C2A000118208958F7090E08F30910549F0FC0164
:10C2B000EE0FFF1FE80FF91FE45AF34F83E6828366
:10C2C0000895EF92FF920F931F93CF93DF93809186
:10C2D0005A0C90915B0C019690935B0C80935A0CD6
:10C2E0008093590C16B31095CCE5DCE0F12C11FBD2
:10C2F000662760F94F2DCE010E949A60F39416953F
:10C30000239686E0F812F3CFE0B2E094CEE4DCE1CD
:10C3100000E010E0FC1AFE0184914C2F4F0D8E219D
:10C3200061E009F460E0C8018259934F0E949A606D
:10C3300021960D5F1F4F0831110569F79091CC01CF
:10C3400061E0C92FC07295FF60E04EE086E89CE096
:10C350000E949A6086B390E0809590958E77992799
:10C360008C2B19F089E080937001DF91CF911F91A0
:10C370000F91FF90EF900895EF92FF920F931F930C
:10C38000CF93DF93F82E80E04AE0282F30E0429FE1
:10C39000F001439FF00D1124EB51FE4F928DF916E1
:10C3A00050F5803261F18AE0E82EE29E8001E39E42
:10C3B000100D1124E801C150DE4F6FE170E0621BE7
:10C3C000730BE69EA001E79E500D11242F5F3F4F97
:10C3D000E29EC001E39E900D1124BE0181509E4F4C
:10C3E0000E94EA6FFE011192EA94E9F7F801EB511D
:10C3F000FE4FF28E06C09923A1F28F5FC6CFCFEF1A
:10C40000D1E0CE01DF91CF911F910F91FF90EF907E
:10C41000089580E491E0EFEFF1E0DF019C011D92CF
:10C4200021503040E1F7089588E2EBECF3E0DF01C2
:10C430001D928A95E9F788E4E3EFF3E0DF011D92AE
:10C440008A95E9F70895FB018830A8F029E0829FDA
:10C45000C00111248B519E4F20E030E04191DC015E
:10C46000A20FB31FAA53BE4F4C932F5F3F4F2930EB
:10C470003105A1F7089525E0829FC00111248B5159
:10C480009E4F20E030E04191DC01A20FB31FAA5182
:10C49000BE4F4C932F5F3F4F25303105A1F70895D4
:10C4A00090E00197FC01EE0FFF1FE80FF91FDF017D
:10C4B000A35CBB4F6F708C91807F862B8C93EB516C
:10C4C000FE4FDF01AA5ABD4F4C93E95AFD4F20831E
:10C4D000089590911605E82FF0E084E0989FE00D14
:10C4E000F11D1124E05CFC4F849108958F929F927E
:10C4F000AF92BF92CF92DF92EF92FF920F931F9372
:10C50000CF93DF93CDB7DEB76D970FB6F894DEBF4C
:10C510000FBECDBFF82E85E0EAE2F1E0DE015596D0
:10C5200001900D928A95E1F785E0EFE2F1E0DE01FE
:10C53000509601900D928A95E1F785E0E4E3F1E0F1
:10C54000DE011B9601900D928A95E1F785E0E9E303
:10C55000F1E0DE01169601900D928A95E1F785E0F3
:10C56000EEE3F1E0DE01119601900D928A95E1F77C
:10C570001A8E1B8E1C8E1D8EE0911B05F0E0E75A73
:10C58000FC4F46E050E0A1E0E4910E2F10E021E0E6
:10C5900030E0C801042E02C0959587950A94E2F711
:10C5A00083709927BC016F5F7F4FEAE1F0E0EC0FE9
:10C5B000FD1F8E0F9F1F6217730711F4FC01A083EC
:10C5C0002F5F3F4F25303105B1F7AF5F4250510922
:10C5D000A530E9F6F11028C00E9409628A8D0E94F8
:10C5E000BC618C0181E00E946962F801818354E69C
:10C5F000F52EF2828B8D0E94BC618C0182E00E943C
:10C600006962F8018183F2828C8D0E94BC618C0189
:10C6100083E00E946962F8018183F2828D8D0E941D
:10C62000BC618C0184E08AC0F1E0FF120EC08C8DE9
:10C630000E94BC61FC0188E081838CE98283F382E3
:10C640008781897F84608783F2C182E0F81249C0C4
:10C650008C8D0E94BC61FC0118E011833CE9E32E43
:10C66000E28285E183838781897F846087838EE08E
:10C670000E94BC6102E2FC01018344E6F42EF282D6
:10C680008EE00E94BC61FC011183E28284E183831D
:10C690008781897F846087838EE00E94BC61FC0172
:10C6A0001183F28281E083838781897F846087831D
:10C6B00083E00E94696290915B04907F9260909306
:10C6C0005B04809359048DE980935A0480915E0441
:10C6D000807F816080935E0400935C0410925D040F
:10C6E000A6C1F3E0FF1230C00E940962EA8C8E2DD1
:10C6F0000E94BC618C0181E00E946962F801818323
:10C7000024E6F22EF2828E2D0E94BC618C0182E022
:10C710000E946962F80181838CE98283EB8C8E2D03
:10C720000E94BC618C0181E00E946962F8018183F2
:10C73000F2828E2D0E94BC618C0182E00E946962AF
:10C74000F8018183F28273C1F4E0FF1230C00E94CD
:10C750000962EB8C8E2D0E94BC618C0182E00E94EC
:10C760006962F801818394E6F92EF2828E2D0E948F
:10C77000BC618C0184E00E946962F8018183F282CD
:10C78000ED8C8E2D0E94BC618C0182E00E9469625A
:10C79000F8018183F2828E2D0E94BC618C0184E0BD
:10C7A0000E946962F80181838CE9828340C1F5E0CF
:10C7B000FF12D1C00E9409620E94146281E00E94AF
:10C7C000BC615AE0B52EFC01B18264E6D62ED2825D
:10C7D00082E00E94BC617BE0C72EFC01C182D28254
:10C7E00083E00E94BC61ECE0EE2EFC01E182D2828B
:10C7F00084E00E94BC618C0181E00E946962F801C2
:10C800008183D28285E00E94BC618C0183E00E941A
:10C810006962F8018183D282A4E0AA2EA38287E014
:10C82000848387818160878385E00E94BC618C015D
:10C8300083E00E946962F8018183D282F382B8E0CA
:10C840008B2E848287818160878385E00E94BC6112
:10C850008C0183E00E946962F8018183D28216E034
:10C86000D12ED38209E0902E9482878181608783C4
:10C8700085E00E94BC61FC0181828CE9828381E0B9
:10C8800083838781897F8460878386E00E94BC617F
:10C89000FC0191828EE1828388EF83838BE00E948A
:10C8A000BC618C0183E00E946962F801818386E4A7
:10C8B000982E9282A382B4828781816087838BE0E5
:10C8C0000E94BC618C0183E00E946962F80181834F
:10C8D0009282F382C4828781816087838BE00E9489
:10C8E000BC618C0183E00E946962F80181839282BD
:10C8F000D382E4828781816087838091FB018F717D
:10C9000080628093FB018FE18093FC01BE016B5E2E
:10C910007F4F80E00E942362BE01605F7F4F81E015
:10C920000E942362BE01655F7F4F82E00E94236206
:10C93000BE016A5F7F4F83E00E942362BE016F5F8A
:10C940007F4F84E00E942362BE016F5F7F4F85E0CE
:10C950000E9423626CC0F6E0FF1216C086E00E94BF
:10C96000BC61FC01F18282E3828388EF838314E659
:10C97000108786E00E94BC61FC01F1828EEC82830C
:10C9800088E08383108753C087E0F81250C08FE09F
:10C990000E94BC61FC0114E2118384E6828388E872
:10C9A000868380E10E94BC61FC0189E081830EE600
:10C9B00002838AE0838380E10E94BC61FC0148E03D
:10C9C000F42EF18282E982838BE083838781897FE1
:10C9D0008460878380E10E94BC61FC01F182028354
:10C9E0008CE083838781897F8460878380913D0485
:10C9F000807F8B6080933D0493E290933B0410937F
:10CA00003C0480914004807F816080934004909337
:10CA10003E0489E680933F0480914304807F8260D6
:10CA2000809343049093410487E98093420482E019
:10CA30000E94A5570E9444586D960FB6F894DEBF29
:10CA40000FBECDBFDF91CF911F910F91FF90EF905F
:10CA5000DF90CF90BF90AF909F908F9008950F93ED
:10CA60001F93CF93DF939091FB0191FF03C060E090
:10CA700075E002C060E074E01091F6011295169521
:10CA80001770882331F0AEEDBCE0833021F420E153
:10CA900003C0A6E9BCE028E09091F501990F910F41
:10CAA000920F4091F80124E64202A0011124485A55
:10CAB0005D4F0091FE01E8EEF3E09F010203E0010B
:10CAC000039FD00D11249E0128533045241B350BA4
:10CAD000FD01882339F032964D935C93833011F435
:10CAE00018EF190FCC27DD27C61BD70B1917F0F449
:10CAF000A12FB0E0AA0FBB1FA55AB84F0D90BC9153
:10CB0000A02D6A177B070CF4DB01AC17BD070CF4F2
:10CB1000DE01A854B44F2A1B3B0BA41BB50BB183F9
:10CB2000A083538342831F5F3496E0CF31832083F9
:10CB3000DF01882371F01296285E33403093920C07
:10CB40002093910C1D921C92DF91CF911F910F9118
:10CB50000895149653834283F5CFE0912601F09116
:10CB6000270129E090E130E0482F4170341302C0E2
:10CB7000905F04C091509083319690E186958068D3
:10CB8000215011F0342FF0CF915F9193F093270152
:10CB9000E093260108951F93CF93DF93182F26E982
:10CBA0003CE03093270120932601C09114018C2F83
:10CBB000877461F08091F501882321F0813021F4A0
:10CBC000C0E906C0C0E804C0C8E902C0C7FF06C08B
:10CBD00087E10E940161882309F45AC0C7FD5AC049
:10CBE00040E060E085E10E941316882309F452C0FA
:10CBF000C062C09314018091FF048F5F8093150180
:10CC0000E7E1F1E0ABE5B7E090E06DE0911729F1E5
:10CC10004D915D91649F9001659F300D112485E0D9
:10CC2000359527958A95E1F73E5F37FD06C02F3F82
:10CC300083E038072CF4822F05C080E030E002C08A
:10CC40008FEF33E0EF012197292F220F220F232BA3
:10CC5000288380839F5F3296D9CFC4E1D1E0899148
:10CC60000E94AD6581E0C232D807C9F7E091260184
:10CC7000F0912701108231978FEF808386E99CE045
:10CC80009093250180932401DF91CF911F91089506
:10CC9000CF77A4CFCF7DADCF1F920F920FB60F925B
:10CCA00011242F938F939F93EF93FF9388B391E079
:10CCB000892788BBE0912401F0912501CF010196DD
:10CCC00090932501809324012081822F90E097BDCD
:10CCD00086BD293C08F0C09A8091950C81608093B4
:10CCE000950CFF91EF919F918F912F910F900FBE17
:10CCF0000F901F9018951F920F920FB60F9211244C
:10CD00002F933F938F939F93EF93FF9388B391E07B
:10CD1000892788BBE0912601F0912701808128B501
:10CD200039B580FD03C0205E3F4F02C0205F3F4FFA
:10CD300039BD28BD90E095958795009791F4CF0176
:10CD400001969093270180932601818181110AC069
:10CD500080917800909179008053984F99BD88BD5B
:10CD600001C080838091950C81608093950CFF9128
:10CD7000EF919F918F913F912F910F900FBE0F9048
:10CD80001F901895EDE7F0E08081857E80831798ED
:10CD90001F9AAAE8B0E01C9210928B0082E88C9354
:10CDA0008081806280830895EDE7F0E080818F7D4F
:10CDB0008083179AAAE8B0E01C9210928B008AE058
:10CDC0008C9380818861808308951F920F920FB6A3
:10CDD0000F9211248F939F93EF93FF938091260DD1
:10CDE000882321F01F9A1092260D04C01F9881E01D
:10CDF0008093260DE0911201F091130180819181C1
:10CE000090938700809386008091910C9091920C72
:10CE1000909385008093840082819381892B11F007
:10CE2000329607C08091FB0181708093260DEEED54
:10CE3000FCE0F0931301E09312018091950C816066
:10CE40008093950CFF91EF919F918F910F900FBE62
:10CE50000F901F901895EAE8FCE020812695269512
:10CE6000282B208381818F5F8183843048F0A281C9
:10CE7000B381CD010196938382832C93108211821A
:10CE80000895882339F08091900C8F5F8093900CE7
:10CE900080E803C01092900C80EC0E942B67809178
:10CEA000900C8530B8F70895CF93DF93C82FE091A9
:10CEB0008E0CE827F0E0EE0FFF1FE654F34E2591AD
:10CEC000349140918F0C50E02427352730938F0CFC
:10CED00020938E0CD8E08C2F80780E944167CC0F75
:10CEE000D150C9F7DF91CF910895CF9380EC0E9484
:10CEF0002B67C6E080E80E942B67C150D9F780EC11
:10CF0000CF910C942B67EF92FF920F931F93CF93C7
:10CF1000DF93C091F40180911E0585FF04C08091CC
:10CF2000E1018111C4E08091940C8C1709F48EC04A
:10CF3000C093940C1EBC1DBC1CBC87B7837C87BFF0
:10CF400080917D008E7F80937D008CE386BF8FE390
:10CF500080937C00C23079F118F4C130A1F006C092
:10CF6000C33009F444C0C43009F45DC00E94C266F5
:10CF700080E49CE99BBD8ABD87B7806187BF1FBCE9
:10CF80008AE08EBD63C00E94C26680E797E199BDCA
:10CF900088BD80EA9FE0909379008093780087B7FE
:10CFA000886087BF80917D00816080937D001FBC79
:10CFB00082E08EBD56C00E94C26688EC90E09093DD
:10CFC0007900809378008CE291E09DBD8CBD80EE6D
:10CFD0009BEA97BD86BD87B7806287BF80917D0041
:10CFE000816080937D001FBC8AE18EBDB9C080E462
:10CFF0009CE99BBD8ABD87B7806187BF1FBC8AE063
:10D000008EBD83E00E942F6580E593EC90938700AE
:10D010008093860088E893E1909385008093840054
:10D020000E94D466A7C084E00E942F6580E593EC3F
:10D03000909387008093860088E893E19093850021
:10D04000809384000E94D466C0989DC0C13049F08E
:10D0500008F490C0C23009F483C0C33009F48AC018
:10D0600092C07894EAE8FCE086E99CE0909327017E
:10D070008093260193838283158214821082118209
:10D0800016820E9475678091F5010E945467809115
:10D09000930C0E94546780E00E9454671092930C96
:10D0A000CBE5D7E028813981C901880F991F820F0C
:10D0B000931F97FD03967C01F594E794F594E7940C
:10D0C00086E3E81A87EFF80A2A813B81C901880FB5
:10D0D000991F820F931F97FD03968C011595079555
:10D0E000159507950653174F8E2D0E9454679F2D57
:10D0F0009F70802F8295807F892B0E945467C80182
:10D1000054E0969587955A95E1F70E9454672496C6
:10D1100087E0CB36D80731F6C0918E0C80918F0C0A
:10D120000E9454678C2F0E9454670E9475678091FB
:10D130008B0C882321F080E00E942B67F8CFE091D0
:10D140008C0CF0918D0C1082809178009091790078
:10D15000805C93469093790080937800C09A13C0C6
:10D16000789486E0DF91CF911F910F91FF90EF901F
:10D170000C94CB6580E0DF91CF911F910F91FF90D0
:10D18000EF900C942F65DF91CF911F910F91FF903D
:10D19000EF9008951F920F920FB60F9211242F93C4
:10D1A0003F934F935F936F937F938F939F93AF932F
:10D1B000BF93CF93DF93EF93FF938CB59DB52091F1
:10D1C000270D222321F0C09A1092270D04C0C09889
:10D1D00021E02093270DC0912201D09123019E01CF
:10D1E0002E5F3F4F30932301209322012881398104
:10D1F0003BBD2ABDE0E1F1E0282F3181381708F46A
:10D2000081833081231708F480838A819B81892B55
:10D21000D9F486E99CE090932301809322018091C8
:10D22000FB01809581708093270D87B78F7E87BF24
:10D230000E9483678091F401882311F0833021F4E8
:10D2400087B7806187BF78948091950C81608093C7
:10D25000950CFF91EF91DF91CF91BF91AF919F918D
:10D260008F917F916F915F914F913F912F910F908F
:10D270000FBE0F901F9018951F920F920FB60F922E
:10D2800011242F933F934F935F936F937F938F93CB
:10D290009F93AF93BF93EF93FF938091F4018230FC
:10D2A000C1F480E492EA97BD86BD809178009091A8
:10D2B00079008F3F910538F488E598E990937900DB
:10D2C0008093780008C088EC90E090937900809378
:10D2D00078000E948367FF91EF91BF91AF919F917A
:10D2E0008F917F916F915F914F913F912F910F900F
:10D2F0000FBE0F901F9018951F920F920FB60F92AE
:10D3000011242F933F934F935F936F937F938F934A
:10D310009F93AF93BF93EF93FF938091F401789421
:10D320009091940C981771F0943061F48091E10120
:10D33000882321F080911E0585FD03C00E9483672C
:10D3400003C084E00E942F65FF91EF91BF91AF91E0
:10D350009F918F917F916F915F914F913F912F910D
:10D360000F900FBE0F901F90189590911505987310
:10D37000903129F49BEA899F812D112402C09831B4
:10D3800011F486950895983211F4880F089590331A
:10D3900019F4982F990F890F0895FC01A5E6B0E0C4
:10D3A0008C918B7F8C93148215821082118216A629
:10D3B00017A608950C94CD6921E0FC0184818111A8
:10D3C00001C020E0822F0895FC0121818081281B6B
:10D3D000277098E0921B81E0933008F480E0089574
:10D3E000CF93DF93FC0184818823F1F08150848303
:10D3F00082819381890F828386A58823F1F187A595
:10D400009FEF980F97A7882331F080916500846083
:10D410008093650032C0809165008B7F80936500AA
:10D420008091200587A729C01B98809165008B7F7C
:10D43000809365008581882319F0815085831DC004
:10D44000808191818917C9F090E0EF01C80FD91F41
:10D450002E8122832E8924832E8523832E8D25835E
:10D4600028A926A717A62EA13FEF320F3EA3211110
:10D4700004C00196877099278083DF91CF9108952A
:10D480008F929F92AF92BF92CF92DF92EF92FF92D4
:10D490000F931F93CF93DF935C01162FD42EF22EA0
:10D4A0000E94E469882339F190911505987319F168
:10D4B000F501C181D0E04E01FFEF8F1A9F0A87E08E
:10D4C00088229924F50180818815A9F0112329F07B
:10D4D00090911F05965F910F01C090E0CA0DDB1D72
:10D4E0009E838D2D0E94B5698E8BFE8EE8AA0EA3B9
:10D4F000CE86F5018182DF91CF911F910F91FF9030
:10D50000EF90DF90CF90BF90AF909F908F90089555
:10D51000CF92DF92EF92FF920F931F93CF93DF93FF
:10D52000EC01162FF42ED22E0E94E469882301F11B
:10D53000909115059873E1F0112329F090911F0542
:10D54000965F910F01C090E09A838F2D0E94B5697C
:10D550008C83DD82EEA61FA6CB828881898300237F
:10D5600039F001502D2D4F2D612FCE010E94406AC0
:10D57000DF91CF911F910F91FF90EF90DF90CF90AF
:10D580000895CF92EF920F931F93CF93DF93EC0107
:10D59000062F642F80911505869586958695877050
:10D5A00038812981321364C110E00132110508F07D
:10D5B0005FC1F801ED58FF4F0C94D56FC12CEE24DC
:10D5C000E39400E021E03AC1C12CEE24E39400E0B2
:10D5D00021E02EC1C12CEE24E39400E021E04EE1D5
:10D5E0002EC192E0C92EEE24E39402E022E04AE04C
:10D5F00064E63BC1C12CEE24E3940AE022E045E05E
:10D600006FE5CE010E94406A01E02AE045E06FE547
:10D61000CE010E94406A0AE022E045E06FE525C1A4
:10D62000CC24CA94E12C02E023E04AE060E5CE017C
:10D630000E94406ACC24C39423E04AE06CE3CE010C
:10D640000E94406AC12C82E0E82E00E021E04AE01E
:10D650006FC0C12CEE24E39401E021E045E066E4D4
:10D66000CE010E94406A22E04FE062E3CE010E94B8
:10D67000406A22E04FE0F8C0C12CEE24E39402E0BF
:10D6800021E045E06EE6CE010E94406A03E021E021
:10D6900045E06CE7EAC0C12CE12C00E025E045E064
:10D6A00062E3CE010E94406A25E045E06AE5CE01D2
:10D6B0000E94406A02E024E043E06EE6D6C0C12C3E
:10D6C000EE24E39403E02AE045E060E5CE010E9409
:10D6D000406A01E024E145E060E5CE010E94406A35
:10D6E00003E02AE045E0C0C0CC24C394EE24E394D8
:10D6F00002E025E044E16AE0B8C0C12CEE24E394E6
:10D7000002E02AE044E062E3CE010E94406A01E0C8
:10D7100024E148E066E4CE010E94406A02E02AE08B
:10D7200048E062E3CE010E94406A01E024E144E067
:10D7300066E49BC0C12CEE24E3940AE02AE005C015
:10D74000C12CEE24E39402E022E345E068E78DC0BB
:10D75000C12CEE24E39401E009C0C12CEE24E39433
:10D7600002E004C0C12CEE24E39403E02AE044E18B
:10D7700060E07BC0C12CEE24E39400E021E048E2AD
:10D780005EC0813009F474C0C12CE12C00E021E0BE
:10D790004AE06BE455C0813009F46AC0C12CE12C29
:10D7A00000E021E04AE061E44BC0C12CE12C00E044
:10D7B00021E046E045C0C12CEE24E39405C0813051
:10D7C00009F456C0C12CE12C00E037C0C12CE12C7B
:10D7D00000E004C0C12CEE24E39401E021E04AE023
:10D7E00020C0C12CEE24E39402E021E04AE06AE785
:10D7F00027C0C12CEE24E39403E021E04AE06CE76B
:10D800001FC0C12CEE24E39403E009C0C12CEE2418
:10D81000E39402E004C0C12CEE24E39401E023E091
:10D820004FE068E70DC0C12CEE24E39401E029E14C
:10D8300044E105C0C12CE12C02E022E04AE066E4AC
:10D84000CE010E94886A14C0CC24C394E12C02E06B
:10D8500023E044E16CE3CE010E94406ACC24CA94E8
:10D86000EE24E39423E044E160E5CE010E94406AA7
:10D87000DF91CF911F910F91EF90CF90089546E4E3
:10D88000682F8FE891E00C94C16A9091210591FF77
:10D8900003C0862F0C9464130C943F6CFF920F937B
:10D8A0001F93CF93DF93EC01162FF42E47FF03C095
:10D8B000842F0E946413D7FF06C0D195C195D1096A
:10D8C0008AE10E946413112371F0123019F464E6A6
:10D8D00070E002C06AE070E0CE010E94806F262FE7
:10D8E000C22FD72F082F64E670E0CE010E94806F10
:10D8F0009B01562F482FC82FD92F2115310551F1E3
:10D900002A303105DCF06AE070E0C9010E94806FC6
:10D910009B018C01EC01653171051CF48EE6820FD0
:10D9200005C08CE8820F0E945F138EE60E9464138C
:10D930000115110559F1502F11E001C010E084E6E6
:10D94000850F0E946413111121C02097F9F08C2FCC
:10D95000845715C08CE8840F0E945F131123B1F027
:10D96000123081F46AE070E0802F90E00E94806FB6
:10D97000C82F86E0860F0E9464138CE88C0F0E94EB
:10D980005F1304C086E0800F0E9464131F1444F4E8
:10D990008F2DDF91CF911F910F91FF900C94641305
:10D9A000DF91CF911F910F91FF9008951F920F92D9
:10D9B0000FB60F9211242F933F938F939F93EF9362
:10D9C000FF938BB19AB12CB18C7129F01092520D4A
:10D9D0001092730D1AC091FD08C02E3FB9F32F3F6E
:10D9E000A1F481E08093520D10C08091730D8032BC
:10D9F00060F431E0380F90E03093730DFC01ED5A84
:10DA0000F24F2F3D09F420E42083FF91EF919F9185
:10DA10008F913F912F910F900FBE0F901F901895EF
:10DA200080EF90E090932901809328011098189836
:10DA30001092900087E689B9599886E38093950003
:10DA400084E08AB95F9B02C08CB1FCCF08955398E3
:10DA50000895539A0895549857980895549A579A48
:10DA600008955D9BFECF509890FD509A8CB9089513
:10DA70005D9BFECF509A8CB90895CF93DF93EC0154
:10DA80008991882319F00E94386DFACFDF91CF91E8
:10DA900008955D9BFECF50988EEF8CB908955D9BE5
:10DAA000FECF50988FEF8CB9089586B380958E770E
:10DAB00008958FEF8ABB1BBA91E897BB9EE798BB8E
:10DAC0009EE394BB91EC95BB11BA82BB88E082B90E
:10DAD00087EF83B9109261001092620084E1809315
:10DAE00064008BEF809365000E94D05F0E94106DF0
:10DAF00080E487B985E886B987E083BF8CE981BF78
:10DB000082E085BD87B7836487BF1FBC8AE08EBD76
:10DB100010928B0082E880938A0080917D00806261
:10DB200080937D0078948DE69FE3909367018093C6
:10DB3000660189E10E9410600E943357D090FF0473
:10DB40000E94556DC0E081FD05C08695CF5FC7304E
:10DB5000D1F71FC0C630E9F08C2F0E94A45688234D
:10DB6000C1F0C093FF048C2F0E94A75681E00E9451
:10DB7000A5570E940D5C24E049EA51E060E086E18F
:10DB80000E94485D88E10E9491110E9423600E94DA
:10DB900058110E941F6081E0809356010E94331744
:10DBA000109256010E9467138091180584FF05C0EA
:10DBB0008091150582FD4FC044C0809121058823C6
:10DBC00021F06CE187E00E94456C0E9412170E94D0
:10DBD0000D5C20E048E753E060E080E00E94185CC4
:10DBE00080911E0584FD08C000E12AE043E255E073
:10DBF00068E380E00E94125D0E9423600E941F6023
:10DC00000E9458110E94880F0E945A148C01F894A7
:10DC1000C0915A0CD0915B0C7894C057DE4F0E9493
:10DC200023600E9412170E94880F0E945A147C01E0
:10DC30000E94556D8111BCCFE016F10609F4F9C0C0
:10DC4000B7CF0E94B858883C910528F460E08AE973
:10DC500091E00E944A1A0E94880F8091150580FD6C
:10DC600039C080911605817012E0181B0E94880F40
:10DC7000E12FF0E0EE0FFF1FEE52FB4F21813281CA
:10DC80008091180580FF06C0319521953109458D99
:10DC9000568D02C047855089241B350BE9016096DB
:10DCA000812F0E947414C817D907A4F46BE871E09F
:10DCB00089E791E00E945F110E94880F0E9412176D
:10DCC000812F0E947414C817D90724F40E94556D3F
:10DCD000882391F3D0912D058091150581FD56C0C3
:10DCE0008D2F8873883041F0803131F0803221F0FF
:10DCF000D77CD860D0932D0516E1C0E0812F0E941B
:10DD00000161CC0FC82B11501E30C1F71C2F1D27ED
:10DD100063E671E082E892E10E945F1110FF04C0A7
:10DD200060E082E00E94851111FF04C063E087E19A
:10DD30000E94851112FF04C066E08CE20E948511EA
:10DD4000812F887371F0C3FF02C069E007C0C4FF70
:10DD500002C06CE003C0C5FF04C06FE081E40E9414
:10DD6000851116FF04C062E186E50E94851117FF48
:10DD700004C065E18BE60E9485110E942360CD17E7
:10DD800029F00E94556D882309F45EC08091150525
:10DD9000887B29F460E083E591E00E944A1A809133
:10DDA0008E01882351F060E088E291E00E944A1AD7
:10DDB00080918E018E7F80938E010E94581180EF9A
:10DDC00090E090930101809300018091EF010E9407
:10DDD0005F130E9483672DE088E190E00FB6F8940E
:10DDE000A89581BD0FBE21BD60E08BE597E00E9444
:10DDF0009E368EE690E390936901809368010E94BD
:10DE00001F608091FF04D81629F081E00E94A55779
:10DE10000E94445880ED97E09BBD8ABD80E186BF9B
:10DE200081E08093E20187B7806187BF0E94ED1A8D
:10DE3000FDCFF89480915A0C90915B0C7894C817A0
:10DE4000D90709F0ECCEB4CE0E94121755CF8FE857
:10DE500091E00C94DA690E94336F332312F48A1B29
:10DE60009B0B0C94446FA29FB001B39FC001A39F72
:10DE7000700D811D1124911DB29F700D811D112403
:10DE8000911D08950E94336FB7FF0895821B930B75
:10DE900008950E94336FA59F900DB49F900DA49F8D
:10DEA000800D911D11240895B7FF0C94496F0E94B5
:10DEB000496F821B930B0895DB018F939F930E9400
:10DEC000496FBF91AF91A29F800D911DA39F900DAF
:10DED000B29F900D11240895AA1BBB1B51E107C0EE
:10DEE000AA1FBB1FA617B70710F0A61BB70B881FEA
:10DEF000991F5A95A9F780959095BC01CD01089579
:10DF000097FB072E16F4009407D077FD09D00E94E6
:10DF10006C6F07FC05D03EF4909581959F4F089556
:10DF2000709561957F4F0895A1E21A2EAA1BBB1B25
:10DF3000FD010DC0AA1FBB1FEE1FFF1FA217B307D5
:10DF4000E407F50720F0A21BB30BE40BF50B661FEB
:10DF5000771F881F991F1A9469F7609570958095AF
:10DF600090959B01AC01BD01CF010895052E97FB53
:10DF70001EF400940E94CD6F57FD07D00E94946F4D
:10DF800007FC03D04EF40C94CD6F5095409530951E
:10DF900021953F4F4F4F5F4F089590958095709515
:10DFA00061957F4F8F4F9F4F0895EE0FFF1F059094
:10DFB000F491E02D0994FB01DC014150504048F000
:10DFC00005900D920020C9F701C01D9241505040AC
:10DFD000E0F708956817790768F4FB01DC01E40FA6
:10DFE000F51FA40FB51F02C002900E924150504081
:10DFF000D8F708950C941370DC0101C06D93415063
:10E000005040E0F70895DC01CB01FC01E199FECF1F
:10E0100006C0FFBBEEBBE09A31960DB20D924150A7
:10E020005040B8F70895FB01DC0102C001900D9249
:0CE0300041505040D8F70895F894FFCFFD
:10E03C00F0004AC703C803C903CA036400000A02FC
:10E04C00FF00DE0CFF0000AA05FF09FF0DFF1354B3
:10E05C0014AA960C960C960CF0009CEC1E465A508A
:10E06C00463C4664645A505A64E2F10032649CCED9
:04E07C00003264000A
:00000001FF
